Archive member included to satisfy reference by file (symbol)

C:/nxp/SDKPackages/SDK_2.6.0_K32W061DK6/middleware/wireless/ieee-802.15.4/lib\libMiniMac.a(MMAC.o)
                              ./source/tis_trp_dut.o (vMMAC_Enable)
C:/nxp/SDKPackages/SDK_2.6.0_K32W061DK6/middleware/wireless/ieee-802.15.4/lib\libMiniMac.a(MMAC_RadioInit_JN518x.o)
                              ./source/tis_trp_dut.o (vMMAC_ConfigureRadio)
C:/nxp/SDKPackages/SDK_2.6.0_K32W061DK6/middleware/wireless/framework/XCVR/lib\libRadio_Test_JN518x.a(radio.o)
                              C:/nxp/SDKPackages/SDK_2.6.0_K32W061DK6/middleware/wireless/ieee-802.15.4/lib\libMiniMac.a(MMAC.o) (u8Radio_GetEDfromRSSI)
C:/nxp/SDKPackages/SDK_2.6.0_K32W061DK6/middleware/wireless/framework/XCVR/lib\libRadio_Test_JN518x.a(radio_test_jn518x.o)
                              ./Common/Command.o (vRadio_Test_Jn518x_TxPowerTest)
c:/nxp/mcuxpressoide_11.1.0_3209/ide/plugins/com.nxp.mcuxpresso.tools.win32_11.1.0.201909161352/tools/bin/../lib/gcc/arm-none-eabi/8.3.1/thumb/v7e-m/nofp\libgcc.a(_arm_addsubdf3.o)
                              C:/nxp/SDKPackages/SDK_2.6.0_K32W061DK6/middleware/wireless/framework/XCVR/lib\libRadio_Test_JN518x.a(radio.o) (__aeabi_dadd)
c:/nxp/mcuxpressoide_11.1.0_3209/ide/plugins/com.nxp.mcuxpresso.tools.win32_11.1.0.201909161352/tools/bin/../lib/gcc/arm-none-eabi/8.3.1/thumb/v7e-m/nofp\libgcc.a(_arm_fixdfsi.o)
                              C:/nxp/SDKPackages/SDK_2.6.0_K32W061DK6/middleware/wireless/framework/XCVR/lib\libRadio_Test_JN518x.a(radio.o) (__aeabi_d2iz)
c:/nxp/mcuxpressoide_11.1.0_3209/ide/plugins/com.nxp.mcuxpresso.tools.win32_11.1.0.201909161352/tools/bin/../lib/gcc/arm-none-eabi/8.3.1/thumb/v7e-m/nofp\libgcc.a(_aeabi_ldivmod.o)
                              ./drivers/fsl_clock.o (__aeabi_ldivmod)
c:/nxp/mcuxpressoide_11.1.0_3209/ide/plugins/com.nxp.mcuxpresso.tools.win32_11.1.0.201909161352/tools/bin/../lib/gcc/arm-none-eabi/8.3.1/thumb/v7e-m/nofp\libgcc.a(_aeabi_uldivmod.o)
                              ./drivers/fsl_clock.o (__aeabi_uldivmod)
c:/nxp/mcuxpressoide_11.1.0_3209/ide/plugins/com.nxp.mcuxpresso.tools.win32_11.1.0.201909161352/tools/bin/../lib/gcc/arm-none-eabi/8.3.1/thumb/v7e-m/nofp\libgcc.a(_udivmoddi4.o)
                              c:/nxp/mcuxpressoide_11.1.0_3209/ide/plugins/com.nxp.mcuxpresso.tools.win32_11.1.0.201909161352/tools/bin/../lib/gcc/arm-none-eabi/8.3.1/thumb/v7e-m/nofp\libgcc.a(_aeabi_ldivmod.o) (__udivmoddi4)
c:/nxp/mcuxpressoide_11.1.0_3209/ide/plugins/com.nxp.mcuxpresso.tools.win32_11.1.0.201909161352/tools/bin/../lib/gcc/arm-none-eabi/8.3.1/thumb/v7e-m/nofp\libgcc.a(_dvmd_tls.o)
                              c:/nxp/mcuxpressoide_11.1.0_3209/ide/plugins/com.nxp.mcuxpresso.tools.win32_11.1.0.201909161352/tools/bin/../lib/gcc/arm-none-eabi/8.3.1/thumb/v7e-m/nofp\libgcc.a(_aeabi_ldivmod.o) (__aeabi_ldiv0)
c:/nxp/mcuxpressoide_11.1.0_3209/ide/plugins/com.nxp.mcuxpresso.tools.win32_11.1.0.201909161352/tools/bin/../lib/gcc/arm-none-eabi/8.3.1/../../../../arm-none-eabi/lib/thumb/v7e-m/nofp\libg.a(lib_a-abs.o)
                              ./Common/Command.o (abs)
c:/nxp/mcuxpressoide_11.1.0_3209/ide/plugins/com.nxp.mcuxpresso.tools.win32_11.1.0.201909161352/tools/bin/../lib/gcc/arm-none-eabi/8.3.1/../../../../arm-none-eabi/lib/thumb/v7e-m/nofp\libg.a(lib_a-malloc.o)
                              ./drivers/fsl_common.o (malloc)
c:/nxp/mcuxpressoide_11.1.0_3209/ide/plugins/com.nxp.mcuxpresso.tools.win32_11.1.0.201909161352/tools/bin/../lib/gcc/arm-none-eabi/8.3.1/../../../../arm-none-eabi/lib/thumb/v7e-m/nofp\libg.a(lib_a-mallocr.o)
                              c:/nxp/mcuxpressoide_11.1.0_3209/ide/plugins/com.nxp.mcuxpresso.tools.win32_11.1.0.201909161352/tools/bin/../lib/gcc/arm-none-eabi/8.3.1/../../../../arm-none-eabi/lib/thumb/v7e-m/nofp\libg.a(lib_a-malloc.o) (_malloc_r)
c:/nxp/mcuxpressoide_11.1.0_3209/ide/plugins/com.nxp.mcuxpresso.tools.win32_11.1.0.201909161352/tools/bin/../lib/gcc/arm-none-eabi/8.3.1/../../../../arm-none-eabi/lib/thumb/v7e-m/nofp\libg.a(lib_a-memcpy.o)
                              ./drivers/fsl_power.o (memcpy)
c:/nxp/mcuxpressoide_11.1.0_3209/ide/plugins/com.nxp.mcuxpresso.tools.win32_11.1.0.201909161352/tools/bin/../lib/gcc/arm-none-eabi/8.3.1/../../../../arm-none-eabi/lib/thumb/v7e-m/nofp\libg.a(lib_a-memset.o)
                              ./utilities/fsl_debug_console.o (memset)
c:/nxp/mcuxpressoide_11.1.0_3209/ide/plugins/com.nxp.mcuxpresso.tools.win32_11.1.0.201909161352/tools/bin/../lib/gcc/arm-none-eabi/8.3.1/../../../../arm-none-eabi/lib/thumb/v7e-m/nofp\libg.a(lib_a-mlock.o)
                              c:/nxp/mcuxpressoide_11.1.0_3209/ide/plugins/com.nxp.mcuxpresso.tools.win32_11.1.0.201909161352/tools/bin/../lib/gcc/arm-none-eabi/8.3.1/../../../../arm-none-eabi/lib/thumb/v7e-m/nofp\libg.a(lib_a-mallocr.o) (__malloc_lock)
c:/nxp/mcuxpressoide_11.1.0_3209/ide/plugins/com.nxp.mcuxpresso.tools.win32_11.1.0.201909161352/tools/bin/../lib/gcc/arm-none-eabi/8.3.1/../../../../arm-none-eabi/lib/thumb/v7e-m/nofp\libg.a(lib_a-sbrkr.o)
                              c:/nxp/mcuxpressoide_11.1.0_3209/ide/plugins/com.nxp.mcuxpresso.tools.win32_11.1.0.201909161352/tools/bin/../lib/gcc/arm-none-eabi/8.3.1/../../../../arm-none-eabi/lib/thumb/v7e-m/nofp\libg.a(lib_a-mallocr.o) (_sbrk_r)
c:/nxp/mcuxpressoide_11.1.0_3209/ide/plugins/com.nxp.mcuxpresso.tools.win32_11.1.0.201909161352/tools/bin/../lib/gcc/arm-none-eabi/8.3.1/../../../../arm-none-eabi/lib/thumb/v7e-m/nofp\libg.a(lib_a-strlen.o)
                              ./drivers/fsl_str.o (strlen)
c:/nxp/mcuxpressoide_11.1.0_3209/ide/plugins/com.nxp.mcuxpresso.tools.win32_11.1.0.201909161352/tools/bin/../lib/gcc/arm-none-eabi/8.3.1/../../../../arm-none-eabi/lib/thumb/v7e-m/nofp\libg.a(lib_a-freer.o)
                              c:/nxp/mcuxpressoide_11.1.0_3209/ide/plugins/com.nxp.mcuxpresso.tools.win32_11.1.0.201909161352/tools/bin/../lib/gcc/arm-none-eabi/8.3.1/../../../../arm-none-eabi/lib/thumb/v7e-m/nofp\libg.a(lib_a-malloc.o) (_free_r)
c:/nxp/mcuxpressoide_11.1.0_3209/ide/plugins/com.nxp.mcuxpresso.tools.win32_11.1.0.201909161352/tools/bin/../lib/gcc/arm-none-eabi/8.3.1/../../../../arm-none-eabi/lib/thumb/v7e-m/nofp\libg.a(lib_a-impure.o)
                              c:/nxp/mcuxpressoide_11.1.0_3209/ide/plugins/com.nxp.mcuxpresso.tools.win32_11.1.0.201909161352/tools/bin/../lib/gcc/arm-none-eabi/8.3.1/../../../../arm-none-eabi/lib/thumb/v7e-m/nofp\libg.a(lib_a-malloc.o) (_impure_ptr)
c:/nxp/mcuxpressoide_11.1.0_3209/ide/plugins/com.nxp.mcuxpresso.tools.win32_11.1.0.201909161352/tools/bin/../lib/gcc/arm-none-eabi/8.3.1/../../../../arm-none-eabi/lib/thumb/v7e-m/nofp\libg.a(lib_a-lock.o)
                              c:/nxp/mcuxpressoide_11.1.0_3209/ide/plugins/com.nxp.mcuxpresso.tools.win32_11.1.0.201909161352/tools/bin/../lib/gcc/arm-none-eabi/8.3.1/../../../../arm-none-eabi/lib/thumb/v7e-m/nofp\libg.a(lib_a-mlock.o) (__retarget_lock_acquire_recursive)
c:/nxp/mcuxpressoide_11.1.0_3209/ide/plugins/com.nxp.mcuxpresso.tools.win32_11.1.0.201909161352/tools/bin/../lib/gcc/arm-none-eabi/8.3.1/../../../../arm-none-eabi/lib/thumb/v7e-m/nofp\libg.a(lib_a-reent.o)
                              c:/nxp/mcuxpressoide_11.1.0_3209/ide/plugins/com.nxp.mcuxpresso.tools.win32_11.1.0.201909161352/tools/bin/../lib/gcc/arm-none-eabi/8.3.1/../../../../arm-none-eabi/lib/thumb/v7e-m/nofp\libg.a(lib_a-sbrkr.o) (errno)

Allocating common symbols
Common symbol       size              file

u32LnaOffsetGainSav
                    0x4               C:/nxp/SDKPackages/SDK_2.6.0_K32W061DK6/middleware/wireless/framework/XCVR/lib\libRadio_Test_JN518x.a(radio.o)
__lock___atexit_recursive_mutex
                    0x1               c:/nxp/mcuxpressoide_11.1.0_3209/ide/plugins/com.nxp.mcuxpresso.tools.win32_11.1.0.201909161352/tools/bin/../lib/gcc/arm-none-eabi/8.3.1/../../../../arm-none-eabi/lib/thumb/v7e-m/nofp\libg.a(lib_a-lock.o)
tsMacFramePtRx      0x4               C:/nxp/SDKPackages/SDK_2.6.0_K32W061DK6/middleware/wireless/framework/XCVR/lib\libRadio_Test_JN518x.a(radio_test_jn518x.o)
__lock___arc4random_mutex
                    0x1               c:/nxp/mcuxpressoide_11.1.0_3209/ide/plugins/com.nxp.mcuxpresso.tools.win32_11.1.0.201909161352/tools/bin/../lib/gcc/arm-none-eabi/8.3.1/../../../../arm-none-eabi/lib/thumb/v7e-m/nofp\libg.a(lib_a-lock.o)
tCalTempValues      0x14              C:/nxp/SDKPackages/SDK_2.6.0_K32W061DK6/middleware/wireless/framework/XCVR/lib\libRadio_Test_JN518x.a(radio.o)
errno               0x4               c:/nxp/mcuxpressoide_11.1.0_3209/ide/plugins/com.nxp.mcuxpresso.tools.win32_11.1.0.201909161352/tools/bin/../lib/gcc/arm-none-eabi/8.3.1/../../../../arm-none-eabi/lib/thumb/v7e-m/nofp\libg.a(lib_a-reent.o)
tsMacFramePtTx      0x4               C:/nxp/SDKPackages/SDK_2.6.0_K32W061DK6/middleware/wireless/framework/XCVR/lib\libRadio_Test_JN518x.a(radio_test_jn518x.o)
FrameTx             0x11c             C:/nxp/SDKPackages/SDK_2.6.0_K32W061DK6/middleware/wireless/framework/XCVR/lib\libRadio_Test_JN518x.a(radio_test_jn518x.o)
__lock___env_recursive_mutex
                    0x1               c:/nxp/mcuxpressoide_11.1.0_3209/ide/plugins/com.nxp.mcuxpresso.tools.win32_11.1.0.201909161352/tools/bin/../lib/gcc/arm-none-eabi/8.3.1/../../../../arm-none-eabi/lib/thumb/v7e-m/nofp\libg.a(lib_a-lock.o)
__lock___sinit_recursive_mutex
                    0x1               c:/nxp/mcuxpressoide_11.1.0_3209/ide/plugins/com.nxp.mcuxpresso.tools.win32_11.1.0.201909161352/tools/bin/../lib/gcc/arm-none-eabi/8.3.1/../../../../arm-none-eabi/lib/thumb/v7e-m/nofp\libg.a(lib_a-lock.o)
u64jn518x_MacAddress
                    0x8               C:/nxp/SDKPackages/SDK_2.6.0_K32W061DK6/middleware/wireless/framework/XCVR/lib\libRadio_Test_JN518x.a(radio_test_jn518x.o)
u32PhyOn_sav        0x4               C:/nxp/SDKPackages/SDK_2.6.0_K32W061DK6/middleware/wireless/framework/XCVR/lib\libRadio_Test_JN518x.a(radio.o)
u32XOSlaveSav       0x4               C:/nxp/SDKPackages/SDK_2.6.0_K32W061DK6/middleware/wireless/framework/XCVR/lib\libRadio_Test_JN518x.a(radio.o)
__lock___malloc_recursive_mutex
                    0x1               c:/nxp/mcuxpressoide_11.1.0_3209/ide/plugins/com.nxp.mcuxpresso.tools.win32_11.1.0.201909161352/tools/bin/../lib/gcc/arm-none-eabi/8.3.1/../../../../arm-none-eabi/lib/thumb/v7e-m/nofp\libg.a(lib_a-lock.o)
sFrame              0x84              ./Common/Command.o
FrameRx             0x11c             C:/nxp/SDKPackages/SDK_2.6.0_K32W061DK6/middleware/wireless/framework/XCVR/lib\libRadio_Test_JN518x.a(radio_test_jn518x.o)
b_event_in_process_patch_on
                    0x1               C:/nxp/SDKPackages/SDK_2.6.0_K32W061DK6/middleware/wireless/framework/XCVR/lib\libRadio_Test_JN518x.a(radio.o)
u32TempReg          0x4               C:/nxp/SDKPackages/SDK_2.6.0_K32W061DK6/middleware/wireless/framework/XCVR/lib\libRadio_Test_JN518x.a(radio.o)
__lock___at_quick_exit_mutex
                    0x1               c:/nxp/mcuxpressoide_11.1.0_3209/ide/plugins/com.nxp.mcuxpresso.tools.win32_11.1.0.201909161352/tools/bin/../lib/gcc/arm-none-eabi/8.3.1/../../../../arm-none-eabi/lib/thumb/v7e-m/nofp\libg.a(lib_a-lock.o)
__lock___dd_hash_mutex
                    0x1               c:/nxp/mcuxpressoide_11.1.0_3209/ide/plugins/com.nxp.mcuxpresso.tools.win32_11.1.0.201909161352/tools/bin/../lib/gcc/arm-none-eabi/8.3.1/../../../../arm-none-eabi/lib/thumb/v7e-m/nofp\libg.a(lib_a-lock.o)
__lock___tz_mutex   0x1               c:/nxp/mcuxpressoide_11.1.0_3209/ide/plugins/com.nxp.mcuxpresso.tools.win32_11.1.0.201909161352/tools/bin/../lib/gcc/arm-none-eabi/8.3.1/../../../../arm-none-eabi/lib/thumb/v7e-m/nofp\libg.a(lib_a-lock.o)
g_serialHandle      0x4               ./utilities/fsl_debug_console.o
sTFrame             0x84              ./Common/Command.o
__lock___sfp_recursive_mutex
                    0x1               c:/nxp/mcuxpressoide_11.1.0_3209/ide/plugins/com.nxp.mcuxpresso.tools.win32_11.1.0.201909161352/tools/bin/../lib/gcc/arm-none-eabi/8.3.1/../../../../arm-none-eabi/lib/thumb/v7e-m/nofp\libg.a(lib_a-lock.o)

Discarded input sections

 .text          0x00000000        0x0 ./utilities/MicroInt_arm_sdk2.o
 .data          0x00000000        0x0 ./utilities/MicroInt_arm_sdk2.o
 .bss           0x00000000        0x0 ./utilities/MicroInt_arm_sdk2.o
 .text          0x00000000        0x0 ./utilities/Panic.o
 .data          0x00000000        0x0 ./utilities/Panic.o
 .bss           0x00000000        0x0 ./utilities/Panic.o
 .text.panic    0x00000000        0x2 ./utilities/Panic.o
 .text          0x00000000        0x0 ./utilities/fsl_assert.o
 .data          0x00000000        0x0 ./utilities/fsl_assert.o
 .bss           0x00000000        0x0 ./utilities/fsl_assert.o
 .text.__assert_func
                0x00000000       0x1c ./utilities/fsl_assert.o
 .rodata.__assert_func.str1.1
                0x00000000       0x3e ./utilities/fsl_assert.o
 .debug_info    0x00000000      0x1a8 ./utilities/fsl_assert.o
 .debug_abbrev  0x00000000       0xec ./utilities/fsl_assert.o
 .debug_loc     0x00000000       0xb9 ./utilities/fsl_assert.o
 .debug_aranges
                0x00000000       0x20 ./utilities/fsl_assert.o
 .debug_ranges  0x00000000       0x10 ./utilities/fsl_assert.o
 .debug_line    0x00000000      0x2f6 ./utilities/fsl_assert.o
 .debug_str     0x00000000      0x2c2 ./utilities/fsl_assert.o
 .comment       0x00000000       0x77 ./utilities/fsl_assert.o
 .debug_frame   0x00000000       0x28 ./utilities/fsl_assert.o
 .ARM.attributes
                0x00000000       0x2e ./utilities/fsl_assert.o
 .text          0x00000000        0x0 ./utilities/fsl_debug_console.o
 .data          0x00000000        0x0 ./utilities/fsl_debug_console.o
 .bss           0x00000000        0x0 ./utilities/fsl_debug_console.o
 .text.DbgConsole_ReadOneCharacter
                0x00000000       0x18 ./utilities/fsl_debug_console.o
 .text.DbgConsole_SendData
                0x00000000       0x34 ./utilities/fsl_debug_console.o
 .text.DbgConsole_ReadLine
                0x00000000       0x4c ./utilities/fsl_debug_console.o
 .text.DbgConsole_ReadCharacter
                0x00000000       0x20 ./utilities/fsl_debug_console.o
 .text.DbgConsole_Deinit
                0x00000000       0x38 ./utilities/fsl_debug_console.o
 .text.DbgConsole_Flush
                0x00000000        0x4 ./utilities/fsl_debug_console.o
 .text.DbgConsole_Putchar
                0x00000000       0x12 ./utilities/fsl_debug_console.o
 .text.DbgConsole_Scanf
                0x00000000       0x34 ./utilities/fsl_debug_console.o
 .text.DbgConsole_Getchar
                0x00000000       0x1a ./utilities/fsl_debug_console.o
 .text.__sys_write
                0x00000000       0x1e ./utilities/fsl_debug_console.o
 .text.__sys_readc
                0x00000000       0x14 ./utilities/fsl_debug_console.o
 .bss.s_debugConsoleReadWaitSemaphore
                0x00000000        0x1 ./utilities/fsl_debug_console.o
 .rodata.DbgConsole_ReadCharacter.str1.1
                0x00000000       0x6d ./utilities/fsl_debug_console.o
 .rodata.DbgConsole_ReadLine.str1.1
                0x00000000       0x76 ./utilities/fsl_debug_console.o
 .rodata.DbgConsole_SendData.str1.1
                0x00000000       0xe9 ./utilities/fsl_debug_console.o
 .text          0x00000000        0x0 ./utilities/serial_manager.o
 .data          0x00000000        0x0 ./utilities/serial_manager.o
 .bss           0x00000000        0x0 ./utilities/serial_manager.o
 .text.SerialManager_Deinit
                0x00000000       0x3c ./utilities/serial_manager.o
 .text.SerialManager_CloseWriteHandle
                0x00000000       0x3c ./utilities/serial_manager.o
 .text.SerialManager_CloseReadHandle
                0x00000000       0x3c ./utilities/serial_manager.o
 .text.SerialManager_ReadBlocking
                0x00000000       0x44 ./utilities/serial_manager.o
 .text.SerialManager_EnterLowpower
                0x00000000       0x14 ./utilities/serial_manager.o
 .text.SerialManager_ExitLowpower
                0x00000000       0x14 ./utilities/serial_manager.o
 .rodata.SerialManager_CloseReadHandle.str1.1
                0x00000000       0xfc ./utilities/serial_manager.o
 .rodata.SerialManager_CloseWriteHandle.str1.1
                0x00000000       0xc7 ./utilities/serial_manager.o
 .rodata.SerialManager_Deinit.str1.1
                0x00000000       0x66 ./utilities/serial_manager.o
 .rodata.SerialManager_EnterLowpower.str1.1
                0x00000000       0x67 ./utilities/serial_manager.o
 .rodata.SerialManager_ExitLowpower.str1.1
                0x00000000       0x67 ./utilities/serial_manager.o
 .rodata.SerialManager_ReadBlocking.str1.1
                0x00000000      0x184 ./utilities/serial_manager.o
 .text          0x00000000        0x0 ./utilities/serial_port_uart.o
 .data          0x00000000        0x0 ./utilities/serial_port_uart.o
 .bss           0x00000000        0x0 ./utilities/serial_port_uart.o
 .text.Serial_UartDeinit
                0x00000000       0x18 ./utilities/serial_port_uart.o
 .text.Serial_UartRead
                0x00000000       0x2c ./utilities/serial_port_uart.o
 .rodata.Serial_UartDeinit.str1.1
                0x00000000       0x68 ./utilities/serial_port_uart.o
 .rodata.Serial_UartRead.str1.1
                0x00000000      0x12c ./utilities/serial_port_uart.o
 .text          0x00000000        0x0 ./utilities/usart_adapter.o
 .data          0x00000000        0x0 ./utilities/usart_adapter.o
 .bss           0x00000000        0x0 ./utilities/usart_adapter.o
 .text.HAL_UartDeinit
                0x00000000       0x24 ./utilities/usart_adapter.o
 .text.HAL_UartReceiveBlocking
                0x00000000       0x40 ./utilities/usart_adapter.o
 .rodata.HAL_UartDeinit.str1.1
                0x00000000       0x55 ./utilities/usart_adapter.o
 .rodata.HAL_UartReceiveBlocking.str1.1
                0x00000000       0xfd ./utilities/usart_adapter.o
 .text          0x00000000        0x0 ./startup/startup_K32W061.o
 .data          0x00000000        0x0 ./startup/startup_K32W061.o
 .bss           0x00000000        0x0 ./startup/startup_K32W061.o
 .text.DMA0_IRQHandler
                0x00000000        0x8 ./startup/startup_K32W061.o
 .text.USART0_IRQHandler
                0x00000000        0x8 ./startup/startup_K32W061.o
 .text.USART1_IRQHandler
                0x00000000        0x8 ./startup/startup_K32W061.o
 .text.I2C0_IRQHandler
                0x00000000        0x8 ./startup/startup_K32W061.o
 .text.I2C1_IRQHandler
                0x00000000        0x8 ./startup/startup_K32W061.o
 .text          0x00000000        0x0 ./startup/system_K32W061.o
 .data          0x00000000        0x0 ./startup/system_K32W061.o
 .bss           0x00000000        0x0 ./startup/system_K32W061.o
 .text          0x00000000        0x0 ./source/tis_trp_dut.o
 .data          0x00000000        0x0 ./source/tis_trp_dut.o
 .bss           0x00000000        0x0 ./source/tis_trp_dut.o
 .bss.bHighPower
                0x00000000        0x1 ./source/tis_trp_dut.o
 .text          0x00000000        0x0 ./drivers/fsl_clock.o
 .data          0x00000000        0x0 ./drivers/fsl_clock.o
 .bss           0x00000000        0x0 ./drivers/fsl_clock.o
 .text.CLOCK_GetClkDiv
                0x00000000        0xc ./drivers/fsl_clock.o
 .text.CLOCK_GetXtal32MFreq
                0x00000000        0x8 ./drivers/fsl_clock.o
 .text.CLOCK_GetFro1MFreq
                0x00000000        0x8 ./drivers/fsl_clock.o
 .text.CLOCK_SetFRGClock
                0x00000000       0x44 ./drivers/fsl_clock.o
 .text.CLOCK_GetSpifiClkFreq
                0x00000000       0x30 ./drivers/fsl_clock.o
 .text.CLOCK_GetAdcClock
                0x00000000       0x3c ./drivers/fsl_clock.o
 .text.CLOCK_DisableClock
                0x00000000       0xa0 ./drivers/fsl_clock.o
 .text.CLOCK_IsClockEnable
                0x00000000       0x1e ./drivers/fsl_clock.o
 .text.CLOCK_DisableAPBBridge
                0x00000000        0xe ./drivers/fsl_clock.o
 .text.CLOCK_Xtal32k_Trim
                0x00000000       0xc4 ./drivers/fsl_clock.o
 .rodata.g_Ext_Clk_Freq
                0x00000000        0x4 ./drivers/fsl_clock.o
 .text          0x00000000        0x0 ./drivers/fsl_common.o
 .data          0x00000000        0x0 ./drivers/fsl_common.o
 .bss           0x00000000        0x0 ./drivers/fsl_common.o
 .text.EnableDeepSleepIRQ
                0x00000000       0x38 ./drivers/fsl_common.o
 .text.DisableDeepSleepIRQ
                0x00000000       0x44 ./drivers/fsl_common.o
 .text.SDK_Malloc
                0x00000000       0x2e ./drivers/fsl_common.o
 .text.SDK_Free
                0x00000000       0x18 ./drivers/fsl_common.o
 .text.SDK_DelayAtLeastUs
                0x00000000       0x44 ./drivers/fsl_common.o
 .rodata.SDK_DelayAtLeastUs.str1.1
                0x00000000       0xc9 ./drivers/fsl_common.o
 .debug_info    0x00000000     0x11e6 ./drivers/fsl_common.o
 .debug_abbrev  0x00000000      0x346 ./drivers/fsl_common.o
 .debug_loc     0x00000000      0x38b ./drivers/fsl_common.o
 .debug_aranges
                0x00000000       0x40 ./drivers/fsl_common.o
 .debug_ranges  0x00000000       0xa0 ./drivers/fsl_common.o
 .debug_line    0x00000000      0x438 ./drivers/fsl_common.o
 .debug_str     0x00000000      0xeb6 ./drivers/fsl_common.o
 .comment       0x00000000       0x77 ./drivers/fsl_common.o
 .debug_frame   0x00000000       0x88 ./drivers/fsl_common.o
 .ARM.attributes
                0x00000000       0x2e ./drivers/fsl_common.o
 .text          0x00000000        0x0 ./drivers/fsl_ctimer.o
 .data          0x00000000        0x0 ./drivers/fsl_ctimer.o
 .bss           0x00000000        0x0 ./drivers/fsl_ctimer.o
 .text.CTIMER_Deinit
                0x00000000       0x50 ./drivers/fsl_ctimer.o
 .text.CTIMER_SetupPwm
                0x00000000       0x9c ./drivers/fsl_ctimer.o
 .text.CTIMER_SetupPwmPeriod
                0x00000000       0x70 ./drivers/fsl_ctimer.o
 .text.CTIMER_UpdatePwmDutycycle
                0x00000000       0x1c ./drivers/fsl_ctimer.o
 .rodata.CTIMER_SetupPwm.str1.1
                0x00000000       0x62 ./drivers/fsl_ctimer.o
 .text          0x00000000        0x0 ./drivers/fsl_flexcomm.o
 .data          0x00000000        0x0 ./drivers/fsl_flexcomm.o
 .bss           0x00000000        0x0 ./drivers/fsl_flexcomm.o
 .text.FLEXCOMM_SetIRQHandler
                0x00000000       0x24 ./drivers/fsl_flexcomm.o
 .rodata.kFlexcommIrqs
                0x00000000        0x7 ./drivers/fsl_flexcomm.o
 .text          0x00000000        0x0 ./drivers/fsl_gpio.o
 .data          0x00000000        0x0 ./drivers/fsl_gpio.o
 .bss           0x00000000        0x0 ./drivers/fsl_gpio.o
 .text.GPIO_PortInit
                0x00000000       0x20 ./drivers/fsl_gpio.o
 .text.GPIO_PinInit
                0x00000000       0x2e ./drivers/fsl_gpio.o
 .rodata.GPIO_PortInit.str1.1
                0x00000000       0x73 ./drivers/fsl_gpio.o
 .debug_info    0x00000000      0x7c2 ./drivers/fsl_gpio.o
 .debug_abbrev  0x00000000      0x204 ./drivers/fsl_gpio.o
 .debug_loc     0x00000000      0x13a ./drivers/fsl_gpio.o
 .debug_aranges
                0x00000000       0x28 ./drivers/fsl_gpio.o
 .debug_ranges  0x00000000       0x18 ./drivers/fsl_gpio.o
 .debug_line    0x00000000      0x2ce ./drivers/fsl_gpio.o
 .debug_str     0x00000000      0xa95 ./drivers/fsl_gpio.o
 .comment       0x00000000       0x77 ./drivers/fsl_gpio.o
 .debug_frame   0x00000000       0x44 ./drivers/fsl_gpio.o
 .ARM.attributes
                0x00000000       0x2e ./drivers/fsl_gpio.o
 .text          0x00000000        0x0 ./drivers/fsl_inputmux.o
 .data          0x00000000        0x0 ./drivers/fsl_inputmux.o
 .bss           0x00000000        0x0 ./drivers/fsl_inputmux.o
 .text.INPUTMUX_Init
                0x00000000        0x6 ./drivers/fsl_inputmux.o
 .text.INPUTMUX_AttachSignal
                0x00000000        0xe ./drivers/fsl_inputmux.o
 .text.INPUTMUX_Deinit
                0x00000000        0x6 ./drivers/fsl_inputmux.o
 .debug_info    0x00000000      0x727 ./drivers/fsl_inputmux.o
 .debug_abbrev  0x00000000      0x17f ./drivers/fsl_inputmux.o
 .debug_loc     0x00000000       0xcf ./drivers/fsl_inputmux.o
 .debug_aranges
                0x00000000       0x30 ./drivers/fsl_inputmux.o
 .debug_ranges  0x00000000       0x20 ./drivers/fsl_inputmux.o
 .debug_line    0x00000000      0x29f ./drivers/fsl_inputmux.o
 .debug_str     0x00000000      0xf8f ./drivers/fsl_inputmux.o
 .comment       0x00000000       0x77 ./drivers/fsl_inputmux.o
 .debug_frame   0x00000000       0x40 ./drivers/fsl_inputmux.o
 .ARM.attributes
                0x00000000       0x2e ./drivers/fsl_inputmux.o
 .text          0x00000000        0x0 ./drivers/fsl_power.o
 .data          0x00000000        0x0 ./drivers/fsl_power.o
 .bss           0x00000000        0x0 ./drivers/fsl_power.o
 .text.POWER_FlexcomClocksDisable
                0x00000000       0x3e ./drivers/fsl_power.o
 .text.POWER_GetLibVersion
                0x00000000        0x8 ./drivers/fsl_power.o
 .text.POWER_GetResetCause
                0x00000000       0x4c ./drivers/fsl_power.o
 .text.POWER_ClearResetCause
                0x00000000        0xc ./drivers/fsl_power.o
 .text.POWER_DisplayActiveVoltage
                0x00000000       0xbc ./drivers/fsl_power.o
 .text.POWER_ApplyLdoActiveVoltage
                0x00000000       0x14 ./drivers/fsl_power.o
 .text.POWER_BodVbatGetDefaultConfig
                0x00000000        0xc ./drivers/fsl_power.o
 .text.POWER_BodVbatConfig
                0x00000000       0x88 ./drivers/fsl_power.o
 .text.POWER_EnterDeepSleepMode
                0x00000000       0x2c ./drivers/fsl_power.o
 .text.POWER_EnterPowerDownMode
                0x00000000      0x360 ./drivers/fsl_power.o
 .text.POWER_EnterDeepDownMode
                0x00000000       0xdc ./drivers/fsl_power.o
 .text.POWER_EnterPowerMode
                0x00000000       0x16 ./drivers/fsl_power.o
 .rodata.POWER_DisplayActiveVoltage.str1.1
                0x00000000       0xb3 ./drivers/fsl_power.o
 .rodata.lowpower_ldovoltage_min
                0x00000000        0x9 ./drivers/fsl_power.o
 .text          0x00000000        0x0 ./drivers/fsl_reset.o
 .data          0x00000000        0x0 ./drivers/fsl_reset.o
 .bss           0x00000000        0x0 ./drivers/fsl_reset.o
 .text          0x00000000        0x0 ./drivers/fsl_str.o
 .data          0x00000000        0x0 ./drivers/fsl_str.o
 .bss           0x00000000        0x0 ./drivers/fsl_str.o
 .text.ScanIgnoreWhiteSpace
                0x00000000       0x20 ./drivers/fsl_str.o
 .text.StrFormatScanf
                0x00000000      0x24e ./drivers/fsl_str.o
 .text          0x00000000        0x0 ./drivers/fsl_usart.o
 .data          0x00000000        0x0 ./drivers/fsl_usart.o
 .bss           0x00000000        0x0 ./drivers/fsl_usart.o
 .text.USART_GetInstance
                0x00000000       0x28 ./drivers/fsl_usart.o
 .text.USART_TransferGetRxRingBufferLength
                0x00000000       0x2c ./drivers/fsl_usart.o
 .text.USART_TransferIsRxRingBufferFull
                0x00000000       0x20 ./drivers/fsl_usart.o
 .text.USART_TransferHandleIRQ
                0x00000000      0x1f4 ./drivers/fsl_usart.o
 .text.USART_TransferStartRingBuffer
                0x00000000       0x3c ./drivers/fsl_usart.o
 .text.USART_TransferStopRingBuffer
                0x00000000       0x34 ./drivers/fsl_usart.o
 .text.USART_Deinit
                0x00000000       0x30 ./drivers/fsl_usart.o
 .text.USART_TransferCreateHandle
                0x00000000       0x88 ./drivers/fsl_usart.o
 .text.USART_TransferSendNonBlocking
                0x00000000       0x4c ./drivers/fsl_usart.o
 .text.USART_TransferAbortSend
                0x00000000       0x2c ./drivers/fsl_usart.o
 .text.USART_TransferGetSendCount
                0x00000000       0x30 ./drivers/fsl_usart.o
 .text.USART_TransferReceiveNonBlocking
                0x00000000       0xe4 ./drivers/fsl_usart.o
 .text.USART_TransferAbortReceive
                0x00000000       0x30 ./drivers/fsl_usart.o
 .text.USART_TransferGetReceiveCount
                0x00000000       0x30 ./drivers/fsl_usart.o
 .rodata.USART_Deinit.str1.1
                0x00000000       0x5f ./drivers/fsl_usart.o
 .rodata.USART_GetInstance.str1.1
                0x00000000       0x57 ./drivers/fsl_usart.o
 .rodata.USART_TransferAbortReceive.str1.1
                0x00000000       0x61 ./drivers/fsl_usart.o
 .rodata.USART_TransferAbortSend.str1.1
                0x00000000       0x61 ./drivers/fsl_usart.o
 .rodata.USART_TransferCreateHandle.str1.1
                0x00000000       0x78 ./drivers/fsl_usart.o
 .rodata.USART_TransferGetReceiveCount.str1.1
                0x00000000       0xc1 ./drivers/fsl_usart.o
 .rodata.USART_TransferGetRxRingBufferLength.str1.1
                0x00000000       0x60 ./drivers/fsl_usart.o
 .rodata.USART_TransferGetSendCount.str1.1
                0x00000000       0xc1 ./drivers/fsl_usart.o
 .rodata.USART_TransferHandleIRQ.str1.1
                0x00000000       0x75 ./drivers/fsl_usart.o
 .rodata.USART_TransferIsRxRingBufferFull.str1.1
                0x00000000       0x60 ./drivers/fsl_usart.o
 .rodata.USART_TransferReceiveNonBlocking.str1.1
                0x00000000      0x10d ./drivers/fsl_usart.o
 .rodata.USART_TransferSendNonBlocking.str1.1
                0x00000000      0x10d ./drivers/fsl_usart.o
 .rodata.USART_TransferStartRingBuffer.str1.1
                0x00000000      0x125 ./drivers/fsl_usart.o
 .rodata.USART_TransferStopRingBuffer.str1.1
                0x00000000       0xc0 ./drivers/fsl_usart.o
 .rodata.s_usartIRQ
                0x00000000        0x2 ./drivers/fsl_usart.o
 .text          0x00000000        0x0 ./drivers/fsl_wtimer.o
 .data          0x00000000        0x0 ./drivers/fsl_wtimer.o
 .bss           0x00000000        0x0 ./drivers/fsl_wtimer.o
 .text.WTIMER_Init
                0x00000000       0x18 ./drivers/fsl_wtimer.o
 .text.WTIMER_DeInit
                0x00000000       0x18 ./drivers/fsl_wtimer.o
 .text.WTIMER_GetStatusFlags
                0x00000000       0x2c ./drivers/fsl_wtimer.o
 .text.WTIMER_EnableInterrupts
                0x00000000       0x40 ./drivers/fsl_wtimer.o
 .text.WTIMER_StartTimer
                0x00000000       0x78 ./drivers/fsl_wtimer.o
 .text.WTIMER_ReadTimerSafe
                0x00000000       0x28 ./drivers/fsl_wtimer.o
 .text.WTIMER_ReadTimer
                0x00000000       0x1c ./drivers/fsl_wtimer.o
 .text.WTIMER_ClearStatusFlags
                0x00000000       0x3c ./drivers/fsl_wtimer.o
 .text.WTIMER_StopTimer
                0x00000000       0x38 ./drivers/fsl_wtimer.o
 .rodata.timer_param
                0x00000000       0x50 ./drivers/fsl_wtimer.o
 .debug_info    0x00000000     0x1517 ./drivers/fsl_wtimer.o
 .debug_abbrev  0x00000000      0x2db ./drivers/fsl_wtimer.o
 .debug_loc     0x00000000      0x397 ./drivers/fsl_wtimer.o
 .debug_aranges
                0x00000000       0x60 ./drivers/fsl_wtimer.o
 .debug_ranges  0x00000000       0x68 ./drivers/fsl_wtimer.o
 .debug_line    0x00000000      0x4f9 ./drivers/fsl_wtimer.o
 .debug_str     0x00000000     0x1852 ./drivers/fsl_wtimer.o
 .comment       0x00000000       0x77 ./drivers/fsl_wtimer.o
 .debug_frame   0x00000000       0xd4 ./drivers/fsl_wtimer.o
 .ARM.attributes
                0x00000000       0x2e ./drivers/fsl_wtimer.o
 .text          0x00000000        0x0 ./board/board.o
 .data          0x00000000        0x0 ./board/board.o
 .bss           0x00000000        0x0 ./board/board.o
 .text.BOARD_DbgDiagEnable
                0x00000000        0x2 ./board/board.o
 .text.BOARD_DbgLpIoSet
                0x00000000        0x2 ./board/board.o
 .data.CLOCK_ai32MXtalIecLoadPfVsTemp_x1000
                0x00000000       0x8c ./board/board.o
 .text          0x00000000        0x0 ./board/clock_config.o
 .data          0x00000000        0x0 ./board/clock_config.o
 .bss           0x00000000        0x0 ./board/clock_config.o
 .text.BOARD_BootClockRUN
                0x00000000       0xe8 ./board/clock_config.o
 .text.BOARD_InitBootClocks
                0x00000000        0x4 ./board/clock_config.o
 .debug_info    0x00000000      0x775 ./board/clock_config.o
 .debug_abbrev  0x00000000      0x135 ./board/clock_config.o
 .debug_aranges
                0x00000000       0x28 ./board/clock_config.o
 .debug_ranges  0x00000000       0x18 ./board/clock_config.o
 .debug_line    0x00000000      0x2b6 ./board/clock_config.o
 .debug_str     0x00000000      0xbf8 ./board/clock_config.o
 .comment       0x00000000       0x77 ./board/clock_config.o
 .debug_frame   0x00000000       0x38 ./board/clock_config.o
 .ARM.attributes
                0x00000000       0x2e ./board/clock_config.o
 .text          0x00000000        0x0 ./board/hardware_init.o
 .data          0x00000000        0x0 ./board/hardware_init.o
 .bss           0x00000000        0x0 ./board/hardware_init.o
 .text          0x00000000        0x0 ./board/pin_mux.o
 .data          0x00000000        0x0 ./board/pin_mux.o
 .bss           0x00000000        0x0 ./board/pin_mux.o
 .text          0x00000000        0x0 ./Common/CRC.o
 .data          0x00000000        0x0 ./Common/CRC.o
 .bss           0x00000000        0x0 ./Common/CRC.o
 .text.straight_16
                0x00000000        0x2 ./Common/CRC.o
 .text.straight_8
                0x00000000        0x2 ./Common/CRC.o
 .text.crc16ccitt
                0x00000000       0x24 ./Common/CRC.o
 .text.crc16ccitt_xmodem
                0x00000000       0x24 ./Common/CRC.o
 .text.crc16ccitt_1d0f
                0x00000000       0x24 ./Common/CRC.o
 .text.crc16ibm
                0x00000000       0x24 ./Common/CRC.o
 .text          0x00000000        0x0 ./Common/Command.o
 .data          0x00000000        0x0 ./Common/Command.o
 .bss           0x00000000        0x0 ./Common/Command.o
 .text.vCommand_SendChannel
                0x00000000       0x16 ./Common/Command.o
 .text          0x00000000        0x0 C:/nxp/SDKPackages/SDK_2.6.0_K32W061DK6/middleware/wireless/ieee-802.15.4/lib\libMiniMac.a(MMAC.o)
 .data          0x00000000        0x0 C:/nxp/SDKPackages/SDK_2.6.0_K32W061DK6/middleware/wireless/ieee-802.15.4/lib\libMiniMac.a(MMAC.o)
 .bss           0x00000000        0x0 C:/nxp/SDKPackages/SDK_2.6.0_K32W061DK6/middleware/wireless/ieee-802.15.4/lib\libMiniMac.a(MMAC.o)
 .text.vMMAC_EnableInterrupts
                0x00000000       0x28 C:/nxp/SDKPackages/SDK_2.6.0_K32W061DK6/middleware/wireless/ieee-802.15.4/lib\libMiniMac.a(MMAC.o)
 .text.vMMAC_RegisterPhyIntHandler
                0x00000000        0xc C:/nxp/SDKPackages/SDK_2.6.0_K32W061DK6/middleware/wireless/ieee-802.15.4/lib\libMiniMac.a(MMAC.o)
 .text.u32MMAC_GetTime
                0x00000000        0xc C:/nxp/SDKPackages/SDK_2.6.0_K32W061DK6/middleware/wireless/ieee-802.15.4/lib\libMiniMac.a(MMAC.o)
 .text.vMMAC_SetCutOffTimer
                0x00000000       0x24 C:/nxp/SDKPackages/SDK_2.6.0_K32W061DK6/middleware/wireless/ieee-802.15.4/lib\libMiniMac.a(MMAC.o)
 .text.vMMAC_SynchroniseBackoffClock
                0x00000000       0x18 C:/nxp/SDKPackages/SDK_2.6.0_K32W061DK6/middleware/wireless/ieee-802.15.4/lib\libMiniMac.a(MMAC.o)
 .text.u8MMAC_EnergyDetect
                0x00000000       0x1c C:/nxp/SDKPackages/SDK_2.6.0_K32W061DK6/middleware/wireless/ieee-802.15.4/lib\libMiniMac.a(MMAC.o)
 .text.vMMAC_SetRxAddress
                0x00000000       0x1c C:/nxp/SDKPackages/SDK_2.6.0_K32W061DK6/middleware/wireless/ieee-802.15.4/lib\libMiniMac.a(MMAC.o)
 .text.vMMAC_SetRxPanId
                0x00000000        0xc C:/nxp/SDKPackages/SDK_2.6.0_K32W061DK6/middleware/wireless/ieee-802.15.4/lib\libMiniMac.a(MMAC.o)
 .text.vMMAC_SetRxShortAddr
                0x00000000        0xc C:/nxp/SDKPackages/SDK_2.6.0_K32W061DK6/middleware/wireless/ieee-802.15.4/lib\libMiniMac.a(MMAC.o)
 .text.vMMAC_SetRxExtendedAddr
                0x00000000       0x14 C:/nxp/SDKPackages/SDK_2.6.0_K32W061DK6/middleware/wireless/ieee-802.15.4/lib\libMiniMac.a(MMAC.o)
 .text.vMMAC_SetRxStartTime
                0x00000000        0xc C:/nxp/SDKPackages/SDK_2.6.0_K32W061DK6/middleware/wireless/ieee-802.15.4/lib\libMiniMac.a(MMAC.o)
 .text.vMMAC_PromiscuousMode
                0x00000000       0x1c C:/nxp/SDKPackages/SDK_2.6.0_K32W061DK6/middleware/wireless/ieee-802.15.4/lib\libMiniMac.a(MMAC.o)
 .text.bMMAC_RxDetected
                0x00000000       0x10 C:/nxp/SDKPackages/SDK_2.6.0_K32W061DK6/middleware/wireless/ieee-802.15.4/lib\libMiniMac.a(MMAC.o)
 .text.u32MMAC_GetRxErrors
                0x00000000        0xc C:/nxp/SDKPackages/SDK_2.6.0_K32W061DK6/middleware/wireless/ieee-802.15.4/lib\libMiniMac.a(MMAC.o)
 .text.u32MMAC_GetRxTime
                0x00000000        0xc C:/nxp/SDKPackages/SDK_2.6.0_K32W061DK6/middleware/wireless/ieee-802.15.4/lib\libMiniMac.a(MMAC.o)
 .text.vMMAC_SetTxStartTime
                0x00000000        0xc C:/nxp/SDKPackages/SDK_2.6.0_K32W061DK6/middleware/wireless/ieee-802.15.4/lib\libMiniMac.a(MMAC.o)
 .text.u32MMAC_GetTxErrors
                0x00000000        0xc C:/nxp/SDKPackages/SDK_2.6.0_K32W061DK6/middleware/wireless/ieee-802.15.4/lib\libMiniMac.a(MMAC.o)
 .text.vMMAC_GetMacAddress
                0x00000000       0x30 C:/nxp/SDKPackages/SDK_2.6.0_K32W061DK6/middleware/wireless/ieee-802.15.4/lib\libMiniMac.a(MMAC.o)
 .text.u32MMAC_PollInterruptSourceUntilFired
                0x00000000       0x14 C:/nxp/SDKPackages/SDK_2.6.0_K32W061DK6/middleware/wireless/ieee-802.15.4/lib\libMiniMac.a(MMAC.o)
 .text.vMMAC_ConfigureInterruptSources
                0x00000000       0x10 C:/nxp/SDKPackages/SDK_2.6.0_K32W061DK6/middleware/wireless/ieee-802.15.4/lib\libMiniMac.a(MMAC.o)
 .text.vMMAC_StartMacTransmit
                0x00000000       0x2c C:/nxp/SDKPackages/SDK_2.6.0_K32W061DK6/middleware/wireless/ieee-802.15.4/lib\libMiniMac.a(MMAC.o)
 .text.vMMAC_StartMacReceive
                0x00000000       0x2c C:/nxp/SDKPackages/SDK_2.6.0_K32W061DK6/middleware/wireless/ieee-802.15.4/lib\libMiniMac.a(MMAC.o)
 .text.u8MMAC_ReadCcaThreshold
                0x00000000       0x24 C:/nxp/SDKPackages/SDK_2.6.0_K32W061DK6/middleware/wireless/ieee-802.15.4/lib\libMiniMac.a(MMAC.o)
 .text.vMMAC_SetComplianceLimits
                0x00000000       0x14 C:/nxp/SDKPackages/SDK_2.6.0_K32W061DK6/middleware/wireless/ieee-802.15.4/lib\libMiniMac.a(MMAC.o)
 .text.i8MMAC_GetTxPowerLevel
                0x00000000        0x4 C:/nxp/SDKPackages/SDK_2.6.0_K32W061DK6/middleware/wireless/ieee-802.15.4/lib\libMiniMac.a(MMAC.o)
 .text          0x00000000        0x0 C:/nxp/SDKPackages/SDK_2.6.0_K32W061DK6/middleware/wireless/ieee-802.15.4/lib\libMiniMac.a(MMAC_RadioInit_JN518x.o)
 .data          0x00000000        0x0 C:/nxp/SDKPackages/SDK_2.6.0_K32W061DK6/middleware/wireless/ieee-802.15.4/lib\libMiniMac.a(MMAC_RadioInit_JN518x.o)
 .bss           0x00000000        0x0 C:/nxp/SDKPackages/SDK_2.6.0_K32W061DK6/middleware/wireless/ieee-802.15.4/lib\libMiniMac.a(MMAC_RadioInit_JN518x.o)
 .group         0x00000000        0xc C:/nxp/SDKPackages/SDK_2.6.0_K32W061DK6/middleware/wireless/framework/XCVR/lib\libRadio_Test_JN518x.a(radio.o)
 .group         0x00000000        0xc C:/nxp/SDKPackages/SDK_2.6.0_K32W061DK6/middleware/wireless/framework/XCVR/lib\libRadio_Test_JN518x.a(radio.o)
 .group         0x00000000        0xc C:/nxp/SDKPackages/SDK_2.6.0_K32W061DK6/middleware/wireless/framework/XCVR/lib\libRadio_Test_JN518x.a(radio.o)
 .group         0x00000000        0xc C:/nxp/SDKPackages/SDK_2.6.0_K32W061DK6/middleware/wireless/framework/XCVR/lib\libRadio_Test_JN518x.a(radio.o)
 .group         0x00000000        0xc C:/nxp/SDKPackages/SDK_2.6.0_K32W061DK6/middleware/wireless/framework/XCVR/lib\libRadio_Test_JN518x.a(radio.o)
 .group         0x00000000        0xc C:/nxp/SDKPackages/SDK_2.6.0_K32W061DK6/middleware/wireless/framework/XCVR/lib\libRadio_Test_JN518x.a(radio.o)
 .group         0x00000000        0xc C:/nxp/SDKPackages/SDK_2.6.0_K32W061DK6/middleware/wireless/framework/XCVR/lib\libRadio_Test_JN518x.a(radio.o)
 .group         0x00000000        0xc C:/nxp/SDKPackages/SDK_2.6.0_K32W061DK6/middleware/wireless/framework/XCVR/lib\libRadio_Test_JN518x.a(radio.o)
 .group         0x00000000        0xc C:/nxp/SDKPackages/SDK_2.6.0_K32W061DK6/middleware/wireless/framework/XCVR/lib\libRadio_Test_JN518x.a(radio.o)
 .group         0x00000000        0xc C:/nxp/SDKPackages/SDK_2.6.0_K32W061DK6/middleware/wireless/framework/XCVR/lib\libRadio_Test_JN518x.a(radio.o)
 .group         0x00000000        0xc C:/nxp/SDKPackages/SDK_2.6.0_K32W061DK6/middleware/wireless/framework/XCVR/lib\libRadio_Test_JN518x.a(radio.o)
 .group         0x00000000        0xc C:/nxp/SDKPackages/SDK_2.6.0_K32W061DK6/middleware/wireless/framework/XCVR/lib\libRadio_Test_JN518x.a(radio.o)
 .group         0x00000000        0xc C:/nxp/SDKPackages/SDK_2.6.0_K32W061DK6/middleware/wireless/framework/XCVR/lib\libRadio_Test_JN518x.a(radio.o)
 .group         0x00000000        0xc C:/nxp/SDKPackages/SDK_2.6.0_K32W061DK6/middleware/wireless/framework/XCVR/lib\libRadio_Test_JN518x.a(radio.o)
 .group         0x00000000        0xc C:/nxp/SDKPackages/SDK_2.6.0_K32W061DK6/middleware/wireless/framework/XCVR/lib\libRadio_Test_JN518x.a(radio.o)
 .group         0x00000000        0xc C:/nxp/SDKPackages/SDK_2.6.0_K32W061DK6/middleware/wireless/framework/XCVR/lib\libRadio_Test_JN518x.a(radio.o)
 .group         0x00000000        0xc C:/nxp/SDKPackages/SDK_2.6.0_K32W061DK6/middleware/wireless/framework/XCVR/lib\libRadio_Test_JN518x.a(radio.o)
 .group         0x00000000        0xc C:/nxp/SDKPackages/SDK_2.6.0_K32W061DK6/middleware/wireless/framework/XCVR/lib\libRadio_Test_JN518x.a(radio.o)
 .group         0x00000000        0xc C:/nxp/SDKPackages/SDK_2.6.0_K32W061DK6/middleware/wireless/framework/XCVR/lib\libRadio_Test_JN518x.a(radio.o)
 .group         0x00000000        0xc C:/nxp/SDKPackages/SDK_2.6.0_K32W061DK6/middleware/wireless/framework/XCVR/lib\libRadio_Test_JN518x.a(radio.o)
 .group         0x00000000        0xc C:/nxp/SDKPackages/SDK_2.6.0_K32W061DK6/middleware/wireless/framework/XCVR/lib\libRadio_Test_JN518x.a(radio.o)
 .group         0x00000000        0xc C:/nxp/SDKPackages/SDK_2.6.0_K32W061DK6/middleware/wireless/framework/XCVR/lib\libRadio_Test_JN518x.a(radio.o)
 .group         0x00000000        0xc C:/nxp/SDKPackages/SDK_2.6.0_K32W061DK6/middleware/wireless/framework/XCVR/lib\libRadio_Test_JN518x.a(radio.o)
 .group         0x00000000        0xc C:/nxp/SDKPackages/SDK_2.6.0_K32W061DK6/middleware/wireless/framework/XCVR/lib\libRadio_Test_JN518x.a(radio.o)
 .group         0x00000000        0xc C:/nxp/SDKPackages/SDK_2.6.0_K32W061DK6/middleware/wireless/framework/XCVR/lib\libRadio_Test_JN518x.a(radio.o)
 .group         0x00000000        0xc C:/nxp/SDKPackages/SDK_2.6.0_K32W061DK6/middleware/wireless/framework/XCVR/lib\libRadio_Test_JN518x.a(radio.o)
 .group         0x00000000        0xc C:/nxp/SDKPackages/SDK_2.6.0_K32W061DK6/middleware/wireless/framework/XCVR/lib\libRadio_Test_JN518x.a(radio.o)
 .group         0x00000000        0xc C:/nxp/SDKPackages/SDK_2.6.0_K32W061DK6/middleware/wireless/framework/XCVR/lib\libRadio_Test_JN518x.a(radio.o)
 .group         0x00000000        0xc C:/nxp/SDKPackages/SDK_2.6.0_K32W061DK6/middleware/wireless/framework/XCVR/lib\libRadio_Test_JN518x.a(radio.o)
 .text          0x00000000        0x0 C:/nxp/SDKPackages/SDK_2.6.0_K32W061DK6/middleware/wireless/framework/XCVR/lib\libRadio_Test_JN518x.a(radio.o)
 .data          0x00000000        0x0 C:/nxp/SDKPackages/SDK_2.6.0_K32W061DK6/middleware/wireless/framework/XCVR/lib\libRadio_Test_JN518x.a(radio.o)
 .bss           0x00000000        0x0 C:/nxp/SDKPackages/SDK_2.6.0_K32W061DK6/middleware/wireless/framework/XCVR/lib\libRadio_Test_JN518x.a(radio.o)
 .text.radio_CLOCK_enableFastuDelay
                0x00000000       0x2c C:/nxp/SDKPackages/SDK_2.6.0_K32W061DK6/middleware/wireless/framework/XCVR/lib\libRadio_Test_JN518x.a(radio.o)
 .text.radio_CLOCK_disableFastuDelay
                0x00000000       0x2c C:/nxp/SDKPackages/SDK_2.6.0_K32W061DK6/middleware/wireless/framework/XCVR/lib\libRadio_Test_JN518x.a(radio.o)
 .text.radio_get_R_cal_results_from_flash
                0x00000000        0x2 C:/nxp/SDKPackages/SDK_2.6.0_K32W061DK6/middleware/wireless/framework/XCVR/lib\libRadio_Test_JN518x.a(radio.o)
 .text.u32Radio_RadioModesAvailable
                0x00000000        0x4 C:/nxp/SDKPackages/SDK_2.6.0_K32W061DK6/middleware/wireless/framework/XCVR/lib\libRadio_Test_JN518x.a(radio.o)
 .text.u32Radio_RadioGetVersion
                0x00000000        0x6 C:/nxp/SDKPackages/SDK_2.6.0_K32W061DK6/middleware/wireless/framework/XCVR/lib\libRadio_Test_JN518x.a(radio.o)
 .text.u32Radio_GetPhyState
                0x00000000       0x58 C:/nxp/SDKPackages/SDK_2.6.0_K32W061DK6/middleware/wireless/framework/XCVR/lib\libRadio_Test_JN518x.a(radio.o)
 .text.vRadio_LockupCheckAndAbortRadio
                0x00000000       0x68 C:/nxp/SDKPackages/SDK_2.6.0_K32W061DK6/middleware/wireless/framework/XCVR/lib\libRadio_Test_JN518x.a(radio.o)
 .text.vRadio_SetComplianceLimits
                0x00000000       0x14 C:/nxp/SDKPackages/SDK_2.6.0_K32W061DK6/middleware/wireless/framework/XCVR/lib\libRadio_Test_JN518x.a(radio.o)
 .text.vRadio_SetChannelStandards
                0x00000000       0x14 C:/nxp/SDKPackages/SDK_2.6.0_K32W061DK6/middleware/wireless/framework/XCVR/lib\libRadio_Test_JN518x.a(radio.o)
 .text.i16Radio_GetRSSI
                0x00000000      0x130 C:/nxp/SDKPackages/SDK_2.6.0_K32W061DK6/middleware/wireless/framework/XCVR/lib\libRadio_Test_JN518x.a(radio.o)
 .text.i16Radio_BoundRssiValue
                0x00000000       0x18 C:/nxp/SDKPackages/SDK_2.6.0_K32W061DK6/middleware/wireless/framework/XCVR/lib\libRadio_Test_JN518x.a(radio.o)
 .text.i8Radio_GetLastPacketRSSI
                0x00000000       0x1c C:/nxp/SDKPackages/SDK_2.6.0_K32W061DK6/middleware/wireless/framework/XCVR/lib\libRadio_Test_JN518x.a(radio.o)
 .text.vWritePartOfBuffer
                0x00000000       0x5a C:/nxp/SDKPackages/SDK_2.6.0_K32W061DK6/middleware/wireless/framework/XCVR/lib\libRadio_Test_JN518x.a(radio.o)
 .text.vRadio_Temp_Update
                0x00000000       0x88 C:/nxp/SDKPackages/SDK_2.6.0_K32W061DK6/middleware/wireless/framework/XCVR/lib\libRadio_Test_JN518x.a(radio.o)
 .text.vSetRecalThres
                0x00000000        0xc C:/nxp/SDKPackages/SDK_2.6.0_K32W061DK6/middleware/wireless/framework/XCVR/lib\libRadio_Test_JN518x.a(radio.o)
 .text.vGetCalTemp
                0x00000000       0x10 C:/nxp/SDKPackages/SDK_2.6.0_K32W061DK6/middleware/wireless/framework/XCVR/lib\libRadio_Test_JN518x.a(radio.o)
 .text.vRadio_SkipXTALInit
                0x00000000       0x10 C:/nxp/SDKPackages/SDK_2.6.0_K32W061DK6/middleware/wireless/framework/XCVR/lib\libRadio_Test_JN518x.a(radio.o)
 .text.vRadio_EnableXTALInit
                0x00000000       0x10 C:/nxp/SDKPackages/SDK_2.6.0_K32W061DK6/middleware/wireless/framework/XCVR/lib\libRadio_Test_JN518x.a(radio.o)
 .text.vRadio_BLE_ResetOn
                0x00000000        0xe C:/nxp/SDKPackages/SDK_2.6.0_K32W061DK6/middleware/wireless/framework/XCVR/lib\libRadio_Test_JN518x.a(radio.o)
 .text.vRadio_BLE_ResetOff
                0x00000000        0xe C:/nxp/SDKPackages/SDK_2.6.0_K32W061DK6/middleware/wireless/framework/XCVR/lib\libRadio_Test_JN518x.a(radio.o)
 .text.vRadio_Enable_AgcReadyPatch
                0x00000000       0x54 C:/nxp/SDKPackages/SDK_2.6.0_K32W061DK6/middleware/wireless/framework/XCVR/lib\libRadio_Test_JN518x.a(radio.o)
 .text.vRadio_Disable_AgcReadyPatch
                0x00000000       0x54 C:/nxp/SDKPackages/SDK_2.6.0_K32W061DK6/middleware/wireless/framework/XCVR/lib\libRadio_Test_JN518x.a(radio.o)
 .text.vRadio_MultiRX_AgcReadyPatch
                0x00000000       0x1c C:/nxp/SDKPackages/SDK_2.6.0_K32W061DK6/middleware/wireless/framework/XCVR/lib\libRadio_Test_JN518x.a(radio.o)
 .text.vRadio_SingleRX_AgcReadyPatch
                0x00000000       0x1c C:/nxp/SDKPackages/SDK_2.6.0_K32W061DK6/middleware/wireless/framework/XCVR/lib\libRadio_Test_JN518x.a(radio.o)
 .text.vRadio_DisableZBRadio
                0x00000000       0x18 C:/nxp/SDKPackages/SDK_2.6.0_K32W061DK6/middleware/wireless/framework/XCVR/lib\libRadio_Test_JN518x.a(radio.o)
 .text.vRadio_DisableBLERadio
                0x00000000       0x18 C:/nxp/SDKPackages/SDK_2.6.0_K32W061DK6/middleware/wireless/framework/XCVR/lib\libRadio_Test_JN518x.a(radio.o)
 .text.vRadio_EnableBLEFastTX
                0x00000000      0x1a0 C:/nxp/SDKPackages/SDK_2.6.0_K32W061DK6/middleware/wireless/framework/XCVR/lib\libRadio_Test_JN518x.a(radio.o)
 .text.vRadio_DisableBLEFastTX
                0x00000000      0x174 C:/nxp/SDKPackages/SDK_2.6.0_K32W061DK6/middleware/wireless/framework/XCVR/lib\libRadio_Test_JN518x.a(radio.o)
 .text.vRadio_ZBtoBLE
                0x00000000       0x54 C:/nxp/SDKPackages/SDK_2.6.0_K32W061DK6/middleware/wireless/framework/XCVR/lib\libRadio_Test_JN518x.a(radio.o)
 .text.vRadio_BLEtoZB
                0x00000000       0x6c C:/nxp/SDKPackages/SDK_2.6.0_K32W061DK6/middleware/wireless/framework/XCVR/lib\libRadio_Test_JN518x.a(radio.o)
 .text.vRadio_AntennaDiversityTxRxEnable
                0x00000000      0x118 C:/nxp/SDKPackages/SDK_2.6.0_K32W061DK6/middleware/wireless/framework/XCVR/lib\libRadio_Test_JN518x.a(radio.o)
 .text.vRadio_AntennaDiversityConfigure
                0x00000000       0x18 C:/nxp/SDKPackages/SDK_2.6.0_K32W061DK6/middleware/wireless/framework/XCVR/lib\libRadio_Test_JN518x.a(radio.o)
 .text.vRadio_AntennaDiversitySwitch
                0x00000000       0x10 C:/nxp/SDKPackages/SDK_2.6.0_K32W061DK6/middleware/wireless/framework/XCVR/lib\libRadio_Test_JN518x.a(radio.o)
 .text.u8Radio_AntennaDiversityStatus
                0x00000000       0x10 C:/nxp/SDKPackages/SDK_2.6.0_K32W061DK6/middleware/wireless/framework/XCVR/lib\libRadio_Test_JN518x.a(radio.o)
 .text.i16Radio_GetNbRSSISync
                0x00000000       0x10 C:/nxp/SDKPackages/SDK_2.6.0_K32W061DK6/middleware/wireless/framework/XCVR/lib\libRadio_Test_JN518x.a(radio.o)
 .text.i16Radio_GetNbRSSISyncCor
                0x00000000       0x6c C:/nxp/SDKPackages/SDK_2.6.0_K32W061DK6/middleware/wireless/framework/XCVR/lib\libRadio_Test_JN518x.a(radio.o)
 .text.vRadio_ActivateXtal32MRadioBiasing
                0x00000000      0x190 C:/nxp/SDKPackages/SDK_2.6.0_K32W061DK6/middleware/wireless/framework/XCVR/lib\libRadio_Test_JN518x.a(radio.o)
 .text.vResetFlashCalData
                0x00000000       0x20 C:/nxp/SDKPackages/SDK_2.6.0_K32W061DK6/middleware/wireless/framework/XCVR/lib\libRadio_Test_JN518x.a(radio.o)
 .text.vRadio_Recal
                0x00000000       0xec C:/nxp/SDKPackages/SDK_2.6.0_K32W061DK6/middleware/wireless/framework/XCVR/lib\libRadio_Test_JN518x.a(radio.o)
 .text.u32Radio_Get_Next_Recal_Duration
                0x00000000       0x84 C:/nxp/SDKPackages/SDK_2.6.0_K32W061DK6/middleware/wireless/framework/XCVR/lib\libRadio_Test_JN518x.a(radio.o)
 .text.u16PopBits
                0x00000000       0x50 C:/nxp/SDKPackages/SDK_2.6.0_K32W061DK6/middleware/wireless/framework/XCVR/lib\libRadio_Test_JN518x.a(radio.o)
 .text.vPushBits
                0x00000000       0x4c C:/nxp/SDKPackages/SDK_2.6.0_K32W061DK6/middleware/wireless/framework/XCVR/lib\libRadio_Test_JN518x.a(radio.o)
 .text.vRadio_Save_ApplicationData_Retention
                0x00000000      0x1e0 C:/nxp/SDKPackages/SDK_2.6.0_K32W061DK6/middleware/wireless/framework/XCVR/lib\libRadio_Test_JN518x.a(radio.o)
 .text.vRadio_Restore_Retention_ApplicationData
                0x00000000      0x26c C:/nxp/SDKPackages/SDK_2.6.0_K32W061DK6/middleware/wireless/framework/XCVR/lib\libRadio_Test_JN518x.a(radio.o)
 .text.vRadio_ConfigCalFlashUsage
                0x00000000       0x1c C:/nxp/SDKPackages/SDK_2.6.0_K32W061DK6/middleware/wireless/framework/XCVR/lib\libRadio_Test_JN518x.a(radio.o)
 .text.vRadio_Reset_RadioConfig
                0x00000000       0x3c C:/nxp/SDKPackages/SDK_2.6.0_K32W061DK6/middleware/wireless/framework/XCVR/lib\libRadio_Test_JN518x.a(radio.o)
 .bss.u8PopBitIndex.22261
                0x00000000        0x1 C:/nxp/SDKPackages/SDK_2.6.0_K32W061DK6/middleware/wireless/framework/XCVR/lib\libRadio_Test_JN518x.a(radio.o)
 .bss.u8PopByteIndex.22260
                0x00000000        0x1 C:/nxp/SDKPackages/SDK_2.6.0_K32W061DK6/middleware/wireless/framework/XCVR/lib\libRadio_Test_JN518x.a(radio.o)
 .bss.u8PushBitIndex.22271
                0x00000000        0x1 C:/nxp/SDKPackages/SDK_2.6.0_K32W061DK6/middleware/wireless/framework/XCVR/lib\libRadio_Test_JN518x.a(radio.o)
 .bss.u8PushByteIndex.22270
                0x00000000        0x1 C:/nxp/SDKPackages/SDK_2.6.0_K32W061DK6/middleware/wireless/framework/XCVR/lib\libRadio_Test_JN518x.a(radio.o)
 .data.u32CoreVadjI1v8SetTx
                0x00000000        0x4 C:/nxp/SDKPackages/SDK_2.6.0_K32W061DK6/middleware/wireless/framework/XCVR/lib\libRadio_Test_JN518x.a(radio.o)
 .data.u32PaDccI1v1Set
                0x00000000        0x4 C:/nxp/SDKPackages/SDK_2.6.0_K32W061DK6/middleware/wireless/framework/XCVR/lib\libRadio_Test_JN518x.a(radio.o)
 .data.u32PowerstageIbiasI1v8Set
                0x00000000        0x4 C:/nxp/SDKPackages/SDK_2.6.0_K32W061DK6/middleware/wireless/framework/XCVR/lib\libRadio_Test_JN518x.a(radio.o)
 .group         0x00000000        0xc C:/nxp/SDKPackages/SDK_2.6.0_K32W061DK6/middleware/wireless/framework/XCVR/lib\libRadio_Test_JN518x.a(radio_test_jn518x.o)
 .group         0x00000000        0xc C:/nxp/SDKPackages/SDK_2.6.0_K32W061DK6/middleware/wireless/framework/XCVR/lib\libRadio_Test_JN518x.a(radio_test_jn518x.o)
 .group         0x00000000        0xc C:/nxp/SDKPackages/SDK_2.6.0_K32W061DK6/middleware/wireless/framework/XCVR/lib\libRadio_Test_JN518x.a(radio_test_jn518x.o)
 .group         0x00000000        0xc C:/nxp/SDKPackages/SDK_2.6.0_K32W061DK6/middleware/wireless/framework/XCVR/lib\libRadio_Test_JN518x.a(radio_test_jn518x.o)
 .group         0x00000000        0xc C:/nxp/SDKPackages/SDK_2.6.0_K32W061DK6/middleware/wireless/framework/XCVR/lib\libRadio_Test_JN518x.a(radio_test_jn518x.o)
 .group         0x00000000        0xc C:/nxp/SDKPackages/SDK_2.6.0_K32W061DK6/middleware/wireless/framework/XCVR/lib\libRadio_Test_JN518x.a(radio_test_jn518x.o)
 .group         0x00000000        0xc C:/nxp/SDKPackages/SDK_2.6.0_K32W061DK6/middleware/wireless/framework/XCVR/lib\libRadio_Test_JN518x.a(radio_test_jn518x.o)
 .group         0x00000000        0xc C:/nxp/SDKPackages/SDK_2.6.0_K32W061DK6/middleware/wireless/framework/XCVR/lib\libRadio_Test_JN518x.a(radio_test_jn518x.o)
 .group         0x00000000        0xc C:/nxp/SDKPackages/SDK_2.6.0_K32W061DK6/middleware/wireless/framework/XCVR/lib\libRadio_Test_JN518x.a(radio_test_jn518x.o)
 .group         0x00000000        0xc C:/nxp/SDKPackages/SDK_2.6.0_K32W061DK6/middleware/wireless/framework/XCVR/lib\libRadio_Test_JN518x.a(radio_test_jn518x.o)
 .group         0x00000000        0xc C:/nxp/SDKPackages/SDK_2.6.0_K32W061DK6/middleware/wireless/framework/XCVR/lib\libRadio_Test_JN518x.a(radio_test_jn518x.o)
 .group         0x00000000        0xc C:/nxp/SDKPackages/SDK_2.6.0_K32W061DK6/middleware/wireless/framework/XCVR/lib\libRadio_Test_JN518x.a(radio_test_jn518x.o)
 .group         0x00000000        0xc C:/nxp/SDKPackages/SDK_2.6.0_K32W061DK6/middleware/wireless/framework/XCVR/lib\libRadio_Test_JN518x.a(radio_test_jn518x.o)
 .group         0x00000000        0xc C:/nxp/SDKPackages/SDK_2.6.0_K32W061DK6/middleware/wireless/framework/XCVR/lib\libRadio_Test_JN518x.a(radio_test_jn518x.o)
 .group         0x00000000        0xc C:/nxp/SDKPackages/SDK_2.6.0_K32W061DK6/middleware/wireless/framework/XCVR/lib\libRadio_Test_JN518x.a(radio_test_jn518x.o)
 .group         0x00000000        0xc C:/nxp/SDKPackages/SDK_2.6.0_K32W061DK6/middleware/wireless/framework/XCVR/lib\libRadio_Test_JN518x.a(radio_test_jn518x.o)
 .group         0x00000000        0xc C:/nxp/SDKPackages/SDK_2.6.0_K32W061DK6/middleware/wireless/framework/XCVR/lib\libRadio_Test_JN518x.a(radio_test_jn518x.o)
 .group         0x00000000        0xc C:/nxp/SDKPackages/SDK_2.6.0_K32W061DK6/middleware/wireless/framework/XCVR/lib\libRadio_Test_JN518x.a(radio_test_jn518x.o)
 .group         0x00000000        0xc C:/nxp/SDKPackages/SDK_2.6.0_K32W061DK6/middleware/wireless/framework/XCVR/lib\libRadio_Test_JN518x.a(radio_test_jn518x.o)
 .group         0x00000000        0xc C:/nxp/SDKPackages/SDK_2.6.0_K32W061DK6/middleware/wireless/framework/XCVR/lib\libRadio_Test_JN518x.a(radio_test_jn518x.o)
 .group         0x00000000        0xc C:/nxp/SDKPackages/SDK_2.6.0_K32W061DK6/middleware/wireless/framework/XCVR/lib\libRadio_Test_JN518x.a(radio_test_jn518x.o)
 .group         0x00000000        0xc C:/nxp/SDKPackages/SDK_2.6.0_K32W061DK6/middleware/wireless/framework/XCVR/lib\libRadio_Test_JN518x.a(radio_test_jn518x.o)
 .group         0x00000000        0xc C:/nxp/SDKPackages/SDK_2.6.0_K32W061DK6/middleware/wireless/framework/XCVR/lib\libRadio_Test_JN518x.a(radio_test_jn518x.o)
 .group         0x00000000        0xc C:/nxp/SDKPackages/SDK_2.6.0_K32W061DK6/middleware/wireless/framework/XCVR/lib\libRadio_Test_JN518x.a(radio_test_jn518x.o)
 .group         0x00000000        0xc C:/nxp/SDKPackages/SDK_2.6.0_K32W061DK6/middleware/wireless/framework/XCVR/lib\libRadio_Test_JN518x.a(radio_test_jn518x.o)
 .group         0x00000000        0xc C:/nxp/SDKPackages/SDK_2.6.0_K32W061DK6/middleware/wireless/framework/XCVR/lib\libRadio_Test_JN518x.a(radio_test_jn518x.o)
 .group         0x00000000        0xc C:/nxp/SDKPackages/SDK_2.6.0_K32W061DK6/middleware/wireless/framework/XCVR/lib\libRadio_Test_JN518x.a(radio_test_jn518x.o)
 .group         0x00000000        0xc C:/nxp/SDKPackages/SDK_2.6.0_K32W061DK6/middleware/wireless/framework/XCVR/lib\libRadio_Test_JN518x.a(radio_test_jn518x.o)
 .group         0x00000000        0xc C:/nxp/SDKPackages/SDK_2.6.0_K32W061DK6/middleware/wireless/framework/XCVR/lib\libRadio_Test_JN518x.a(radio_test_jn518x.o)
 .group         0x00000000        0xc C:/nxp/SDKPackages/SDK_2.6.0_K32W061DK6/middleware/wireless/framework/XCVR/lib\libRadio_Test_JN518x.a(radio_test_jn518x.o)
 .text          0x00000000        0x0 C:/nxp/SDKPackages/SDK_2.6.0_K32W061DK6/middleware/wireless/framework/XCVR/lib\libRadio_Test_JN518x.a(radio_test_jn518x.o)
 .data          0x00000000        0x0 C:/nxp/SDKPackages/SDK_2.6.0_K32W061DK6/middleware/wireless/framework/XCVR/lib\libRadio_Test_JN518x.a(radio_test_jn518x.o)
 .bss           0x00000000        0x0 C:/nxp/SDKPackages/SDK_2.6.0_K32W061DK6/middleware/wireless/framework/XCVR/lib\libRadio_Test_JN518x.a(radio_test_jn518x.o)
 .text.u32Radio_Test_Jn518x_Init
                0x00000000       0x40 C:/nxp/SDKPackages/SDK_2.6.0_K32W061DK6/middleware/wireless/framework/XCVR/lib\libRadio_Test_JN518x.a(radio_test_jn518x.o)
 .text.vRadio_Test_Jn518x_PostRadioInit
                0x00000000       0xa0 C:/nxp/SDKPackages/SDK_2.6.0_K32W061DK6/middleware/wireless/framework/XCVR/lib\libRadio_Test_JN518x.a(radio_test_jn518x.o)
 .text.vRadio_Test_Jn518x_RadioInit
                0x00000000       0xa0 C:/nxp/SDKPackages/SDK_2.6.0_K32W061DK6/middleware/wireless/framework/XCVR/lib\libRadio_Test_JN518x.a(radio_test_jn518x.o)
 .text.vRadio_Test_Jn518x_AntennaDiversityPinEnable
                0x00000000       0x8c C:/nxp/SDKPackages/SDK_2.6.0_K32W061DK6/middleware/wireless/framework/XCVR/lib\libRadio_Test_JN518x.a(radio_test_jn518x.o)
 .text.u32GetDieID
                0x00000000        0xa C:/nxp/SDKPackages/SDK_2.6.0_K32W061DK6/middleware/wireless/framework/XCVR/lib\libRadio_Test_JN518x.a(radio_test_jn518x.o)
 .text.vRadio_Test_Jn518x_PacketTxSend
                0x00000000       0xe0 C:/nxp/SDKPackages/SDK_2.6.0_K32W061DK6/middleware/wireless/framework/XCVR/lib\libRadio_Test_JN518x.a(radio_test_jn518x.o)
 .text.bRadio_Test_Jn518x_PacketTxWaitTransmitted
                0x00000000       0x20 C:/nxp/SDKPackages/SDK_2.6.0_K32W061DK6/middleware/wireless/framework/XCVR/lib\libRadio_Test_JN518x.a(radio_test_jn518x.o)
 .text.bRadio_Test_Jn518x_PacketTxWaitPhyTransmitted
                0x00000000       0x34 C:/nxp/SDKPackages/SDK_2.6.0_K32W061DK6/middleware/wireless/framework/XCVR/lib\libRadio_Test_JN518x.a(radio_test_jn518x.o)
 .text.bRadio_Test_Jn518x_PacketRx
                0x00000000       0xec C:/nxp/SDKPackages/SDK_2.6.0_K32W061DK6/middleware/wireless/framework/XCVR/lib\libRadio_Test_JN518x.a(radio_test_jn518x.o)
 .text.bRadio_Test_Jn518x_RadioSetChannel
                0x00000000       0x48 C:/nxp/SDKPackages/SDK_2.6.0_K32W061DK6/middleware/wireless/framework/XCVR/lib\libRadio_Test_JN518x.a(radio_test_jn518x.o)
 .text.u8Radio_Test_Jn518x_RadioGetChannel
                0x00000000       0x10 C:/nxp/SDKPackages/SDK_2.6.0_K32W061DK6/middleware/wireless/framework/XCVR/lib\libRadio_Test_JN518x.a(radio_test_jn518x.o)
 .text.i8Radio_Test_Jn518x_RadioGetPower
                0x00000000        0xc C:/nxp/SDKPackages/SDK_2.6.0_K32W061DK6/middleware/wireless/framework/XCVR/lib\libRadio_Test_JN518x.a(radio_test_jn518x.o)
 .text.vRadio_Test_Jn518x_RadioSetPower
                0x00000000       0x60 C:/nxp/SDKPackages/SDK_2.6.0_K32W061DK6/middleware/wireless/framework/XCVR/lib\libRadio_Test_JN518x.a(radio_test_jn518x.o)
 .text.i16Radio_Test_Jn518x_GetRSSI
                0x00000000       0x90 C:/nxp/SDKPackages/SDK_2.6.0_K32W061DK6/middleware/wireless/framework/XCVR/lib\libRadio_Test_JN518x.a(radio_test_jn518x.o)
 .text.vRadio_Test_Jn518x_Set_Max_Gains_and_Release
                0x00000000       0x88 C:/nxp/SDKPackages/SDK_2.6.0_K32W061DK6/middleware/wireless/framework/XCVR/lib\libRadio_Test_JN518x.a(radio_test_jn518x.o)
 .text.vRadio_Test_Jn518x_Set_Min_Gains_and_Release
                0x00000000       0x7c C:/nxp/SDKPackages/SDK_2.6.0_K32W061DK6/middleware/wireless/framework/XCVR/lib\libRadio_Test_JN518x.a(radio_test_jn518x.o)
 .text.vRadio_Test_Jn518x_Freeze_Gains
                0x00000000       0x34 C:/nxp/SDKPackages/SDK_2.6.0_K32W061DK6/middleware/wireless/framework/XCVR/lib\libRadio_Test_JN518x.a(radio_test_jn518x.o)
 .text.vRadio_Test_Jn518x_Set_Max_Gains
                0x00000000       0x3c C:/nxp/SDKPackages/SDK_2.6.0_K32W061DK6/middleware/wireless/framework/XCVR/lib\libRadio_Test_JN518x.a(radio_test_jn518x.o)
 .text.vRadio_Test_Jn518x_Set_Min_Gains
                0x00000000       0x34 C:/nxp/SDKPackages/SDK_2.6.0_K32W061DK6/middleware/wireless/framework/XCVR/lib\libRadio_Test_JN518x.a(radio_test_jn518x.o)
 .text.vRadio_Test_Jn518x_Release_Gains
                0x00000000       0x2c C:/nxp/SDKPackages/SDK_2.6.0_K32W061DK6/middleware/wireless/framework/XCVR/lib\libRadio_Test_JN518x.a(radio_test_jn518x.o)
 .text.bRadio_Test_Jn518x_CCA
                0x00000000      0x16c C:/nxp/SDKPackages/SDK_2.6.0_K32W061DK6/middleware/wireless/framework/XCVR/lib\libRadio_Test_JN518x.a(radio_test_jn518x.o)
 .text.vRadio_Test_Jn518x_SetMaxInputLevel
                0x00000000        0x2 C:/nxp/SDKPackages/SDK_2.6.0_K32W061DK6/middleware/wireless/framework/XCVR/lib\libRadio_Test_JN518x.a(radio_test_jn518x.o)
 .text.vRadio_Test_Jn518x_AntennaDiversityEnable
                0x00000000        0x2 C:/nxp/SDKPackages/SDK_2.6.0_K32W061DK6/middleware/wireless/framework/XCVR/lib\libRadio_Test_JN518x.a(radio_test_jn518x.o)
 .text.vRadio_Test_Jn518x_TxPowerAdjust
                0x00000000        0x2 C:/nxp/SDKPackages/SDK_2.6.0_K32W061DK6/middleware/wireless/framework/XCVR/lib\libRadio_Test_JN518x.a(radio_test_jn518x.o)
 .text.i8Radio_Test_Jn518x_RadioGetPowerFine
                0x00000000        0x4 C:/nxp/SDKPackages/SDK_2.6.0_K32W061DK6/middleware/wireless/framework/XCVR/lib\libRadio_Test_JN518x.a(radio_test_jn518x.o)
 .text.vRadio_Test_Jn518x_RadioSetPowerFine
                0x00000000        0x2 C:/nxp/SDKPackages/SDK_2.6.0_K32W061DK6/middleware/wireless/framework/XCVR/lib\libRadio_Test_JN518x.a(radio_test_jn518x.o)
 .text.u32Radio_Test_Jn518x_WaitPacket
                0x00000000       0x68 C:/nxp/SDKPackages/SDK_2.6.0_K32W061DK6/middleware/wireless/framework/XCVR/lib\libRadio_Test_JN518x.a(radio_test_jn518x.o)
 .text.u32Radio_Test_Jn518x_TPT_WaitPacket
                0x00000000       0x1c C:/nxp/SDKPackages/SDK_2.6.0_K32W061DK6/middleware/wireless/framework/XCVR/lib\libRadio_Test_JN518x.a(radio_test_jn518x.o)
 .text.vRadio_Test_Jn518x_BLE_PacketTx_Start
                0x00000000      0x254 C:/nxp/SDKPackages/SDK_2.6.0_K32W061DK6/middleware/wireless/framework/XCVR/lib\libRadio_Test_JN518x.a(radio_test_jn518x.o)
 .text.u32Radio_Test_Jn518x_BLE_PacketTx_Loop
                0x00000000        0xc C:/nxp/SDKPackages/SDK_2.6.0_K32W061DK6/middleware/wireless/framework/XCVR/lib\libRadio_Test_JN518x.a(radio_test_jn518x.o)
 .text.vRadio_Test_Jn518x_BLE_PacketRx_Start
                0x00000000      0x1b0 C:/nxp/SDKPackages/SDK_2.6.0_K32W061DK6/middleware/wireless/framework/XCVR/lib\libRadio_Test_JN518x.a(radio_test_jn518x.o)
 .text.u32Radio_Test_Jn518x_BLE_PacketRx_Loop
                0x00000000        0xc C:/nxp/SDKPackages/SDK_2.6.0_K32W061DK6/middleware/wireless/framework/XCVR/lib\libRadio_Test_JN518x.a(radio_test_jn518x.o)
 .text.RX_descriptor_decode
                0x00000000       0x30 C:/nxp/SDKPackages/SDK_2.6.0_K32W061DK6/middleware/wireless/framework/XCVR/lib\libRadio_Test_JN518x.a(radio_test_jn518x.o)
 .text.bRadio_Test_Jn518x_PT_FrameTxComplete
                0x00000000       0x30 C:/nxp/SDKPackages/SDK_2.6.0_K32W061DK6/middleware/wireless/framework/XCVR/lib\libRadio_Test_JN518x.a(radio_test_jn518x.o)
 .text.vRadio_Test_Jn518x_PacketTx
                0x00000000       0x16 C:/nxp/SDKPackages/SDK_2.6.0_K32W061DK6/middleware/wireless/framework/XCVR/lib\libRadio_Test_JN518x.a(radio_test_jn518x.o)
 .text.u8Radio_Test_Jn518x_GetLQIfromRSSI
                0x00000000       0x2a C:/nxp/SDKPackages/SDK_2.6.0_K32W061DK6/middleware/wireless/framework/XCVR/lib\libRadio_Test_JN518x.a(radio_test_jn518x.o)
 .text.vPrintDebugInfos
                0x00000000        0x2 C:/nxp/SDKPackages/SDK_2.6.0_K32W061DK6/middleware/wireless/framework/XCVR/lib\libRadio_Test_JN518x.a(radio_test_jn518x.o)
 .text.vRadio_Test_Jn518x_Print_RFP_registers
                0x00000000        0x2 C:/nxp/SDKPackages/SDK_2.6.0_K32W061DK6/middleware/wireless/framework/XCVR/lib\libRadio_Test_JN518x.a(radio_test_jn518x.o)
 .text.vRadio_Test_Jn518x_Print_transceiver_registers
                0x00000000        0x2 C:/nxp/SDKPackages/SDK_2.6.0_K32W061DK6/middleware/wireless/framework/XCVR/lib\libRadio_Test_JN518x.a(radio_test_jn518x.o)
 .text.vRadio_Test_jn518x_Read_Cal_Values
                0x00000000       0xe0 C:/nxp/SDKPackages/SDK_2.6.0_K32W061DK6/middleware/wireless/framework/XCVR/lib\libRadio_Test_JN518x.a(radio_test_jn518x.o)
 .text.vRadio_Test_jn518x_Print_Cal_Values
                0x00000000        0x2 C:/nxp/SDKPackages/SDK_2.6.0_K32W061DK6/middleware/wireless/framework/XCVR/lib\libRadio_Test_JN518x.a(radio_test_jn518x.o)
 .text.vRadio_Test_Jn518x_DisableRXTX
                0x00000000       0x28 C:/nxp/SDKPackages/SDK_2.6.0_K32W061DK6/middleware/wireless/framework/XCVR/lib\libRadio_Test_JN518x.a(radio_test_jn518x.o)
 .text.vRadio_Test_Jn518x_SetTXMBEBT
                0x00000000       0x24 C:/nxp/SDKPackages/SDK_2.6.0_K32W061DK6/middleware/wireless/framework/XCVR/lib\libRadio_Test_JN518x.a(radio_test_jn518x.o)
 .text.vRadio_Test_Jn518x_Enable_ITs_RFT1788
                0x00000000       0xa8 C:/nxp/SDKPackages/SDK_2.6.0_K32W061DK6/middleware/wireless/framework/XCVR/lib\libRadio_Test_JN518x.a(radio_test_jn518x.o)
 .text.vRadio_Test_Jn518x_StartRX_ACK_NOPROM
                0x00000000       0x24 C:/nxp/SDKPackages/SDK_2.6.0_K32W061DK6/middleware/wireless/framework/XCVR/lib\libRadio_Test_JN518x.a(radio_test_jn518x.o)
 .text.vRadio_Test_Jn518x_StartRX_ACK_PROM
                0x00000000       0x20 C:/nxp/SDKPackages/SDK_2.6.0_K32W061DK6/middleware/wireless/framework/XCVR/lib\libRadio_Test_JN518x.a(radio_test_jn518x.o)
 .text.vRadio_Test_Jn518x_TPT_Start
                0x00000000       0x44 C:/nxp/SDKPackages/SDK_2.6.0_K32W061DK6/middleware/wireless/framework/XCVR/lib\libRadio_Test_JN518x.a(radio_test_jn518x.o)
 .text.vRadio_Test_Jn518x_TPT_Start_ISR
                0x00000000       0x18 C:/nxp/SDKPackages/SDK_2.6.0_K32W061DK6/middleware/wireless/framework/XCVR/lib\libRadio_Test_JN518x.a(radio_test_jn518x.o)
 .text.vRadio_Test_Jn518x_Disable_ITs_RFT1778
                0x00000000       0x64 C:/nxp/SDKPackages/SDK_2.6.0_K32W061DK6/middleware/wireless/framework/XCVR/lib\libRadio_Test_JN518x.a(radio_test_jn518x.o)
 .text.vRadio_Test_Jn518x_RadioDeInit
                0x00000000       0x40 C:/nxp/SDKPackages/SDK_2.6.0_K32W061DK6/middleware/wireless/framework/XCVR/lib\libRadio_Test_JN518x.a(radio_test_jn518x.o)
 .text.vRadio_Test_Jn518x_TPT_Stop
                0x00000000       0x3c C:/nxp/SDKPackages/SDK_2.6.0_K32W061DK6/middleware/wireless/framework/XCVR/lib\libRadio_Test_JN518x.a(radio_test_jn518x.o)
 .text.vRadio_Test_Jn518x_Register_ISR_MAC_Handler
                0x00000000        0xc C:/nxp/SDKPackages/SDK_2.6.0_K32W061DK6/middleware/wireless/framework/XCVR/lib\libRadio_Test_JN518x.a(radio_test_jn518x.o)
 .text.radio_test_jn518x_PowerOn
                0x00000000      0x178 C:/nxp/SDKPackages/SDK_2.6.0_K32W061DK6/middleware/wireless/framework/XCVR/lib\libRadio_Test_JN518x.a(radio_test_jn518x.o)
 .text.vRadio_Test_JN518x_XO_Trim
                0x00000000       0x3c C:/nxp/SDKPackages/SDK_2.6.0_K32W061DK6/middleware/wireless/framework/XCVR/lib\libRadio_Test_JN518x.a(radio_test_jn518x.o)
 .text.vRadio_test_jn518x_InitXtal
                0x00000000       0x54 C:/nxp/SDKPackages/SDK_2.6.0_K32W061DK6/middleware/wireless/framework/XCVR/lib\libRadio_Test_JN518x.a(radio_test_jn518x.o)
 .text.vRadio_Test_Jn518x_PA_cal_ate_result
                0x00000000       0x3c C:/nxp/SDKPackages/SDK_2.6.0_K32W061DK6/middleware/wireless/framework/XCVR/lib\libRadio_Test_JN518x.a(radio_test_jn518x.o)
 .text.vRadio_Test_Print_Banked_Registers
                0x00000000       0x30 C:/nxp/SDKPackages/SDK_2.6.0_K32W061DK6/middleware/wireless/framework/XCVR/lib\libRadio_Test_JN518x.a(radio_test_jn518x.o)
 .text.vRadio_Test_Reset_RadioConfig
                0x00000000        0x8 C:/nxp/SDKPackages/SDK_2.6.0_K32W061DK6/middleware/wireless/framework/XCVR/lib\libRadio_Test_JN518x.a(radio_test_jn518x.o)
 .rodata        0x00000000       0x94 C:/nxp/SDKPackages/SDK_2.6.0_K32W061DK6/middleware/wireless/framework/XCVR/lib\libRadio_Test_JN518x.a(radio_test_jn518x.o)
 .bss.AcceptMal
                0x00000000        0x4 C:/nxp/SDKPackages/SDK_2.6.0_K32W061DK6/middleware/wireless/framework/XCVR/lib\libRadio_Test_JN518x.a(radio_test_jn518x.o)
 .bss.AddressMatch
                0x00000000        0x4 C:/nxp/SDKPackages/SDK_2.6.0_K32W061DK6/middleware/wireless/framework/XCVR/lib\libRadio_Test_JN518x.a(radio_test_jn518x.o)
 .bss.MaxPayLen
                0x00000000        0x4 C:/nxp/SDKPackages/SDK_2.6.0_K32W061DK6/middleware/wireless/framework/XCVR/lib\libRadio_Test_JN518x.a(radio_test_jn518x.o)
 .bss.PhyMode   0x00000000        0x4 C:/nxp/SDKPackages/SDK_2.6.0_K32W061DK6/middleware/wireless/framework/XCVR/lib\libRadio_Test_JN518x.a(radio_test_jn518x.o)
 .bss.Sniff     0x00000000        0x4 C:/nxp/SDKPackages/SDK_2.6.0_K32W061DK6/middleware/wireless/framework/XCVR/lib\libRadio_Test_JN518x.a(radio_test_jn518x.o)
 .bss.TxAck     0x00000000        0x4 C:/nxp/SDKPackages/SDK_2.6.0_K32W061DK6/middleware/wireless/framework/XCVR/lib\libRadio_Test_JN518x.a(radio_test_jn518x.o)
 .bss.TxCSMA    0x00000000        0x4 C:/nxp/SDKPackages/SDK_2.6.0_K32W061DK6/middleware/wireless/framework/XCVR/lib\libRadio_Test_JN518x.a(radio_test_jn518x.o)
 .bss.bPatchActivated
                0x00000000        0x1 C:/nxp/SDKPackages/SDK_2.6.0_K32W061DK6/middleware/wireless/framework/XCVR/lib\libRadio_Test_JN518x.a(radio_test_jn518x.o)
 .bss.u32BbcRxprom
                0x00000000        0x4 C:/nxp/SDKPackages/SDK_2.6.0_K32W061DK6/middleware/wireless/framework/XCVR/lib\libRadio_Test_JN518x.a(radio_test_jn518x.o)
 .bss.u32SniffWorkaroundTimer.21664
                0x00000000        0x4 C:/nxp/SDKPackages/SDK_2.6.0_K32W061DK6/middleware/wireless/framework/XCVR/lib\libRadio_Test_JN518x.a(radio_test_jn518x.o)
 .bss.u8SQI.21665
                0x00000000        0x1 C:/nxp/SDKPackages/SDK_2.6.0_K32W061DK6/middleware/wireless/framework/XCVR/lib\libRadio_Test_JN518x.a(radio_test_jn518x.o)
 .data.TotalPackets
                0x00000000        0x4 C:/nxp/SDKPackages/SDK_2.6.0_K32W061DK6/middleware/wireless/framework/XCVR/lib\libRadio_Test_JN518x.a(radio_test_jn518x.o)
 .data.TxTries  0x00000000        0x4 C:/nxp/SDKPackages/SDK_2.6.0_K32W061DK6/middleware/wireless/framework/XCVR/lib\libRadio_Test_JN518x.a(radio_test_jn518x.o)
 .data.u16ADConfigThr
                0x00000000        0x2 C:/nxp/SDKPackages/SDK_2.6.0_K32W061DK6/middleware/wireless/framework/XCVR/lib\libRadio_Test_JN518x.a(radio_test_jn518x.o)
 .data.u8ADConfigTimer
                0x00000000        0x1 C:/nxp/SDKPackages/SDK_2.6.0_K32W061DK6/middleware/wireless/framework/XCVR/lib\libRadio_Test_JN518x.a(radio_test_jn518x.o)
 .debug_macro   0x00000000      0xaa8 C:/nxp/SDKPackages/SDK_2.6.0_K32W061DK6/middleware/wireless/framework/XCVR/lib\libRadio_Test_JN518x.a(radio_test_jn518x.o)
 .debug_macro   0x00000000       0x10 C:/nxp/SDKPackages/SDK_2.6.0_K32W061DK6/middleware/wireless/framework/XCVR/lib\libRadio_Test_JN518x.a(radio_test_jn518x.o)
 .debug_macro   0x00000000       0x22 C:/nxp/SDKPackages/SDK_2.6.0_K32W061DK6/middleware/wireless/framework/XCVR/lib\libRadio_Test_JN518x.a(radio_test_jn518x.o)
 .debug_macro   0x00000000      0x12e C:/nxp/SDKPackages/SDK_2.6.0_K32W061DK6/middleware/wireless/framework/XCVR/lib\libRadio_Test_JN518x.a(radio_test_jn518x.o)
 .debug_macro   0x00000000      0x5b3 C:/nxp/SDKPackages/SDK_2.6.0_K32W061DK6/middleware/wireless/framework/XCVR/lib\libRadio_Test_JN518x.a(radio_test_jn518x.o)
 .debug_macro   0x00000000       0x22 C:/nxp/SDKPackages/SDK_2.6.0_K32W061DK6/middleware/wireless/framework/XCVR/lib\libRadio_Test_JN518x.a(radio_test_jn518x.o)
 .debug_macro   0x00000000       0x16 C:/nxp/SDKPackages/SDK_2.6.0_K32W061DK6/middleware/wireless/framework/XCVR/lib\libRadio_Test_JN518x.a(radio_test_jn518x.o)
 .debug_macro   0x00000000       0x38 C:/nxp/SDKPackages/SDK_2.6.0_K32W061DK6/middleware/wireless/framework/XCVR/lib\libRadio_Test_JN518x.a(radio_test_jn518x.o)
 .debug_macro   0x00000000       0x1c C:/nxp/SDKPackages/SDK_2.6.0_K32W061DK6/middleware/wireless/framework/XCVR/lib\libRadio_Test_JN518x.a(radio_test_jn518x.o)
 .debug_macro   0x00000000       0x22 C:/nxp/SDKPackages/SDK_2.6.0_K32W061DK6/middleware/wireless/framework/XCVR/lib\libRadio_Test_JN518x.a(radio_test_jn518x.o)
 .debug_macro   0x00000000       0xdf C:/nxp/SDKPackages/SDK_2.6.0_K32W061DK6/middleware/wireless/framework/XCVR/lib\libRadio_Test_JN518x.a(radio_test_jn518x.o)
 .debug_macro   0x00000000      0xff5 C:/nxp/SDKPackages/SDK_2.6.0_K32W061DK6/middleware/wireless/framework/XCVR/lib\libRadio_Test_JN518x.a(radio_test_jn518x.o)
 .debug_macro   0x00000000       0xe2 C:/nxp/SDKPackages/SDK_2.6.0_K32W061DK6/middleware/wireless/framework/XCVR/lib\libRadio_Test_JN518x.a(radio_test_jn518x.o)
 .debug_macro   0x00000000       0x10 C:/nxp/SDKPackages/SDK_2.6.0_K32W061DK6/middleware/wireless/framework/XCVR/lib\libRadio_Test_JN518x.a(radio_test_jn518x.o)
 .debug_macro   0x00000000     0x9cc0 C:/nxp/SDKPackages/SDK_2.6.0_K32W061DK6/middleware/wireless/framework/XCVR/lib\libRadio_Test_JN518x.a(radio_test_jn518x.o)
 .debug_macro   0x00000000      0x213 C:/nxp/SDKPackages/SDK_2.6.0_K32W061DK6/middleware/wireless/framework/XCVR/lib\libRadio_Test_JN518x.a(radio_test_jn518x.o)
 .debug_macro   0x00000000       0xd0 C:/nxp/SDKPackages/SDK_2.6.0_K32W061DK6/middleware/wireless/framework/XCVR/lib\libRadio_Test_JN518x.a(radio_test_jn518x.o)
 .debug_macro   0x00000000       0x16 C:/nxp/SDKPackages/SDK_2.6.0_K32W061DK6/middleware/wireless/framework/XCVR/lib\libRadio_Test_JN518x.a(radio_test_jn518x.o)
 .debug_macro   0x00000000       0xa9 C:/nxp/SDKPackages/SDK_2.6.0_K32W061DK6/middleware/wireless/framework/XCVR/lib\libRadio_Test_JN518x.a(radio_test_jn518x.o)
 .debug_macro   0x00000000       0xbc C:/nxp/SDKPackages/SDK_2.6.0_K32W061DK6/middleware/wireless/framework/XCVR/lib\libRadio_Test_JN518x.a(radio_test_jn518x.o)
 .debug_macro   0x00000000       0xcf C:/nxp/SDKPackages/SDK_2.6.0_K32W061DK6/middleware/wireless/framework/XCVR/lib\libRadio_Test_JN518x.a(radio_test_jn518x.o)
 .debug_macro   0x00000000       0x10 C:/nxp/SDKPackages/SDK_2.6.0_K32W061DK6/middleware/wireless/framework/XCVR/lib\libRadio_Test_JN518x.a(radio_test_jn518x.o)
 .debug_macro   0x00000000      0x398 C:/nxp/SDKPackages/SDK_2.6.0_K32W061DK6/middleware/wireless/framework/XCVR/lib\libRadio_Test_JN518x.a(radio_test_jn518x.o)
 .debug_macro   0x00000000      0x4f6 C:/nxp/SDKPackages/SDK_2.6.0_K32W061DK6/middleware/wireless/framework/XCVR/lib\libRadio_Test_JN518x.a(radio_test_jn518x.o)
 .debug_macro   0x00000000      0x494 C:/nxp/SDKPackages/SDK_2.6.0_K32W061DK6/middleware/wireless/framework/XCVR/lib\libRadio_Test_JN518x.a(radio_test_jn518x.o)
 .debug_macro   0x00000000     0xddcb C:/nxp/SDKPackages/SDK_2.6.0_K32W061DK6/middleware/wireless/framework/XCVR/lib\libRadio_Test_JN518x.a(radio_test_jn518x.o)
 .debug_macro   0x00000000     0xd2d4 C:/nxp/SDKPackages/SDK_2.6.0_K32W061DK6/middleware/wireless/framework/XCVR/lib\libRadio_Test_JN518x.a(radio_test_jn518x.o)
 .debug_macro   0x00000000      0x150 C:/nxp/SDKPackages/SDK_2.6.0_K32W061DK6/middleware/wireless/framework/XCVR/lib\libRadio_Test_JN518x.a(radio_test_jn518x.o)
 .debug_macro   0x00000000       0xff C:/nxp/SDKPackages/SDK_2.6.0_K32W061DK6/middleware/wireless/framework/XCVR/lib\libRadio_Test_JN518x.a(radio_test_jn518x.o)
 COMMON         0x00000000      0x24c C:/nxp/SDKPackages/SDK_2.6.0_K32W061DK6/middleware/wireless/framework/XCVR/lib\libRadio_Test_JN518x.a(radio_test_jn518x.o)
 .data          0x00000000        0x0 c:/nxp/mcuxpressoide_11.1.0_3209/ide/plugins/com.nxp.mcuxpresso.tools.win32_11.1.0.201909161352/tools/bin/../lib/gcc/arm-none-eabi/8.3.1/thumb/v7e-m/nofp\libgcc.a(_arm_addsubdf3.o)
 .bss           0x00000000        0x0 c:/nxp/mcuxpressoide_11.1.0_3209/ide/plugins/com.nxp.mcuxpresso.tools.win32_11.1.0.201909161352/tools/bin/../lib/gcc/arm-none-eabi/8.3.1/thumb/v7e-m/nofp\libgcc.a(_arm_addsubdf3.o)
 .data          0x00000000        0x0 c:/nxp/mcuxpressoide_11.1.0_3209/ide/plugins/com.nxp.mcuxpresso.tools.win32_11.1.0.201909161352/tools/bin/../lib/gcc/arm-none-eabi/8.3.1/thumb/v7e-m/nofp\libgcc.a(_arm_fixdfsi.o)
 .bss           0x00000000        0x0 c:/nxp/mcuxpressoide_11.1.0_3209/ide/plugins/com.nxp.mcuxpresso.tools.win32_11.1.0.201909161352/tools/bin/../lib/gcc/arm-none-eabi/8.3.1/thumb/v7e-m/nofp\libgcc.a(_arm_fixdfsi.o)
 .text          0x00000000       0xa0 c:/nxp/mcuxpressoide_11.1.0_3209/ide/plugins/com.nxp.mcuxpresso.tools.win32_11.1.0.201909161352/tools/bin/../lib/gcc/arm-none-eabi/8.3.1/thumb/v7e-m/nofp\libgcc.a(_aeabi_ldivmod.o)
 .data          0x00000000        0x0 c:/nxp/mcuxpressoide_11.1.0_3209/ide/plugins/com.nxp.mcuxpresso.tools.win32_11.1.0.201909161352/tools/bin/../lib/gcc/arm-none-eabi/8.3.1/thumb/v7e-m/nofp\libgcc.a(_aeabi_ldivmod.o)
 .bss           0x00000000        0x0 c:/nxp/mcuxpressoide_11.1.0_3209/ide/plugins/com.nxp.mcuxpresso.tools.win32_11.1.0.201909161352/tools/bin/../lib/gcc/arm-none-eabi/8.3.1/thumb/v7e-m/nofp\libgcc.a(_aeabi_ldivmod.o)
 .debug_frame   0x00000000       0x44 c:/nxp/mcuxpressoide_11.1.0_3209/ide/plugins/com.nxp.mcuxpresso.tools.win32_11.1.0.201909161352/tools/bin/../lib/gcc/arm-none-eabi/8.3.1/thumb/v7e-m/nofp\libgcc.a(_aeabi_ldivmod.o)
 .ARM.attributes
                0x00000000       0x1e c:/nxp/mcuxpressoide_11.1.0_3209/ide/plugins/com.nxp.mcuxpresso.tools.win32_11.1.0.201909161352/tools/bin/../lib/gcc/arm-none-eabi/8.3.1/thumb/v7e-m/nofp\libgcc.a(_aeabi_ldivmod.o)
 .data          0x00000000        0x0 c:/nxp/mcuxpressoide_11.1.0_3209/ide/plugins/com.nxp.mcuxpresso.tools.win32_11.1.0.201909161352/tools/bin/../lib/gcc/arm-none-eabi/8.3.1/thumb/v7e-m/nofp\libgcc.a(_aeabi_uldivmod.o)
 .bss           0x00000000        0x0 c:/nxp/mcuxpressoide_11.1.0_3209/ide/plugins/com.nxp.mcuxpresso.tools.win32_11.1.0.201909161352/tools/bin/../lib/gcc/arm-none-eabi/8.3.1/thumb/v7e-m/nofp\libgcc.a(_aeabi_uldivmod.o)
 .data          0x00000000        0x0 c:/nxp/mcuxpressoide_11.1.0_3209/ide/plugins/com.nxp.mcuxpresso.tools.win32_11.1.0.201909161352/tools/bin/../lib/gcc/arm-none-eabi/8.3.1/thumb/v7e-m/nofp\libgcc.a(_udivmoddi4.o)
 .bss           0x00000000        0x0 c:/nxp/mcuxpressoide_11.1.0_3209/ide/plugins/com.nxp.mcuxpresso.tools.win32_11.1.0.201909161352/tools/bin/../lib/gcc/arm-none-eabi/8.3.1/thumb/v7e-m/nofp\libgcc.a(_udivmoddi4.o)
 .ARM.extab     0x00000000        0x0 c:/nxp/mcuxpressoide_11.1.0_3209/ide/plugins/com.nxp.mcuxpresso.tools.win32_11.1.0.201909161352/tools/bin/../lib/gcc/arm-none-eabi/8.3.1/thumb/v7e-m/nofp\libgcc.a(_udivmoddi4.o)
 .data          0x00000000        0x0 c:/nxp/mcuxpressoide_11.1.0_3209/ide/plugins/com.nxp.mcuxpresso.tools.win32_11.1.0.201909161352/tools/bin/../lib/gcc/arm-none-eabi/8.3.1/thumb/v7e-m/nofp\libgcc.a(_dvmd_tls.o)
 .bss           0x00000000        0x0 c:/nxp/mcuxpressoide_11.1.0_3209/ide/plugins/com.nxp.mcuxpresso.tools.win32_11.1.0.201909161352/tools/bin/../lib/gcc/arm-none-eabi/8.3.1/thumb/v7e-m/nofp\libgcc.a(_dvmd_tls.o)
 .text          0x00000000        0x0 c:/nxp/mcuxpressoide_11.1.0_3209/ide/plugins/com.nxp.mcuxpresso.tools.win32_11.1.0.201909161352/tools/bin/../lib/gcc/arm-none-eabi/8.3.1/../../../../arm-none-eabi/lib/thumb/v7e-m/nofp\libg.a(lib_a-abs.o)
 .data          0x00000000        0x0 c:/nxp/mcuxpressoide_11.1.0_3209/ide/plugins/com.nxp.mcuxpresso.tools.win32_11.1.0.201909161352/tools/bin/../lib/gcc/arm-none-eabi/8.3.1/../../../../arm-none-eabi/lib/thumb/v7e-m/nofp\libg.a(lib_a-abs.o)
 .bss           0x00000000        0x0 c:/nxp/mcuxpressoide_11.1.0_3209/ide/plugins/com.nxp.mcuxpresso.tools.win32_11.1.0.201909161352/tools/bin/../lib/gcc/arm-none-eabi/8.3.1/../../../../arm-none-eabi/lib/thumb/v7e-m/nofp\libg.a(lib_a-abs.o)
 .text          0x00000000        0x0 c:/nxp/mcuxpressoide_11.1.0_3209/ide/plugins/com.nxp.mcuxpresso.tools.win32_11.1.0.201909161352/tools/bin/../lib/gcc/arm-none-eabi/8.3.1/../../../../arm-none-eabi/lib/thumb/v7e-m/nofp\libg.a(lib_a-malloc.o)
 .data          0x00000000        0x0 c:/nxp/mcuxpressoide_11.1.0_3209/ide/plugins/com.nxp.mcuxpresso.tools.win32_11.1.0.201909161352/tools/bin/../lib/gcc/arm-none-eabi/8.3.1/../../../../arm-none-eabi/lib/thumb/v7e-m/nofp\libg.a(lib_a-malloc.o)
 .bss           0x00000000        0x0 c:/nxp/mcuxpressoide_11.1.0_3209/ide/plugins/com.nxp.mcuxpresso.tools.win32_11.1.0.201909161352/tools/bin/../lib/gcc/arm-none-eabi/8.3.1/../../../../arm-none-eabi/lib/thumb/v7e-m/nofp\libg.a(lib_a-malloc.o)
 .text.malloc   0x00000000       0x10 c:/nxp/mcuxpressoide_11.1.0_3209/ide/plugins/com.nxp.mcuxpresso.tools.win32_11.1.0.201909161352/tools/bin/../lib/gcc/arm-none-eabi/8.3.1/../../../../arm-none-eabi/lib/thumb/v7e-m/nofp\libg.a(lib_a-malloc.o)
 .text.free     0x00000000       0x10 c:/nxp/mcuxpressoide_11.1.0_3209/ide/plugins/com.nxp.mcuxpresso.tools.win32_11.1.0.201909161352/tools/bin/../lib/gcc/arm-none-eabi/8.3.1/../../../../arm-none-eabi/lib/thumb/v7e-m/nofp\libg.a(lib_a-malloc.o)
 .debug_frame   0x00000000       0x30 c:/nxp/mcuxpressoide_11.1.0_3209/ide/plugins/com.nxp.mcuxpresso.tools.win32_11.1.0.201909161352/tools/bin/../lib/gcc/arm-none-eabi/8.3.1/../../../../arm-none-eabi/lib/thumb/v7e-m/nofp\libg.a(lib_a-malloc.o)
 .ARM.attributes
                0x00000000       0x2e c:/nxp/mcuxpressoide_11.1.0_3209/ide/plugins/com.nxp.mcuxpresso.tools.win32_11.1.0.201909161352/tools/bin/../lib/gcc/arm-none-eabi/8.3.1/../../../../arm-none-eabi/lib/thumb/v7e-m/nofp\libg.a(lib_a-malloc.o)
 .text          0x00000000        0x0 c:/nxp/mcuxpressoide_11.1.0_3209/ide/plugins/com.nxp.mcuxpresso.tools.win32_11.1.0.201909161352/tools/bin/../lib/gcc/arm-none-eabi/8.3.1/../../../../arm-none-eabi/lib/thumb/v7e-m/nofp\libg.a(lib_a-mallocr.o)
 .data          0x00000000        0x0 c:/nxp/mcuxpressoide_11.1.0_3209/ide/plugins/com.nxp.mcuxpresso.tools.win32_11.1.0.201909161352/tools/bin/../lib/gcc/arm-none-eabi/8.3.1/../../../../arm-none-eabi/lib/thumb/v7e-m/nofp\libg.a(lib_a-mallocr.o)
 .bss           0x00000000        0x0 c:/nxp/mcuxpressoide_11.1.0_3209/ide/plugins/com.nxp.mcuxpresso.tools.win32_11.1.0.201909161352/tools/bin/../lib/gcc/arm-none-eabi/8.3.1/../../../../arm-none-eabi/lib/thumb/v7e-m/nofp\libg.a(lib_a-mallocr.o)
 .text._malloc_r
                0x00000000      0x570 c:/nxp/mcuxpressoide_11.1.0_3209/ide/plugins/com.nxp.mcuxpresso.tools.win32_11.1.0.201909161352/tools/bin/../lib/gcc/arm-none-eabi/8.3.1/../../../../arm-none-eabi/lib/thumb/v7e-m/nofp\libg.a(lib_a-mallocr.o)
 .bss.__malloc_current_mallinfo
                0x00000000       0x28 c:/nxp/mcuxpressoide_11.1.0_3209/ide/plugins/com.nxp.mcuxpresso.tools.win32_11.1.0.201909161352/tools/bin/../lib/gcc/arm-none-eabi/8.3.1/../../../../arm-none-eabi/lib/thumb/v7e-m/nofp\libg.a(lib_a-mallocr.o)
 .bss.__malloc_max_sbrked_mem
                0x00000000        0x4 c:/nxp/mcuxpressoide_11.1.0_3209/ide/plugins/com.nxp.mcuxpresso.tools.win32_11.1.0.201909161352/tools/bin/../lib/gcc/arm-none-eabi/8.3.1/../../../../arm-none-eabi/lib/thumb/v7e-m/nofp\libg.a(lib_a-mallocr.o)
 .bss.__malloc_max_total_mem
                0x00000000        0x4 c:/nxp/mcuxpressoide_11.1.0_3209/ide/plugins/com.nxp.mcuxpresso.tools.win32_11.1.0.201909161352/tools/bin/../lib/gcc/arm-none-eabi/8.3.1/../../../../arm-none-eabi/lib/thumb/v7e-m/nofp\libg.a(lib_a-mallocr.o)
 .bss.__malloc_top_pad
                0x00000000        0x4 c:/nxp/mcuxpressoide_11.1.0_3209/ide/plugins/com.nxp.mcuxpresso.tools.win32_11.1.0.201909161352/tools/bin/../lib/gcc/arm-none-eabi/8.3.1/../../../../arm-none-eabi/lib/thumb/v7e-m/nofp\libg.a(lib_a-mallocr.o)
 .data.__malloc_av_
                0x00000000      0x408 c:/nxp/mcuxpressoide_11.1.0_3209/ide/plugins/com.nxp.mcuxpresso.tools.win32_11.1.0.201909161352/tools/bin/../lib/gcc/arm-none-eabi/8.3.1/../../../../arm-none-eabi/lib/thumb/v7e-m/nofp\libg.a(lib_a-mallocr.o)
 .data.__malloc_sbrk_base
                0x00000000        0x4 c:/nxp/mcuxpressoide_11.1.0_3209/ide/plugins/com.nxp.mcuxpresso.tools.win32_11.1.0.201909161352/tools/bin/../lib/gcc/arm-none-eabi/8.3.1/../../../../arm-none-eabi/lib/thumb/v7e-m/nofp\libg.a(lib_a-mallocr.o)
 .data.__malloc_trim_threshold
                0x00000000        0x4 c:/nxp/mcuxpressoide_11.1.0_3209/ide/plugins/com.nxp.mcuxpresso.tools.win32_11.1.0.201909161352/tools/bin/../lib/gcc/arm-none-eabi/8.3.1/../../../../arm-none-eabi/lib/thumb/v7e-m/nofp\libg.a(lib_a-mallocr.o)
 .debug_frame   0x00000000       0x4c c:/nxp/mcuxpressoide_11.1.0_3209/ide/plugins/com.nxp.mcuxpresso.tools.win32_11.1.0.201909161352/tools/bin/../lib/gcc/arm-none-eabi/8.3.1/../../../../arm-none-eabi/lib/thumb/v7e-m/nofp\libg.a(lib_a-mallocr.o)
 .ARM.attributes
                0x00000000       0x2e c:/nxp/mcuxpressoide_11.1.0_3209/ide/plugins/com.nxp.mcuxpresso.tools.win32_11.1.0.201909161352/tools/bin/../lib/gcc/arm-none-eabi/8.3.1/../../../../arm-none-eabi/lib/thumb/v7e-m/nofp\libg.a(lib_a-mallocr.o)
 .data          0x00000000        0x0 c:/nxp/mcuxpressoide_11.1.0_3209/ide/plugins/com.nxp.mcuxpresso.tools.win32_11.1.0.201909161352/tools/bin/../lib/gcc/arm-none-eabi/8.3.1/../../../../arm-none-eabi/lib/thumb/v7e-m/nofp\libg.a(lib_a-memcpy.o)
 .bss           0x00000000        0x0 c:/nxp/mcuxpressoide_11.1.0_3209/ide/plugins/com.nxp.mcuxpresso.tools.win32_11.1.0.201909161352/tools/bin/../lib/gcc/arm-none-eabi/8.3.1/../../../../arm-none-eabi/lib/thumb/v7e-m/nofp\libg.a(lib_a-memcpy.o)
 .text          0x00000000        0x0 c:/nxp/mcuxpressoide_11.1.0_3209/ide/plugins/com.nxp.mcuxpresso.tools.win32_11.1.0.201909161352/tools/bin/../lib/gcc/arm-none-eabi/8.3.1/../../../../arm-none-eabi/lib/thumb/v7e-m/nofp\libg.a(lib_a-memset.o)
 .data          0x00000000        0x0 c:/nxp/mcuxpressoide_11.1.0_3209/ide/plugins/com.nxp.mcuxpresso.tools.win32_11.1.0.201909161352/tools/bin/../lib/gcc/arm-none-eabi/8.3.1/../../../../arm-none-eabi/lib/thumb/v7e-m/nofp\libg.a(lib_a-memset.o)
 .bss           0x00000000        0x0 c:/nxp/mcuxpressoide_11.1.0_3209/ide/plugins/com.nxp.mcuxpresso.tools.win32_11.1.0.201909161352/tools/bin/../lib/gcc/arm-none-eabi/8.3.1/../../../../arm-none-eabi/lib/thumb/v7e-m/nofp\libg.a(lib_a-memset.o)
 .text          0x00000000        0x0 c:/nxp/mcuxpressoide_11.1.0_3209/ide/plugins/com.nxp.mcuxpresso.tools.win32_11.1.0.201909161352/tools/bin/../lib/gcc/arm-none-eabi/8.3.1/../../../../arm-none-eabi/lib/thumb/v7e-m/nofp\libg.a(lib_a-mlock.o)
 .data          0x00000000        0x0 c:/nxp/mcuxpressoide_11.1.0_3209/ide/plugins/com.nxp.mcuxpresso.tools.win32_11.1.0.201909161352/tools/bin/../lib/gcc/arm-none-eabi/8.3.1/../../../../arm-none-eabi/lib/thumb/v7e-m/nofp\libg.a(lib_a-mlock.o)
 .bss           0x00000000        0x0 c:/nxp/mcuxpressoide_11.1.0_3209/ide/plugins/com.nxp.mcuxpresso.tools.win32_11.1.0.201909161352/tools/bin/../lib/gcc/arm-none-eabi/8.3.1/../../../../arm-none-eabi/lib/thumb/v7e-m/nofp\libg.a(lib_a-mlock.o)
 .text.__malloc_lock
                0x00000000        0xc c:/nxp/mcuxpressoide_11.1.0_3209/ide/plugins/com.nxp.mcuxpresso.tools.win32_11.1.0.201909161352/tools/bin/../lib/gcc/arm-none-eabi/8.3.1/../../../../arm-none-eabi/lib/thumb/v7e-m/nofp\libg.a(lib_a-mlock.o)
 .text.__malloc_unlock
                0x00000000        0xc c:/nxp/mcuxpressoide_11.1.0_3209/ide/plugins/com.nxp.mcuxpresso.tools.win32_11.1.0.201909161352/tools/bin/../lib/gcc/arm-none-eabi/8.3.1/../../../../arm-none-eabi/lib/thumb/v7e-m/nofp\libg.a(lib_a-mlock.o)
 .debug_frame   0x00000000       0x30 c:/nxp/mcuxpressoide_11.1.0_3209/ide/plugins/com.nxp.mcuxpresso.tools.win32_11.1.0.201909161352/tools/bin/../lib/gcc/arm-none-eabi/8.3.1/../../../../arm-none-eabi/lib/thumb/v7e-m/nofp\libg.a(lib_a-mlock.o)
 .ARM.attributes
                0x00000000       0x2e c:/nxp/mcuxpressoide_11.1.0_3209/ide/plugins/com.nxp.mcuxpresso.tools.win32_11.1.0.201909161352/tools/bin/../lib/gcc/arm-none-eabi/8.3.1/../../../../arm-none-eabi/lib/thumb/v7e-m/nofp\libg.a(lib_a-mlock.o)
 .text          0x00000000        0x0 c:/nxp/mcuxpressoide_11.1.0_3209/ide/plugins/com.nxp.mcuxpresso.tools.win32_11.1.0.201909161352/tools/bin/../lib/gcc/arm-none-eabi/8.3.1/../../../../arm-none-eabi/lib/thumb/v7e-m/nofp\libg.a(lib_a-sbrkr.o)
 .data          0x00000000        0x0 c:/nxp/mcuxpressoide_11.1.0_3209/ide/plugins/com.nxp.mcuxpresso.tools.win32_11.1.0.201909161352/tools/bin/../lib/gcc/arm-none-eabi/8.3.1/../../../../arm-none-eabi/lib/thumb/v7e-m/nofp\libg.a(lib_a-sbrkr.o)
 .bss           0x00000000        0x0 c:/nxp/mcuxpressoide_11.1.0_3209/ide/plugins/com.nxp.mcuxpresso.tools.win32_11.1.0.201909161352/tools/bin/../lib/gcc/arm-none-eabi/8.3.1/../../../../arm-none-eabi/lib/thumb/v7e-m/nofp\libg.a(lib_a-sbrkr.o)
 .text._sbrk_r  0x00000000       0x24 c:/nxp/mcuxpressoide_11.1.0_3209/ide/plugins/com.nxp.mcuxpresso.tools.win32_11.1.0.201909161352/tools/bin/../lib/gcc/arm-none-eabi/8.3.1/../../../../arm-none-eabi/lib/thumb/v7e-m/nofp\libg.a(lib_a-sbrkr.o)
 .debug_frame   0x00000000       0x2c c:/nxp/mcuxpressoide_11.1.0_3209/ide/plugins/com.nxp.mcuxpresso.tools.win32_11.1.0.201909161352/tools/bin/../lib/gcc/arm-none-eabi/8.3.1/../../../../arm-none-eabi/lib/thumb/v7e-m/nofp\libg.a(lib_a-sbrkr.o)
 .ARM.attributes
                0x00000000       0x2e c:/nxp/mcuxpressoide_11.1.0_3209/ide/plugins/com.nxp.mcuxpresso.tools.win32_11.1.0.201909161352/tools/bin/../lib/gcc/arm-none-eabi/8.3.1/../../../../arm-none-eabi/lib/thumb/v7e-m/nofp\libg.a(lib_a-sbrkr.o)
 .data          0x00000000        0x0 c:/nxp/mcuxpressoide_11.1.0_3209/ide/plugins/com.nxp.mcuxpresso.tools.win32_11.1.0.201909161352/tools/bin/../lib/gcc/arm-none-eabi/8.3.1/../../../../arm-none-eabi/lib/thumb/v7e-m/nofp\libg.a(lib_a-strlen.o)
 .bss           0x00000000        0x0 c:/nxp/mcuxpressoide_11.1.0_3209/ide/plugins/com.nxp.mcuxpresso.tools.win32_11.1.0.201909161352/tools/bin/../lib/gcc/arm-none-eabi/8.3.1/../../../../arm-none-eabi/lib/thumb/v7e-m/nofp\libg.a(lib_a-strlen.o)
 .text          0x00000000        0x0 c:/nxp/mcuxpressoide_11.1.0_3209/ide/plugins/com.nxp.mcuxpresso.tools.win32_11.1.0.201909161352/tools/bin/../lib/gcc/arm-none-eabi/8.3.1/../../../../arm-none-eabi/lib/thumb/v7e-m/nofp\libg.a(lib_a-freer.o)
 .data          0x00000000        0x0 c:/nxp/mcuxpressoide_11.1.0_3209/ide/plugins/com.nxp.mcuxpresso.tools.win32_11.1.0.201909161352/tools/bin/../lib/gcc/arm-none-eabi/8.3.1/../../../../arm-none-eabi/lib/thumb/v7e-m/nofp\libg.a(lib_a-freer.o)
 .bss           0x00000000        0x0 c:/nxp/mcuxpressoide_11.1.0_3209/ide/plugins/com.nxp.mcuxpresso.tools.win32_11.1.0.201909161352/tools/bin/../lib/gcc/arm-none-eabi/8.3.1/../../../../arm-none-eabi/lib/thumb/v7e-m/nofp\libg.a(lib_a-freer.o)
 .text._malloc_trim_r
                0x00000000       0xa0 c:/nxp/mcuxpressoide_11.1.0_3209/ide/plugins/com.nxp.mcuxpresso.tools.win32_11.1.0.201909161352/tools/bin/../lib/gcc/arm-none-eabi/8.3.1/../../../../arm-none-eabi/lib/thumb/v7e-m/nofp\libg.a(lib_a-freer.o)
 .text._free_r  0x00000000      0x1f4 c:/nxp/mcuxpressoide_11.1.0_3209/ide/plugins/com.nxp.mcuxpresso.tools.win32_11.1.0.201909161352/tools/bin/../lib/gcc/arm-none-eabi/8.3.1/../../../../arm-none-eabi/lib/thumb/v7e-m/nofp\libg.a(lib_a-freer.o)
 .debug_frame   0x00000000       0x8c c:/nxp/mcuxpressoide_11.1.0_3209/ide/plugins/com.nxp.mcuxpresso.tools.win32_11.1.0.201909161352/tools/bin/../lib/gcc/arm-none-eabi/8.3.1/../../../../arm-none-eabi/lib/thumb/v7e-m/nofp\libg.a(lib_a-freer.o)
 .ARM.attributes
                0x00000000       0x2e c:/nxp/mcuxpressoide_11.1.0_3209/ide/plugins/com.nxp.mcuxpresso.tools.win32_11.1.0.201909161352/tools/bin/../lib/gcc/arm-none-eabi/8.3.1/../../../../arm-none-eabi/lib/thumb/v7e-m/nofp\libg.a(lib_a-freer.o)
 .text          0x00000000        0x0 c:/nxp/mcuxpressoide_11.1.0_3209/ide/plugins/com.nxp.mcuxpresso.tools.win32_11.1.0.201909161352/tools/bin/../lib/gcc/arm-none-eabi/8.3.1/../../../../arm-none-eabi/lib/thumb/v7e-m/nofp\libg.a(lib_a-impure.o)
 .data          0x00000000        0x0 c:/nxp/mcuxpressoide_11.1.0_3209/ide/plugins/com.nxp.mcuxpresso.tools.win32_11.1.0.201909161352/tools/bin/../lib/gcc/arm-none-eabi/8.3.1/../../../../arm-none-eabi/lib/thumb/v7e-m/nofp\libg.a(lib_a-impure.o)
 .bss           0x00000000        0x0 c:/nxp/mcuxpressoide_11.1.0_3209/ide/plugins/com.nxp.mcuxpresso.tools.win32_11.1.0.201909161352/tools/bin/../lib/gcc/arm-none-eabi/8.3.1/../../../../arm-none-eabi/lib/thumb/v7e-m/nofp\libg.a(lib_a-impure.o)
 .data._impure_ptr
                0x00000000        0x4 c:/nxp/mcuxpressoide_11.1.0_3209/ide/plugins/com.nxp.mcuxpresso.tools.win32_11.1.0.201909161352/tools/bin/../lib/gcc/arm-none-eabi/8.3.1/../../../../arm-none-eabi/lib/thumb/v7e-m/nofp\libg.a(lib_a-impure.o)
 .data.impure_data
                0x00000000      0x428 c:/nxp/mcuxpressoide_11.1.0_3209/ide/plugins/com.nxp.mcuxpresso.tools.win32_11.1.0.201909161352/tools/bin/../lib/gcc/arm-none-eabi/8.3.1/../../../../arm-none-eabi/lib/thumb/v7e-m/nofp\libg.a(lib_a-impure.o)
 .rodata._global_impure_ptr
                0x00000000        0x4 c:/nxp/mcuxpressoide_11.1.0_3209/ide/plugins/com.nxp.mcuxpresso.tools.win32_11.1.0.201909161352/tools/bin/../lib/gcc/arm-none-eabi/8.3.1/../../../../arm-none-eabi/lib/thumb/v7e-m/nofp\libg.a(lib_a-impure.o)
 .ARM.attributes
                0x00000000       0x2e c:/nxp/mcuxpressoide_11.1.0_3209/ide/plugins/com.nxp.mcuxpresso.tools.win32_11.1.0.201909161352/tools/bin/../lib/gcc/arm-none-eabi/8.3.1/../../../../arm-none-eabi/lib/thumb/v7e-m/nofp\libg.a(lib_a-impure.o)
 .text          0x00000000        0x0 c:/nxp/mcuxpressoide_11.1.0_3209/ide/plugins/com.nxp.mcuxpresso.tools.win32_11.1.0.201909161352/tools/bin/../lib/gcc/arm-none-eabi/8.3.1/../../../../arm-none-eabi/lib/thumb/v7e-m/nofp\libg.a(lib_a-lock.o)
 .data          0x00000000        0x0 c:/nxp/mcuxpressoide_11.1.0_3209/ide/plugins/com.nxp.mcuxpresso.tools.win32_11.1.0.201909161352/tools/bin/../lib/gcc/arm-none-eabi/8.3.1/../../../../arm-none-eabi/lib/thumb/v7e-m/nofp\libg.a(lib_a-lock.o)
 .bss           0x00000000        0x0 c:/nxp/mcuxpressoide_11.1.0_3209/ide/plugins/com.nxp.mcuxpresso.tools.win32_11.1.0.201909161352/tools/bin/../lib/gcc/arm-none-eabi/8.3.1/../../../../arm-none-eabi/lib/thumb/v7e-m/nofp\libg.a(lib_a-lock.o)
 .text.__retarget_lock_init
                0x00000000        0x4 c:/nxp/mcuxpressoide_11.1.0_3209/ide/plugins/com.nxp.mcuxpresso.tools.win32_11.1.0.201909161352/tools/bin/../lib/gcc/arm-none-eabi/8.3.1/../../../../arm-none-eabi/lib/thumb/v7e-m/nofp\libg.a(lib_a-lock.o)
 .text.__retarget_lock_init_recursive
                0x00000000        0x4 c:/nxp/mcuxpressoide_11.1.0_3209/ide/plugins/com.nxp.mcuxpresso.tools.win32_11.1.0.201909161352/tools/bin/../lib/gcc/arm-none-eabi/8.3.1/../../../../arm-none-eabi/lib/thumb/v7e-m/nofp\libg.a(lib_a-lock.o)
 .text.__retarget_lock_close
                0x00000000        0x4 c:/nxp/mcuxpressoide_11.1.0_3209/ide/plugins/com.nxp.mcuxpresso.tools.win32_11.1.0.201909161352/tools/bin/../lib/gcc/arm-none-eabi/8.3.1/../../../../arm-none-eabi/lib/thumb/v7e-m/nofp\libg.a(lib_a-lock.o)
 .text.__retarget_lock_close_recursive
                0x00000000        0x4 c:/nxp/mcuxpressoide_11.1.0_3209/ide/plugins/com.nxp.mcuxpresso.tools.win32_11.1.0.201909161352/tools/bin/../lib/gcc/arm-none-eabi/8.3.1/../../../../arm-none-eabi/lib/thumb/v7e-m/nofp\libg.a(lib_a-lock.o)
 .text.__retarget_lock_acquire
                0x00000000        0x4 c:/nxp/mcuxpressoide_11.1.0_3209/ide/plugins/com.nxp.mcuxpresso.tools.win32_11.1.0.201909161352/tools/bin/../lib/gcc/arm-none-eabi/8.3.1/../../../../arm-none-eabi/lib/thumb/v7e-m/nofp\libg.a(lib_a-lock.o)
 .text.__retarget_lock_acquire_recursive
                0x00000000        0x4 c:/nxp/mcuxpressoide_11.1.0_3209/ide/plugins/com.nxp.mcuxpresso.tools.win32_11.1.0.201909161352/tools/bin/../lib/gcc/arm-none-eabi/8.3.1/../../../../arm-none-eabi/lib/thumb/v7e-m/nofp\libg.a(lib_a-lock.o)
 .text.__retarget_lock_try_acquire
                0x00000000        0x4 c:/nxp/mcuxpressoide_11.1.0_3209/ide/plugins/com.nxp.mcuxpresso.tools.win32_11.1.0.201909161352/tools/bin/../lib/gcc/arm-none-eabi/8.3.1/../../../../arm-none-eabi/lib/thumb/v7e-m/nofp\libg.a(lib_a-lock.o)
 .text.__retarget_lock_try_acquire_recursive
                0x00000000        0x4 c:/nxp/mcuxpressoide_11.1.0_3209/ide/plugins/com.nxp.mcuxpresso.tools.win32_11.1.0.201909161352/tools/bin/../lib/gcc/arm-none-eabi/8.3.1/../../../../arm-none-eabi/lib/thumb/v7e-m/nofp\libg.a(lib_a-lock.o)
 .text.__retarget_lock_release
                0x00000000        0x4 c:/nxp/mcuxpressoide_11.1.0_3209/ide/plugins/com.nxp.mcuxpresso.tools.win32_11.1.0.201909161352/tools/bin/../lib/gcc/arm-none-eabi/8.3.1/../../../../arm-none-eabi/lib/thumb/v7e-m/nofp\libg.a(lib_a-lock.o)
 .text.__retarget_lock_release_recursive
                0x00000000        0x4 c:/nxp/mcuxpressoide_11.1.0_3209/ide/plugins/com.nxp.mcuxpresso.tools.win32_11.1.0.201909161352/tools/bin/../lib/gcc/arm-none-eabi/8.3.1/../../../../arm-none-eabi/lib/thumb/v7e-m/nofp\libg.a(lib_a-lock.o)
 .debug_frame   0x00000000       0xb0 c:/nxp/mcuxpressoide_11.1.0_3209/ide/plugins/com.nxp.mcuxpresso.tools.win32_11.1.0.201909161352/tools/bin/../lib/gcc/arm-none-eabi/8.3.1/../../../../arm-none-eabi/lib/thumb/v7e-m/nofp\libg.a(lib_a-lock.o)
 .ARM.attributes
                0x00000000       0x2e c:/nxp/mcuxpressoide_11.1.0_3209/ide/plugins/com.nxp.mcuxpresso.tools.win32_11.1.0.201909161352/tools/bin/../lib/gcc/arm-none-eabi/8.3.1/../../../../arm-none-eabi/lib/thumb/v7e-m/nofp\libg.a(lib_a-lock.o)
 COMMON         0x00000000       0x21 c:/nxp/mcuxpressoide_11.1.0_3209/ide/plugins/com.nxp.mcuxpresso.tools.win32_11.1.0.201909161352/tools/bin/../lib/gcc/arm-none-eabi/8.3.1/../../../../arm-none-eabi/lib/thumb/v7e-m/nofp\libg.a(lib_a-lock.o)
 .text          0x00000000        0x0 c:/nxp/mcuxpressoide_11.1.0_3209/ide/plugins/com.nxp.mcuxpresso.tools.win32_11.1.0.201909161352/tools/bin/../lib/gcc/arm-none-eabi/8.3.1/../../../../arm-none-eabi/lib/thumb/v7e-m/nofp\libg.a(lib_a-reent.o)
 .data          0x00000000        0x0 c:/nxp/mcuxpressoide_11.1.0_3209/ide/plugins/com.nxp.mcuxpresso.tools.win32_11.1.0.201909161352/tools/bin/../lib/gcc/arm-none-eabi/8.3.1/../../../../arm-none-eabi/lib/thumb/v7e-m/nofp\libg.a(lib_a-reent.o)
 .bss           0x00000000        0x0 c:/nxp/mcuxpressoide_11.1.0_3209/ide/plugins/com.nxp.mcuxpresso.tools.win32_11.1.0.201909161352/tools/bin/../lib/gcc/arm-none-eabi/8.3.1/../../../../arm-none-eabi/lib/thumb/v7e-m/nofp\libg.a(lib_a-reent.o)
 .text.cleanup_glue
                0x00000000       0x1c c:/nxp/mcuxpressoide_11.1.0_3209/ide/plugins/com.nxp.mcuxpresso.tools.win32_11.1.0.201909161352/tools/bin/../lib/gcc/arm-none-eabi/8.3.1/../../../../arm-none-eabi/lib/thumb/v7e-m/nofp\libg.a(lib_a-reent.o)
 .text._reclaim_reent
                0x00000000       0x88 c:/nxp/mcuxpressoide_11.1.0_3209/ide/plugins/com.nxp.mcuxpresso.tools.win32_11.1.0.201909161352/tools/bin/../lib/gcc/arm-none-eabi/8.3.1/../../../../arm-none-eabi/lib/thumb/v7e-m/nofp\libg.a(lib_a-reent.o)
 .debug_frame   0x00000000       0x60 c:/nxp/mcuxpressoide_11.1.0_3209/ide/plugins/com.nxp.mcuxpresso.tools.win32_11.1.0.201909161352/tools/bin/../lib/gcc/arm-none-eabi/8.3.1/../../../../arm-none-eabi/lib/thumb/v7e-m/nofp\libg.a(lib_a-reent.o)
 .ARM.attributes
                0x00000000       0x2e c:/nxp/mcuxpressoide_11.1.0_3209/ide/plugins/com.nxp.mcuxpresso.tools.win32_11.1.0.201909161352/tools/bin/../lib/gcc/arm-none-eabi/8.3.1/../../../../arm-none-eabi/lib/thumb/v7e-m/nofp\libg.a(lib_a-reent.o)
 COMMON         0x00000000        0x4 c:/nxp/mcuxpressoide_11.1.0_3209/ide/plugins/com.nxp.mcuxpresso.tools.win32_11.1.0.201909161352/tools/bin/../lib/gcc/arm-none-eabi/8.3.1/../../../../arm-none-eabi/lib/thumb/v7e-m/nofp\libg.a(lib_a-reent.o)

Memory Configuration

Name             Origin             Length             Attributes
Flash640         0x00000000         0x000a0000         xr
RAM0             0x04000400         0x00015c00         xrw
RAM1             0x04020000         0x00010000         xrw
*default*        0x00000000         0xffffffff

Linker script and memory map

LOAD ./utilities/MicroInt_arm_sdk2.o
LOAD ./utilities/Panic.o
LOAD ./utilities/fsl_assert.o
LOAD ./utilities/fsl_debug_console.o
LOAD ./utilities/serial_manager.o
LOAD ./utilities/serial_port_uart.o
LOAD ./utilities/usart_adapter.o
LOAD ./startup/startup_K32W061.o
LOAD ./startup/system_K32W061.o
LOAD ./source/tis_trp_dut.o
LOAD ./drivers/fsl_clock.o
LOAD ./drivers/fsl_common.o
LOAD ./drivers/fsl_ctimer.o
LOAD ./drivers/fsl_flexcomm.o
LOAD ./drivers/fsl_gpio.o
LOAD ./drivers/fsl_inputmux.o
LOAD ./drivers/fsl_power.o
LOAD ./drivers/fsl_reset.o
LOAD ./drivers/fsl_str.o
LOAD ./drivers/fsl_usart.o
LOAD ./drivers/fsl_wtimer.o
LOAD ./board/board.o
LOAD ./board/clock_config.o
LOAD ./board/hardware_init.o
LOAD ./board/pin_mux.o
LOAD ./Common/CRC.o
LOAD ./Common/Command.o
LOAD C:/nxp/SDKPackages/SDK_2.6.0_K32W061DK6/middleware/wireless/ieee-802.15.4/lib\libMiniMac.a
LOAD C:/nxp/SDKPackages/SDK_2.6.0_K32W061DK6/middleware/wireless/framework/XCVR/lib\libRadio_Test_JN518x.a
LOAD C:/nxp/SDKPackages/SDK_2.6.0_K32W061DK6/middleware/wireless/framework/XCVR/lib\libRadio.a
START GROUP
LOAD c:/nxp/mcuxpressoide_11.1.0_3209/ide/plugins/com.nxp.mcuxpresso.tools.win32_11.1.0.201909161352/tools/bin/../lib/gcc/arm-none-eabi/8.3.1/thumb/v7e-m/nofp\libgcc.a
LOAD c:/nxp/mcuxpressoide_11.1.0_3209/ide/plugins/com.nxp.mcuxpresso.tools.win32_11.1.0.201909161352/tools/bin/../lib/gcc/arm-none-eabi/8.3.1/../../../../arm-none-eabi/lib/thumb/v7e-m/nofp\libg.a
LOAD c:/nxp/mcuxpressoide_11.1.0_3209/ide/plugins/com.nxp.mcuxpresso.tools.win32_11.1.0.201909161352/tools/bin/../lib/gcc/arm-none-eabi/8.3.1/../../../../arm-none-eabi/lib/thumb/v7e-m/nofp\libc.a
END GROUP
                [!provide]                PROVIDE (aesInit = 0x3001161)
                [!provide]                PROVIDE (aesWriteByte = 0x3001175)
                [!provide]                PROVIDE (aesWrite = 0x300118d)
                [!provide]                PROVIDE (aesRead = 0x30011a5)
                [!provide]                PROVIDE (aesWriteBlock = 0x30011c1)
                [!provide]                PROVIDE (aesReadBlock = 0x30011e9)
                [!provide]                PROVIDE (aesMode = 0x3001211)
                [!provide]                PROVIDE (aesAbort = 0x3001269)
                [!provide]                PROVIDE (aesLoadCounter = 0x3001291)
                [!provide]                PROVIDE (aesLoadKeyFromSW = 0x30012a9)
                [!provide]                PROVIDE (aesLoadIV = 0x30012fd)
                [!provide]                PROVIDE (aesProcess = 0x30013d1)
                [!provide]                PROVIDE (aesWriteYInputGf128 = 0x300132d)
                [!provide]                PROVIDE (aesReadGf128Hash = 0x300135d)
                [!provide]                PROVIDE (aesReadGcmTag = 0x300138d)
                [!provide]                PROVIDE (aesGetDriverVersion = 0x30013bd)
                [!provide]                PROVIDE (aesIsSupported = 0x300115d)
                [!provide]                PROVIDE (BOOT_CPU_Slave_Boot = 0x3000489)
                [!provide]                PROVIDE (BOOT_CPU_Slave_Disable = 0x30004f1)
                [!provide]                PROVIDE (BOOT_RemapAddress = 0x3000dc9)
                [!provide]                PROVIDE (boot_Verify_eScoreImageList = 0x30003e5)
                [!provide]                PROVIDE (BOOT_FindImage = 0x3000519)
                [!provide]                PROVIDE (BOOT_GetStartPowerMode = 0x3000e9d)
                [!provide]                PROVIDE (BOOT_SetResumeStackPointer = 0x3000ea9)
                [!provide]                PROVIDE (ROM_GetFlash = 0x3000e0d)
                [!provide]                PROVIDE (ROM_GetSRAM0 = 0x3000e21)
                [!provide]                PROVIDE (ROM_GetSRAM1 = 0x3000e35)
                [!provide]                PROVIDE (psector_Read_HwTestModeDisable = 0x30054d1)
                [!provide]                PROVIDE (psector_Read_ISP_AccessLevel = 0x30054f5)
                [!provide]                PROVIDE (flashConfig_ExtractTempSensorTrimValues = 0x3001fbd)
                [!provide]                PROVIDE (flashConfig_ExtractRfpModemTrimValues = 0x3002065)
                [!provide]                PROVIDE (flashConfig_ExtractUlpbgTrimValues = 0x30020a5)
                [!provide]                PROVIDE (flashConfig_ExtractFro1MTrimValues = 0x30020fd)
                [!provide]                PROVIDE (flashConfig_ExtractGpAdcTrimValues = 0x3002131)
                [!provide]                PROVIDE (flashConfig_ExtractFRO32kTrimValues = 0x3002189)
                [!provide]                PROVIDE (flashConfig_ExtractDcDcTrimValues = 0x30021bd)
                [!provide]                PROVIDE (efuse_ReadBit = 0x3001671)
                [!provide]                PROVIDE (ISP_Entry = 0x3002fb1)
                [!provide]                PROVIDE (MPU_pSectorGrantAccessRights = 0x30017e5)
                [!provide]                PROVIDE (MPU_pSectorWithdrawAccessRights = 0x3001841)
                [!provide]                PROVIDE (MPU_GetCurrentSettings = 0x300178d)
                [!provide]                PROVIDE (MPU_SetRegionAccessRights = 0x3001821)
                [!provide]                PROVIDE (MPU_ClearRegionSetting = 0x300184d)
                [!provide]                PROVIDE (MPU_AllocateRegionDesc = 0x30017c1)
                [!provide]                PROVIDE (nxHal_Patch_Init = 0x300473d)
                [!provide]                PROVIDE (nxHal_Patch_SetSVCHandler = 0x30047bd)
                [!provide]                PROVIDE (nxHal_Patch_Apply = 0x3004839)
                [!provide]                PROVIDE (nxHal_Patch_EnableDisable = 0x30047c9)
                [!provide]                PROVIDE (nxHal_Patch_GetGlobalPatchMarkerIndex = 0x3004821)
                [!provide]                PROVIDE (nxHal_Patch_ReadPatchEntry = 0x300482d)
                [!provide]                PROVIDE (nxHal_Patch_LoadDynamicPatches = 0x300488d)
                [!provide]                PROVIDE (eSCORE_PatchTestFunction1 = 0x3004919)
                [!provide]                PROVIDE (eSCORE_PatchTestFunction2 = 0x300492d)
                [!provide]                PROVIDE (eSCORE_PatchTestFunction3 = 0x3004941)
                [!provide]                PROVIDE (pmc_reset_get_cause = 0x30046e9)
                [!provide]                PROVIDE (pmc_reset_clear_cause = 0x30046f5)
                [!provide]                PROVIDE (psector_WriteUpdatePage = 0x3004e11)
                [!provide]                PROVIDE (psector_EraseUpdate = 0x3004d59)
                [!provide]                PROVIDE (psector_Read_CustomerId = 0x30051dd)
                [!provide]                PROVIDE (psector_Read_RomPatchInfo = 0x3005209)
                [!provide]                PROVIDE (psector_Read_ImgAuthLevel = 0x3005299)
                [!provide]                PROVIDE (psector_Read_AppSearchGranularity = 0x30052d5)
                [!provide]                PROVIDE (psector_Read_QspiAppSearchGranularity = 0x3005305)
                [!provide]                PROVIDE (psector_Read_UnlockKey = 0x3005519)
                [!provide]                PROVIDE (psector_Read_DeviceId = 0x3005329)
                [!provide]                PROVIDE (psector_Read_ISP_protocol_key = 0x3005355)
                [!provide]                PROVIDE (psector_ReadIeee802_15_4_MacId2 = 0x3005385)
                [!provide]                PROVIDE (psector_ReadIeee802_15_4_MacId1 = 0x30053b1)
                [!provide]                PROVIDE (psector_Read_MinDeviceId = 0x30053dd)
                [!provide]                PROVIDE (psector_Read_MaxDeviceId = 0x3005409)
                [!provide]                PROVIDE (psector_Read_MinVersion = 0x3005439)
                [!provide]                PROVIDE (psector_SetEscoreImageData = 0x300545d)
                [!provide]                PROVIDE (psector_ReadEscoreImageData = 0x3005491)
                [!provide]                PROVIDE (psector_Read_ImagePubKey = 0x3005531)
                [!provide]                PROVIDE (psector_ReadData = 0x3004ef1)
                [!provide]                PROVIDE (psector_CalculateChecksum = 0x30050bd)
                [!provide]                PROVIDE (secure_VerifySignature = 0x3005c65)
                [!provide]                PROVIDE (secure_VerifyBlock = 0x3005cad)
                [!provide]                PROVIDE (secure_VerifyCertificate = 0x3005cd1)
                [!provide]                PROVIDE (secure_VerifyImage = 0x3005d59)
                [!provide]                PROVIDE (NMI_Handler = 0x300012d)
                [!provide]                PROVIDE (HardFault_Handler = 0x3000131)
                [!provide]                PROVIDE (MemManage_Handler = 0x3000135)
                [!provide]                PROVIDE (BusFault_Handler = 0x3000e81)
                [!provide]                PROVIDE (UsageFault_Handler = 0x300013d)
                [!provide]                PROVIDE (SVC_Handler = 0x3005e85)
                [!provide]                PROVIDE (DebugMon_Handler = 0x3000145)
                [!provide]                PROVIDE (PendSV_Handler = 0x3000149)
                [!provide]                PROVIDE (SysTick_Handler = 0x300014d)
                [!provide]                PROVIDE (IntDefaultHandler = 0x3000151)
                [!provide]                PROVIDE (System_IRQHandler = 0x3000151)
                [!provide]                PROVIDE (DMA_IRQHandler = 0x3000151)
                [!provide]                PROVIDE (GINT_IRQHandler = 0x3000151)
                [!provide]                PROVIDE (IRBlaster_IRQHandler = 0x3000151)
                [!provide]                PROVIDE (PINT0_IRQHandler = 0x3000151)
                [!provide]                PROVIDE (PINT1_IRQHandler = 0x3000151)
                [!provide]                PROVIDE (PINT2_IRQHandler = 0x3000151)
                [!provide]                PROVIDE (PINT3_IRQHandler = 0x3000151)
                [!provide]                PROVIDE (SPIFI_IRQHandler = 0x3000151)
                [!provide]                PROVIDE (Timer0_IRQHandler = 0x3000151)
                [!provide]                PROVIDE (Timer1_IRQHandler = 0x3000151)
                [!provide]                PROVIDE (USART0_IRQHandler = 0x3000151)
                [!provide]                PROVIDE (USART1_IRQHandler = 0x3000151)
                [!provide]                PROVIDE (I2C0_IRQHandler = 0x3000151)
                [!provide]                PROVIDE (I2C1_IRQHandler = 0x3000151)
                [!provide]                PROVIDE (SPI0_IRQHandler = 0x3000151)
                [!provide]                PROVIDE (SPI1_IRQHandler = 0x3000151)
                [!provide]                PROVIDE (PWM0_IRQHandler = 0x3000151)
                [!provide]                PROVIDE (PWM1_IRQHandler = 0x3000151)
                [!provide]                PROVIDE (PWM2_IRQHandler = 0x3000151)
                [!provide]                PROVIDE (PWM3_IRQHandler = 0x3000151)
                [!provide]                PROVIDE (PWM4_IRQHandler = 0x3000151)
                [!provide]                PROVIDE (PWM5_IRQHandler = 0x3000151)
                [!provide]                PROVIDE (PWM6_IRQHandler = 0x3000151)
                [!provide]                PROVIDE (PWM7_IRQHandler = 0x3000151)
                [!provide]                PROVIDE (PWM8_IRQHandler = 0x3000151)
                [!provide]                PROVIDE (PWM9_IRQHandler = 0x3000151)
                [!provide]                PROVIDE (PWM10_IRQHandler = 0x3000151)
                [!provide]                PROVIDE (I2C2_IRQHandler = 0x3000151)
                [!provide]                PROVIDE (RTC_IRQHandler = 0x3000151)
                [!provide]                PROVIDE (NFCTag_IRQHandler = 0x3000151)
                [!provide]                PROVIDE (MAILBOX_IRQHandler = 0x3000151)
                [!provide]                PROVIDE (ADC_SEQA_IRQHandler = 0x3000151)
                [!provide]                PROVIDE (ADC_SEQB_IRQHandler = 0x3000151)
                [!provide]                PROVIDE (ADC_THCMP_OVR_IRQHandler = 0x3000151)
                [!provide]                PROVIDE (DMIC_IRQHandler = 0x3000151)
                [!provide]                PROVIDE (HWVAD_IRQHandler = 0x3000151)
                [!provide]                PROVIDE (BLE_DP_IRQHandler = 0x3000151)
                [!provide]                PROVIDE (BLE_DP0_IRQHandler = 0x3000151)
                [!provide]                PROVIDE (BLE_DP1_IRQHandler = 0x3000151)
                [!provide]                PROVIDE (BLE_DP2_IRQHandler = 0x3000151)
                [!provide]                PROVIDE (BLE_LL_ALL_IRQHandler = 0x3000151)
                [!provide]                PROVIDE (ZIGBEE_MAC_IRQHandler = 0x3006b65)
                [!provide]                PROVIDE (ZIGBEE_MODEM_IRQHandler = 0x3000151)
                [!provide]                PROVIDE (RFP_TMU_IRQHandler = 0x3000151)
                [!provide]                PROVIDE (RFP_AGC_IRQHandler = 0x3000151)
                [!provide]                PROVIDE (ISO7816_IRQHandler = 0x3000151)
                [!provide]                PROVIDE (ANA_COMP_IRQHandler = 0x3000151)
                [!provide]                PROVIDE (WAKE_UP_TIMER0_IRQHandler = 0x3000151)
                [!provide]                PROVIDE (WAKE_UP_TIMER1_IRQHandler = 0x3000151)
                [!provide]                PROVIDE (PVT_AMBER0_IRQHandler = 0x3000151)
                [!provide]                PROVIDE (PVT_RED0_IRQHandler = 0x3000151)
                [!provide]                PROVIDE (PVT_AMBER1_IRQHandler = 0x3000151)
                [!provide]                PROVIDE (PVT_RED1_IRQHandler = 0x3000151)
                [!provide]                PROVIDE (Chip_LOWPOWER_SetUpLowPowerModeWakeUpTimer = 0x30038d1)
                [!provide]                PROVIDE (Chip_LOWPOWER_SetSystemFrequency = 0x3003d55)
                [!provide]                PROVIDE (Chip_LOWPOWER_SetMemoryLowPowerMode = 0x3003d89)
                [!provide]                PROVIDE (Chip_LOWPOWER_GetSystemVoltages = 0x3003de1)
                [!provide]                PROVIDE (Chip_LOWPOWER_SetSystemVoltages = 0x3003e99)
                [!provide]                PROVIDE (Chip_LOWPOWER_SetLowPowerMode = 0x300404d)
                [!provide]                PROVIDE (Chip_LOWPOWER_ChipSoftwareReset = 0x3003fa1)
                [!provide]                PROVIDE (Chip_LOWPOWER_ArmSoftwareReset = 0x300400d)
                0x00000400                BOOT_RESUME_STACK_SIZE = 0x400
                0x00000fe0                STACK_SIZE = 0xfe0
                0x00000000                FLASH_BASE_DEFAULT = 0x0
                0x000a0000                FLASH_SIZE_DEFAULT = 0xa0000
                0x04000400                RAM0_BASE_DEFAULT = 0x4000400
                0x00015c00                RAM0_SIZE_DEFAULT = 0x15c00
                0x00004000                FLASH_SIZE_SSBL = 0x4000
                0x0004f000                FLASH_SIZE_ZIGBEE_STACK = 0x4f000
                0x00040000                FLASH_SIZE_BLE_STACK = 0x40000
                0x00000000                FLASH_BASE_SSBL = FLASH_BASE_DEFAULT
                0x00004000                FLASH_BASE_ZIGBEE_STACK = (FLASH_BASE_SSBL + FLASH_SIZE_SSBL)
                0x00053000                FLASH_BASE_BLE_STACK = (FLASH_BASE_ZIGBEE_STACK + FLASH_SIZE_ZIGBEE_STACK)
                0x00000000                MEM_FLASH_BASE = DEFINED (MEM_FLASH_BASE)?MEM_FLASH_BASE:DEFINED (BUILD_SSBL)?FLASH_BASE_SSBL:DEFINED (BUILD_ZIGBEE_STACK)?FLASH_BASE_ZIGBEE_STACK:DEFINED (BUILD_BLE_STACK)?FLASH_BASE_BLE_STACK:FLASH_BASE_DEFAULT
                0x000a0000                MEM_FLASH_SIZE = DEFINED (MEM_FLASH_SIZE)?MEM_FLASH_SIZE:DEFINED (BUILD_SSBL)?FLASH_SIZE_SSBL:DEFINED (BUILD_ZIGBEE_STACK)?FLASH_SIZE_ZIGBEE_STACK:DEFINED (BUILD_BLE_STACK)?FLASH_SIZE_BLE_STACK:FLASH_SIZE_DEFAULT
                0x04000400                MEM_RAM0_BASE = DEFINED (MEM_RAM0_BASE)?MEM_RAM0_BASE:RAM0_BASE_DEFAULT
                0x00015c00                MEM_RAM0_SIZE = DEFINED (MEM_RAM0_SIZE)?MEM_RAM0_SIZE:RAM0_SIZE_DEFAULT
                0x00000000                __base_Flash640 = MEM_FLASH_BASE
                0x00000000                __base_Flash = MEM_FLASH_BASE
                0x000a0000                __top_Flash640 = (MEM_FLASH_BASE + MEM_FLASH_SIZE)
                0x000a0000                __top_Flash = (MEM_FLASH_BASE + MEM_FLASH_SIZE)
                0x04000400                __base_RAM0 = MEM_RAM0_BASE
                0x04000400                __base_RAM = MEM_RAM0_BASE
                0x04016000                __top_RAM0 = (MEM_RAM0_BASE + MEM_RAM0_SIZE)
                0x04016000                __top_RAM = (MEM_RAM0_BASE + MEM_RAM0_SIZE)
                0x04020000                __base_RAM1 = 0x4020000
                0x04020000                __base_RAM2 = 0x4020000
                0x04030000                __top_RAM1 = 0x4030000
                0x04030000                __top_RAM2 = 0x4030000
                0x000002f4                HEAP_SIZE = DEFINED (HEAP_SIZE)?HEAP_SIZE:0x2f4
                0x00000000                m_flash_start = 0x0
                0x0009ffff                m_flash_end = 0x9ffff
                0x000a0000                m_flash_size = 0xa0000
                0x00000200                m_sector_size = 0x200
                0x00000200                m_fsl_prodInfo_size = m_sector_size
                0x0009ddff                m_fsl_prodInfo_end = ((m_flash_size - (0x11 * m_sector_size)) - 0x1)
                0x0009dc00                m_fsl_prodInfo_start = ((m_fsl_prodInfo_end - m_fsl_prodInfo_size) + 0x1)
                0x00007e00                NV_STORAGE_SIZE = (0x3f * m_sector_size)
                0x0009dbff                NV_STORAGE_START_ADDRESS = (m_fsl_prodInfo_start - 0x1)
                0x00095e00                NV_STORAGE_END_ADDRESS = ((NV_STORAGE_START_ADDRESS - NV_STORAGE_SIZE) + 0x1)
                0x00095dff                INT_STORAGE_START = (NV_STORAGE_END_ADDRESS - 0x1)
                0x00048000                INT_STORAGE_END = 0x48000
                0x0004ddff                INT_STORAGE_SIZE = (INT_STORAGE_START - INT_STORAGE_END)
                0x0009dc00                FREESCALE_PROD_DATA_BASE_ADDR = m_fsl_prodInfo_start
                0x00000200                INT_STORAGE_SECTOR_SIZE = m_sector_size
                0x00000000                M_VECTOR_RAM_SIZE = DEFINED (__ram_vector_table__)?vector_table_size:0x0

.header         0x00000000      0x150
                0x00000000                _flash_start = ABSOLUTE (.)
                0x00000000                _flash_beg = ABSOLUTE (.)
 FILL mask 0xff
                0x00000000                __vectors_start__ = ABSOLUTE (.)
                0x00000000                __VECTOR_TABLE = .
                0x00000000                __Vectors = .
 *(.isr_vector)
 .isr_vector    0x00000000      0x120 ./startup/startup_K32W061.o
                0x00000000                g_pfnVectors
                0x00000120                . = ALIGN (0x4)
                0x00000120                __section_table_start = .
                0x00000120                __data_section_table = .
                0x00000120        0x4 LONG 0x7594 LOADADDR (.data)
                0x00000124        0x4 LONG 0x4000400 ADDR (.data)
                0x00000128        0x4 LONG 0x84 SIZEOF (.data)
                0x0000012c        0x4 LONG 0x7594 LOADADDR (.data_RAM2)
                0x00000130        0x4 LONG 0x4020000 ADDR (.data_RAM2)
                0x00000134        0x4 LONG 0x0 SIZEOF (.data_RAM2)
                0x00000138                __data_section_table_end = .
                0x00000138                __bss_section_table = .
                0x00000138        0x4 LONG 0x4000484 ADDR (.bss)
                0x0000013c        0x4 LONG 0x1d4 SIZEOF (.bss)
                0x00000140        0x4 LONG 0x4020000 ADDR (.bss_RAM2)
                0x00000144        0x4 LONG 0x0 SIZEOF (.bss_RAM2)
                0x00000148                __bss_section_table_end = .
                0x00000148                __section_table_end = .
 FILL mask 0xff
                0x00000150                . = ALIGN (0x10)
 *fill*         0x00000148        0x8 ff

.ro_nonce       0x00000150        0x0
                0x00000150                _FlsNonceStart = ABSOLUTE (.)
 *(.ro_nonce)
 FILL mask 0xff
                0x00000150                . = ALIGN (0x10)

.ro_ota_header  0x00000150        0x0
                0x00000150                _enc_start = ABSOLUTE (.)
                0x00000150                _enc_offset = (_enc_start & 0xf)
                0x00000150                _FlsOtaHeader = ABSOLUTE (.)
 *(.ro_ota_header)
 FILL mask 0xff
                0x00000150                . = ALIGN (0x10)

.ro_se_lnkKey   0x00000150        0x0
                0x00000150                _FlsLinkKey = ABSOLUTE (.)
 *(.ro_se_lnkKey)
 FILL mask 0xff
                0x00000150                . = ALIGN (0x10)

.filler         0x00000150       0x30
                0x00000150        0x1 BYTE 0xff
 FILL mask 0xff
                0x00000180                . = ALIGN (0x40)
 *fill*         0x00000151       0x2f ff

.text           0x00000180     0x740c
 FILL mask 0xff
 *(.after_vectors*)
 .after_vectors.reset
                0x00000180       0x20 ./startup/startup_K32W061.o
                0x00000180                ResetISR
 .after_vectors
                0x000001a0      0x190 ./startup/startup_K32W061.o
                0x000001a0                SHA_IRQHandler
                0x000001a0                GINT0_DriverIRQHandler
                0x000001a0                PWM5_IRQHandler
                0x000001a0                DMA0_DriverIRQHandler
                0x000001a0                CIC_IRB_DriverIRQHandler
                0x000001a0                PVT_AMBER0_IRQHandler
                0x000001a0                PWM9_IRQHandler
                0x000001a0                BLE_DP1_IRQHandler
                0x000001a0                BLE_DP0_IRQHandler
                0x000001a0                PWM1_IRQHandler
                0x000001a0                PWM6_IRQHandler
                0x000001a0                BLE_WakeupTimer_IRQHandler
                0x000001a0                BLE_DP_IRQHandler
                0x000001a0                ADC_SEQB_IRQHandler
                0x000001a0                PWM8_IRQHandler
                0x000001a0                PIN_INT3_DriverIRQHandler
                0x000001a0                PIN_INT2_DriverIRQHandler
                0x000001a0                PWM3_IRQHandler
                0x000001a0                PIN_INT0_DriverIRQHandler
                0x000001a0                NFCTag_IRQHandler
                0x000001a0                BLE_LL_ALL_IRQHandler
                0x000001a0                PWM0_IRQHandler
                0x000001a0                IntDefaultHandler
                0x000001a0                ISO7816_IRQHandler
                0x000001a0                PVT_RED1_IRQHandler
                0x000001a0                DMIC0_DriverIRQHandler
                0x000001a0                RTC_IRQHandler
                0x000001a0                WAKE_UP_TIMER1_IRQHandler
                0x000001a0                RFP_AGC_IRQHandler
                0x000001a0                System_IRQHandler
                0x000001a0                WAKE_UP_TIMER0_IRQHandler
                0x000001a0                BLE_DP2_IRQHandler
                0x000001a0                PWM2_IRQHandler
                0x000001a0                PIN_INT1_DriverIRQHandler
                0x000001a0                PVT_RED0_IRQHandler
                0x000001a0                HWVAD0_DriverIRQHandler
                0x000001a0                PVT_AMBER1_IRQHandler
                0x000001a0                PWM10_IRQHandler
                0x000001a0                PWM4_IRQHandler
                0x000001a0                PWM7_IRQHandler
                0x000001a0                SPIFI_IRQHandler
                0x000001a0                MAILBOX_IRQHandler
                0x000001a0                ANA_COMP_IRQHandler
                0x000001a0                ADC_SEQA_IRQHandler
                0x000001a0                ADC_THCMP_OVR_IRQHandler
                0x000001a2                NMI_Handler
                0x000001a4                HardFault_Handler
                0x000001a6                MemManage_Handler
                0x000001a8                BusFault_Handler
                0x000001aa                UsageFault_Handler
                0x000001ac                SVC_Handler
                0x000001ae                DebugMon_Handler
                0x000001b0                PendSV_Handler
                0x000001b2                SysTick_Handler
                0x000001b4                MAC_154_IRQHandler
                0x000001d8                MODEM_154_IRQHandler
                0x000001fc                data_init
                0x00000210                bss_init
                0x00000232                ResetISR2
 *(.text*)
 .text.vMicroIntEnableOnly
                0x00000330       0x18 ./utilities/MicroInt_arm_sdk2.o
                0x00000330                vMicroIntEnableOnly
 .text.vMicroIntRestoreState
                0x00000348        0x8 ./utilities/MicroInt_arm_sdk2.o
                0x00000348                vMicroIntRestoreState
 .text.__assertion_failed
                0x00000350        0x2 ./utilities/Panic.o
                0x00000350                __assertion_failed
 *fill*         0x00000352        0x2 ff
 .text.DbgConsole_SendDataReliable
                0x00000354       0x34 ./utilities/fsl_debug_console.o
                0x00000354                DbgConsole_SendDataReliable
 .text.DbgConsole_PrintCallback
                0x00000388       0x3a ./utilities/fsl_debug_console.o
 *fill*         0x000003c2        0x2 ff
 .text.DbgConsole_Init
                0x000003c4       0x88 ./utilities/fsl_debug_console.o
                0x000003c4                DbgConsole_Init
 .text.DbgConsole_Printf
                0x0000044c       0x40 ./utilities/fsl_debug_console.o
                0x0000044c                DbgConsole_Printf
 .text.SerialManager_Init
                0x0000048c       0x40 ./utilities/serial_manager.o
                0x0000048c                SerialManager_Init
 .text.SerialManager_OpenWriteHandle
                0x000004cc       0x3c ./utilities/serial_manager.o
                0x000004cc                SerialManager_OpenWriteHandle
 .text.SerialManager_OpenReadHandle
                0x00000508       0x48 ./utilities/serial_manager.o
                0x00000508                SerialManager_OpenReadHandle
 .text.SerialManager_WriteBlocking
                0x00000550       0x44 ./utilities/serial_manager.o
                0x00000550                SerialManager_WriteBlocking
 .text.Serial_UartInit
                0x00000594       0x50 ./utilities/serial_port_uart.o
                0x00000594                Serial_UartInit
 .text.Serial_UartWrite
                0x000005e4       0x2c ./utilities/serial_port_uart.o
                0x000005e4                Serial_UartWrite
 .text.HAL_UartInit
                0x00000610       0xac ./utilities/usart_adapter.o
                0x00000610                HAL_UartInit
 .text.HAL_UartSendBlocking
                0x000006bc       0x38 ./utilities/usart_adapter.o
                0x000006bc                HAL_UartSendBlocking
 .text.DMIC0_IRQHandler
                0x000006f4        0x8 ./startup/startup_K32W061.o
                0x000006f4                DMIC0_IRQHandler
 .text.CIC_IRB_IRQHandler
                0x000006fc        0x8 ./startup/startup_K32W061.o
                0x000006fc                CIC_IRB_IRQHandler
 .text.HWVAD0_IRQHandler
                0x00000704        0x8 ./startup/startup_K32W061.o
                0x00000704                HWVAD0_IRQHandler
 .text.PINT0_IRQHandler
                0x0000070c        0x8 ./startup/startup_K32W061.o
                0x0000070c                PINT0_IRQHandler
 .text.PINT1_IRQHandler
                0x00000714        0x8 ./startup/startup_K32W061.o
                0x00000714                PINT1_IRQHandler
 .text.PINT2_IRQHandler
                0x0000071c        0x8 ./startup/startup_K32W061.o
                0x0000071c                PINT2_IRQHandler
 .text.PINT3_IRQHandler
                0x00000724        0x8 ./startup/startup_K32W061.o
                0x00000724                PINT3_IRQHandler
 .text.GINT0_IRQHandler
                0x0000072c        0x8 ./startup/startup_K32W061.o
                0x0000072c                GINT0_IRQHandler
 .text.CTIMER0_IRQHandler
                0x00000734        0x8 ./startup/startup_K32W061.o
                0x00000734                CTIMER0_IRQHandler
 .text.CTIMER1_IRQHandler
                0x0000073c        0x8 ./startup/startup_K32W061.o
                0x0000073c                CTIMER1_IRQHandler
 .text.FLEXCOMM0_IRQHandler
                0x00000744        0x8 ./startup/startup_K32W061.o
                0x00000744                FLEXCOMM0_IRQHandler
 .text.FLEXCOMM1_IRQHandler
                0x0000074c        0x8 ./startup/startup_K32W061.o
                0x0000074c                FLEXCOMM1_IRQHandler
 .text.FLEXCOMM2_IRQHandler
                0x00000754        0x8 ./startup/startup_K32W061.o
                0x00000754                FLEXCOMM2_IRQHandler
 .text.FLEXCOMM3_IRQHandler
                0x0000075c        0x8 ./startup/startup_K32W061.o
                0x0000075c                FLEXCOMM3_IRQHandler
 .text.FLEXCOMM4_IRQHandler
                0x00000764        0x8 ./startup/startup_K32W061.o
                0x00000764                FLEXCOMM4_IRQHandler
 .text.FLEXCOMM5_IRQHandler
                0x0000076c        0x8 ./startup/startup_K32W061.o
                0x0000076c                FLEXCOMM5_IRQHandler
 .text.FLEXCOMM6_IRQHandler
                0x00000774        0x8 ./startup/startup_K32W061.o
                0x00000774                FLEXCOMM6_IRQHandler
 .text.SystemCoreClockUpdate
                0x0000077c       0xa0 ./startup/system_K32W061.o
                0x0000077c                SystemCoreClockUpdate
 .text.SystemInit
                0x0000081c       0x44 ./startup/system_K32W061.o
                0x0000081c                SystemInit
 .text.bUartRxDataAvailable
                0x00000860        0xa ./source/tis_trp_dut.o
                0x00000860                bUartRxDataAvailable
 *fill*         0x0000086a        0x2 ff
 .text.APP_taskAtSerial
                0x0000086c       0x34 ./source/tis_trp_dut.o
                0x0000086c                APP_taskAtSerial
 .text.GPIO_set_level
                0x000008a0        0xc ./source/tis_trp_dut.o
                0x000008a0                GPIO_set_level
 .text.__main   0x000008ac       0x64 ./source/tis_trp_dut.o
                0x000008ac                __main
 .text.CLOCK_u8OscCapConvert
                0x00000910       0x22 ./drivers/fsl_clock.o
 *fill*         0x00000932        0x2 ff
 .text.CLOCK_AttachClk
                0x00000934      0x10c ./drivers/fsl_clock.o
                0x00000934                CLOCK_AttachClk
 .text.CLOCK_SetClkDiv
                0x00000a40       0x34 ./drivers/fsl_clock.o
                0x00000a40                CLOCK_SetClkDiv
 .text.CLOCK_GetXtal32kFreq
                0x00000a74       0x18 ./drivers/fsl_clock.o
                0x00000a74                CLOCK_GetXtal32kFreq
 .text.CLOCK_GetFro32kFreq
                0x00000a8c       0x18 ./drivers/fsl_clock.o
                0x00000a8c                CLOCK_GetFro32kFreq
 .text.CLOCK_GetOsc32kFreq
                0x00000aa4       0x14 ./drivers/fsl_clock.o
                0x00000aa4                CLOCK_GetOsc32kFreq
 .text.CLOCK_GetFro12MFreq
                0x00000ab8       0x18 ./drivers/fsl_clock.o
                0x00000ab8                CLOCK_GetFro12MFreq
 .text.CLOCK_GetFro32MFreq
                0x00000ad0       0x18 ./drivers/fsl_clock.o
                0x00000ad0                CLOCK_GetFro32MFreq
 .text.CLOCK_GetOsc32MFreq
                0x00000ae8       0x18 ./drivers/fsl_clock.o
                0x00000ae8                CLOCK_GetOsc32MFreq
 .text.CLOCK_GetWdtOscFreq
                0x00000b00       0x2c ./drivers/fsl_clock.o
                0x00000b00                CLOCK_GetWdtOscFreq
 .text.CLOCK_GetFro48MFreq
                0x00000b2c       0x18 ./drivers/fsl_clock.o
                0x00000b2c                CLOCK_GetFro48MFreq
 .text.CLOCK_GetPWMClockFreq
                0x00000b44       0x1e ./drivers/fsl_clock.o
                0x00000b44                CLOCK_GetPWMClockFreq
 *fill*         0x00000b62        0x2 ff
 .text.CLOCK_GetMainClockRate
                0x00000b64       0x40 ./drivers/fsl_clock.o
                0x00000b64                CLOCK_GetMainClockRate
 .text.CLOCK_GetCoreSysClkFreq
                0x00000ba4       0x18 ./drivers/fsl_clock.o
                0x00000ba4                CLOCK_GetCoreSysClkFreq
 .text.CLOCK_GetFRGInputClock
                0x00000bbc       0x26 ./drivers/fsl_clock.o
                0x00000bbc                CLOCK_GetFRGInputClock
 .text.CLOCK_GetFRGClock
                0x00000be2       0x32 ./drivers/fsl_clock.o
                0x00000be2                CLOCK_GetFRGClock
 .text.CLOCK_GetFro64MFreq
                0x00000c14       0x18 ./drivers/fsl_clock.o
                0x00000c14                CLOCK_GetFro64MFreq
 .text.CLOCK_GetClkOutFreq
                0x00000c2c       0x64 ./drivers/fsl_clock.o
                0x00000c2c                CLOCK_GetClkOutFreq
 .text.CLOCK_GetSpifiOscFreq
                0x00000c90       0x48 ./drivers/fsl_clock.o
                0x00000c90                CLOCK_GetSpifiOscFreq
 .text.CLOCK_GetApbCLkFreq
                0x00000cd8       0x2c ./drivers/fsl_clock.o
                0x00000cd8                CLOCK_GetApbCLkFreq
 .text.CLOCK_GetFreq
                0x00000d04      0x114 ./drivers/fsl_clock.o
                0x00000d04                CLOCK_GetFreq
 .text.CLOCK_EnableAPBBridge
                0x00000e18        0xe ./drivers/fsl_clock.o
                0x00000e18                CLOCK_EnableAPBBridge
 *fill*         0x00000e26        0x2 ff
 .text.CLOCK_uDelay
                0x00000e28       0x60 ./drivers/fsl_clock.o
                0x00000e28                CLOCK_uDelay
 .text.CLOCK_SetXtal32M_LDO
                0x00000e88       0x30 ./drivers/fsl_clock.o
                0x00000e88                CLOCK_SetXtal32M_LDO
 .text.CLOCK_Xtal32M_Trim
                0x00000eb8       0xf4 ./drivers/fsl_clock.o
                0x00000eb8                CLOCK_Xtal32M_Trim
 .text.CLOCK_XtalBasicTrim
                0x00000fac        0xc ./drivers/fsl_clock.o
                0x00000fac                CLOCK_XtalBasicTrim
 .text.CLOCK_Xtal32M_WaitUntilStable
                0x00000fb8       0x14 ./drivers/fsl_clock.o
                0x00000fb8                CLOCK_Xtal32M_WaitUntilStable
 .text.CLOCK_EnableClock
                0x00000fcc       0xdc ./drivers/fsl_clock.o
                0x00000fcc                CLOCK_EnableClock
 .text.EnableIRQ
                0x000010a8       0x28 ./drivers/fsl_ctimer.o
 .text.CTIMER_GetInstance.part.0
                0x000010d0       0x28 ./drivers/fsl_ctimer.o
 .text.CTIMER_Init
                0x000010f8       0x40 ./drivers/fsl_ctimer.o
                0x000010f8                CTIMER_Init
 .text.CTIMER_GetDefaultConfig
                0x00001138       0x20 ./drivers/fsl_ctimer.o
                0x00001138                CTIMER_GetDefaultConfig
 .text.CTIMER_SetupMatch
                0x00001158       0x88 ./drivers/fsl_ctimer.o
                0x00001158                CTIMER_SetupMatch
 .text.CTIMER_RegisterCallBack
                0x000011e0       0x20 ./drivers/fsl_ctimer.o
                0x000011e0                CTIMER_RegisterCallBack
 .text.CTIMER_GenericIRQHandler
                0x00001200       0x60 ./drivers/fsl_ctimer.o
                0x00001200                CTIMER_GenericIRQHandler
 .text.CTIMER0_DriverIRQHandler
                0x00001260        0xe ./drivers/fsl_ctimer.o
                0x00001260                CTIMER0_DriverIRQHandler
 .text.CTIMER1_DriverIRQHandler
                0x0000126e        0xe ./drivers/fsl_ctimer.o
                0x0000126e                CTIMER1_DriverIRQHandler
 .text.FLEXCOMM_GetInstance
                0x0000127c       0x28 ./drivers/fsl_flexcomm.o
                0x0000127c                FLEXCOMM_GetInstance
 .text.FLEXCOMM_Init
                0x000012a4       0x6c ./drivers/fsl_flexcomm.o
                0x000012a4                FLEXCOMM_Init
 .text.FLEXCOMM0_DriverIRQHandler
                0x00001310       0x2c ./drivers/fsl_flexcomm.o
                0x00001310                FLEXCOMM0_DriverIRQHandler
 .text.FLEXCOMM1_DriverIRQHandler
                0x0000133c       0x2c ./drivers/fsl_flexcomm.o
                0x0000133c                FLEXCOMM1_DriverIRQHandler
 .text.FLEXCOMM2_DriverIRQHandler
                0x00001368       0x2c ./drivers/fsl_flexcomm.o
                0x00001368                FLEXCOMM2_DriverIRQHandler
 .text.FLEXCOMM3_DriverIRQHandler
                0x00001394       0x2c ./drivers/fsl_flexcomm.o
                0x00001394                FLEXCOMM3_DriverIRQHandler
 .text.FLEXCOMM4_DriverIRQHandler
                0x000013c0       0x2c ./drivers/fsl_flexcomm.o
                0x000013c0                FLEXCOMM4_DriverIRQHandler
 .text.FLEXCOMM5_DriverIRQHandler
                0x000013ec       0x2c ./drivers/fsl_flexcomm.o
                0x000013ec                FLEXCOMM5_DriverIRQHandler
 .text.FLEXCOMM6_DriverIRQHandler
                0x00001418       0x2c ./drivers/fsl_flexcomm.o
                0x00001418                FLEXCOMM6_DriverIRQHandler
 .text.POWER_ApplyActiveVoltage
                0x00001444      0x128 ./drivers/fsl_power.o
                0x00001444                POWER_ApplyActiveVoltage
 .text.POWER_SetTrimDefaultActiveVoltage
                0x0000156c       0x50 ./drivers/fsl_power.o
                0x0000156c                POWER_SetTrimDefaultActiveVoltage
 .text.POWER_Init
                0x000015bc       0x20 ./drivers/fsl_power.o
                0x000015bc                POWER_Init
 .text.RESET_SetPeripheralReset
                0x000015dc       0x48 ./drivers/fsl_reset.o
                0x000015dc                RESET_SetPeripheralReset
 .text.RESET_ClearPeripheralReset
                0x00001624       0x4c ./drivers/fsl_reset.o
                0x00001624                RESET_ClearPeripheralReset
 .text.RESET_PeripheralReset
                0x00001670       0x12 ./drivers/fsl_reset.o
                0x00001670                RESET_PeripheralReset
 *fill*         0x00001682        0x2 ff
 .text.RESET_SystemReset
                0x00001684        0xc ./drivers/fsl_reset.o
                0x00001684                RESET_SystemReset
 .text.StrFormatPrintf
                0x00001690      0x21c ./drivers/fsl_str.o
                0x00001690                StrFormatPrintf
 .text.USART_GetDefaultConfig
                0x000018ac       0x30 ./drivers/fsl_usart.o
                0x000018ac                USART_GetDefaultConfig
 .text.USART_SetBaudRate
                0x000018dc       0x98 ./drivers/fsl_usart.o
                0x000018dc                USART_SetBaudRate
 .text.USART_Init
                0x00001974       0xfc ./drivers/fsl_usart.o
                0x00001974                USART_Init
 .text.USART_WriteBlocking
                0x00001a70       0x38 ./drivers/fsl_usart.o
                0x00001a70                USART_WriteBlocking
 .text.USART_ReadBlocking
                0x00001aa8       0x9c ./drivers/fsl_usart.o
                0x00001aa8                USART_ReadBlocking
 .text.BOARD_InitDebugConsole
                0x00001b44       0x28 ./board/board.o
                0x00001b44                BOARD_InitDebugConsole
 .text.BOARD_InitClocks
                0x00001b6c       0x88 ./board/hardware_init.o
                0x00001b6c                BOARD_InitClocks
 .text.BOARD_InitHardware
                0x00001bf4       0x40 ./board/hardware_init.o
                0x00001bf4                BOARD_InitHardware
 .text.BOARD_InitPins
                0x00001c34       0x48 ./board/pin_mux.o
                0x00001c34                BOARD_InitPins
 .text.reverse_16
                0x00001c7c       0x1a ./Common/CRC.o
 .text.reverse_8
                0x00001c96       0x1a ./Common/CRC.o
 .text.crc16    0x00001cb0       0x4e ./Common/CRC.o
 *fill*         0x00001cfe        0x2 ff
 .text.crc16ccitt_kermit
                0x00001d00       0x28 ./Common/CRC.o
                0x00001d00                crc16ccitt_kermit
 .text.ctimer_match0_callback
                0x00001d28       0x7c ./Common/Command.o
                0x00001d28                ctimer_match0_callback
 .text.vCommand_SetPower
                0x00001da4       0x30 ./Common/Command.o
                0x00001da4                vCommand_SetPower
 .text.vCommand_StartModulatedWaveTx
                0x00001dd4       0x80 ./Common/Command.o
                0x00001dd4                vCommand_StartModulatedWaveTx
 .text.vCommand_ResetCounters
                0x00001e54       0x60 ./Common/Command.o
                0x00001e54                vCommand_ResetCounters
 .text.vCommand_Transmit
                0x00001eb4       0x70 ./Common/Command.o
                0x00001eb4                vCommand_Transmit
 .text.vCommand_Task
                0x00001f24      0x1a8 ./Common/Command.o
                0x00001f24                vCommand_Task
 .text.vMMAC_Enable
                0x000020cc       0x64 C:/nxp/SDKPackages/SDK_2.6.0_K32W061DK6/middleware/wireless/ieee-802.15.4/lib\libMiniMac.a(MMAC.o)
                0x000020cc                vMMAC_Enable
 .text.u8MMAC_GetRxLqi
                0x00002130       0x18 C:/nxp/SDKPackages/SDK_2.6.0_K32W061DK6/middleware/wireless/ieee-802.15.4/lib\libMiniMac.a(MMAC.o)
                0x00002130                u8MMAC_GetRxLqi
 .text.vMMAC_SetTxParameters
                0x00002148       0x30 C:/nxp/SDKPackages/SDK_2.6.0_K32W061DK6/middleware/wireless/ieee-802.15.4/lib\libMiniMac.a(MMAC.o)
                0x00002148                vMMAC_SetTxParameters
 .text.vMMAC_SetCcaMode
                0x00002178       0x14 C:/nxp/SDKPackages/SDK_2.6.0_K32W061DK6/middleware/wireless/ieee-802.15.4/lib\libMiniMac.a(MMAC.o)
                0x00002178                vMMAC_SetCcaMode
 .text.u32MMAC_PollInterruptSource
                0x0000218c       0x10 C:/nxp/SDKPackages/SDK_2.6.0_K32W061DK6/middleware/wireless/ieee-802.15.4/lib\libMiniMac.a(MMAC.o)
                0x0000218c                u32MMAC_PollInterruptSource
 .text.u32MMAC_GetPhyState
                0x0000219c       0x44 C:/nxp/SDKPackages/SDK_2.6.0_K32W061DK6/middleware/wireless/ieee-802.15.4/lib\libMiniMac.a(MMAC.o)
                0x0000219c                u32MMAC_GetPhyState
 .text.vMMAC_CheckRxStarted
                0x000021e0       0x64 C:/nxp/SDKPackages/SDK_2.6.0_K32W061DK6/middleware/wireless/ieee-802.15.4/lib\libMiniMac.a(MMAC.o)
                0x000021e0                vMMAC_CheckRxStarted
 .text.vMMAC_AbortRadio
                0x00002244       0x4c C:/nxp/SDKPackages/SDK_2.6.0_K32W061DK6/middleware/wireless/ieee-802.15.4/lib\libMiniMac.a(MMAC.o)
                0x00002244                vMMAC_AbortRadio
 .text.vMMAC_RxCtlUpdate
                0x00002290       0x40 C:/nxp/SDKPackages/SDK_2.6.0_K32W061DK6/middleware/wireless/ieee-802.15.4/lib\libMiniMac.a(MMAC.o)
                0x00002290                vMMAC_RxCtlUpdate
 .text.vMMAC_RadioOff
                0x000022d0        0x6 C:/nxp/SDKPackages/SDK_2.6.0_K32W061DK6/middleware/wireless/ieee-802.15.4/lib\libMiniMac.a(MMAC.o)
                0x000022d0                vMMAC_RadioOff
 *fill*         0x000022d6        0x2 ff
 .text.vMMAC_RadioToOffAndWait
                0x000022d8       0x4c C:/nxp/SDKPackages/SDK_2.6.0_K32W061DK6/middleware/wireless/ieee-802.15.4/lib\libMiniMac.a(MMAC.o)
                0x000022d8                vMMAC_RadioToOffAndWait
 .text.vMMAC_StartPhyTransmit
                0x00002324       0x30 C:/nxp/SDKPackages/SDK_2.6.0_K32W061DK6/middleware/wireless/ieee-802.15.4/lib\libMiniMac.a(MMAC.o)
                0x00002324                vMMAC_StartPhyTransmit
 .text.vMMAC_SetChannelAndPower
                0x00002354       0x48 C:/nxp/SDKPackages/SDK_2.6.0_K32W061DK6/middleware/wireless/ieee-802.15.4/lib\libMiniMac.a(MMAC.o)
                0x00002354                vMMAC_SetChannelAndPower
 .text.vMMAC_SetChannel
                0x0000239c       0x14 C:/nxp/SDKPackages/SDK_2.6.0_K32W061DK6/middleware/wireless/ieee-802.15.4/lib\libMiniMac.a(MMAC.o)
                0x0000239c                vMMAC_SetChannel
 .text.vMMAC_StartPhyReceive
                0x000023b0       0x30 C:/nxp/SDKPackages/SDK_2.6.0_K32W061DK6/middleware/wireless/ieee-802.15.4/lib\libMiniMac.a(MMAC.o)
                0x000023b0                vMMAC_StartPhyReceive
 .text.vMMAC_WriteCcaThreshold
                0x000023e0       0x34 C:/nxp/SDKPackages/SDK_2.6.0_K32W061DK6/middleware/wireless/ieee-802.15.4/lib\libMiniMac.a(MMAC.o)
                0x000023e0                vMMAC_WriteCcaThreshold
 .text.vMMAC_SetHighPowerOptions
                0x00002414       0x10 C:/nxp/SDKPackages/SDK_2.6.0_K32W061DK6/middleware/wireless/ieee-802.15.4/lib\libMiniMac.a(MMAC.o)
                0x00002414                vMMAC_SetHighPowerOptions
 .text.vMMAC_IntHandlerBbc
                0x00002424       0x30 C:/nxp/SDKPackages/SDK_2.6.0_K32W061DK6/middleware/wireless/ieee-802.15.4/lib\libMiniMac.a(MMAC.o)
                0x00002424                vMMAC_IntHandlerBbc
 .text.vMMAC_IntHandlerPhy
                0x00002454       0x34 C:/nxp/SDKPackages/SDK_2.6.0_K32W061DK6/middleware/wireless/ieee-802.15.4/lib\libMiniMac.a(MMAC.o)
                0x00002454                vMMAC_IntHandlerPhy
 .text.bMMAC_PowerStatus
                0x00002488        0xe C:/nxp/SDKPackages/SDK_2.6.0_K32W061DK6/middleware/wireless/ieee-802.15.4/lib\libMiniMac.a(MMAC.o)
                0x00002488                bMMAC_PowerStatus
 *fill*         0x00002496        0x2 ff
 .text.vMMAC_Disable
                0x00002498       0x40 C:/nxp/SDKPackages/SDK_2.6.0_K32W061DK6/middleware/wireless/ieee-802.15.4/lib\libMiniMac.a(MMAC.o)
                0x00002498                vMMAC_Disable
 .text.vMMAC_ConfigureRadio
                0x000024d8       0x28 C:/nxp/SDKPackages/SDK_2.6.0_K32W061DK6/middleware/wireless/ieee-802.15.4/lib\libMiniMac.a(MMAC_RadioInit_JN518x.o)
                0x000024d8                vMMAC_ConfigureRadio
 .text.radio_IsNotC2MF
                0x00002500       0x4c C:/nxp/SDKPackages/SDK_2.6.0_K32W061DK6/middleware/wireless/framework/XCVR/lib\libRadio_Test_JN518x.a(radio.o)
                0x00002500                radio_IsNotC2MF
 .text.radio_CLOCK_FastuDelay
                0x0000254c       0x18 C:/nxp/SDKPackages/SDK_2.6.0_K32W061DK6/middleware/wireless/framework/XCVR/lib\libRadio_Test_JN518x.a(radio.o)
                0x0000254c                radio_CLOCK_FastuDelay
 .text.radio_TX_ZigBee_pll_dac_banked_set
                0x00002564       0x44 C:/nxp/SDKPackages/SDK_2.6.0_K32W061DK6/middleware/wireless/framework/XCVR/lib\libRadio_Test_JN518x.a(radio.o)
                0x00002564                radio_TX_ZigBee_pll_dac_banked_set
 .text.radio_fill_std_ZB_regs
                0x000025a8       0x1e C:/nxp/SDKPackages/SDK_2.6.0_K32W061DK6/middleware/wireless/framework/XCVR/lib\libRadio_Test_JN518x.a(radio.o)
                0x000025a8                radio_fill_std_ZB_regs
 .text.radio_fill_std_BLE1M_regs
                0x000025c6       0x1e C:/nxp/SDKPackages/SDK_2.6.0_K32W061DK6/middleware/wireless/framework/XCVR/lib\libRadio_Test_JN518x.a(radio.o)
                0x000025c6                radio_fill_std_BLE1M_regs
 .text.radio_fill_std_BLE2M_regs
                0x000025e4       0x1e C:/nxp/SDKPackages/SDK_2.6.0_K32W061DK6/middleware/wireless/framework/XCVR/lib\libRadio_Test_JN518x.a(radio.o)
                0x000025e4                radio_fill_std_BLE2M_regs
 .text.radio_fill_zbble_ZB_regs
                0x00002602       0x1e C:/nxp/SDKPackages/SDK_2.6.0_K32W061DK6/middleware/wireless/framework/XCVR/lib\libRadio_Test_JN518x.a(radio.o)
                0x00002602                radio_fill_zbble_ZB_regs
 .text.radio_fill_zbble_BLE_regs
                0x00002620       0x1e C:/nxp/SDKPackages/SDK_2.6.0_K32W061DK6/middleware/wireless/framework/XCVR/lib\libRadio_Test_JN518x.a(radio.o)
                0x00002620                radio_fill_zbble_BLE_regs
 .text.radio_fill_regs
                0x0000263e       0x1e C:/nxp/SDKPackages/SDK_2.6.0_K32W061DK6/middleware/wireless/framework/XCVR/lib\libRadio_Test_JN518x.a(radio.o)
                0x0000263e                radio_fill_regs
 .text.radio_power_down_to_off_polled
                0x0000265c       0x40 C:/nxp/SDKPackages/SDK_2.6.0_K32W061DK6/middleware/wireless/framework/XCVR/lib\libRadio_Test_JN518x.a(radio.o)
                0x0000265c                radio_power_down_to_off_polled
 .text.radio_pre_start_to_pll_polled
                0x0000269c       0x88 C:/nxp/SDKPackages/SDK_2.6.0_K32W061DK6/middleware/wireless/framework/XCVR/lib\libRadio_Test_JN518x.a(radio.o)
                0x0000269c                radio_pre_start_to_pll_polled
 .text.radio_rx_assert_polled
                0x00002724       0x40 C:/nxp/SDKPackages/SDK_2.6.0_K32W061DK6/middleware/wireless/framework/XCVR/lib\libRadio_Test_JN518x.a(radio.o)
                0x00002724                radio_rx_assert_polled
 .text.radio_rx_deassert_polled
                0x00002764       0x40 C:/nxp/SDKPackages/SDK_2.6.0_K32W061DK6/middleware/wireless/framework/XCVR/lib\libRadio_Test_JN518x.a(radio.o)
                0x00002764                radio_rx_deassert_polled
 .text.radio_RSSI_cal
                0x000027a4       0x6c C:/nxp/SDKPackages/SDK_2.6.0_K32W061DK6/middleware/wireless/framework/XCVR/lib\libRadio_Test_JN518x.a(radio.o)
                0x000027a4                radio_RSSI_cal
 .text.radio_Init
                0x00002810       0x44 C:/nxp/SDKPackages/SDK_2.6.0_K32W061DK6/middleware/wireless/framework/XCVR/lib\libRadio_Test_JN518x.a(radio.o)
                0x00002810                radio_Init
 .text.radio_TMU_Init
                0x00002854       0x18 C:/nxp/SDKPackages/SDK_2.6.0_K32W061DK6/middleware/wireless/framework/XCVR/lib\libRadio_Test_JN518x.a(radio.o)
                0x00002854                radio_TMU_Init
 .text.radio_Use_Cal_Values
                0x0000286c      0x14c C:/nxp/SDKPackages/SDK_2.6.0_K32W061DK6/middleware/wireless/framework/XCVR/lib\libRadio_Test_JN518x.a(radio.o)
                0x0000286c                radio_Use_Cal_Values
 .text.radio_Use_Retained_Cal_Values
                0x000029b8       0x50 C:/nxp/SDKPackages/SDK_2.6.0_K32W061DK6/middleware/wireless/framework/XCVR/lib\libRadio_Test_JN518x.a(radio.o)
                0x000029b8                radio_Use_Retained_Cal_Values
 .text.radio_rfbandgap_cal
                0x00002a08       0x30 C:/nxp/SDKPackages/SDK_2.6.0_K32W061DK6/middleware/wireless/framework/XCVR/lib\libRadio_Test_JN518x.a(radio.o)
                0x00002a08                radio_rfbandgap_cal
 .text.radio_Rc_Cal_init
                0x00002a38       0x78 C:/nxp/SDKPackages/SDK_2.6.0_K32W061DK6/middleware/wireless/framework/XCVR/lib\libRadio_Test_JN518x.a(radio.o)
                0x00002a38                radio_Rc_Cal_init
 .text.radio_Rc_Cal_algo
                0x00002ab0       0x4c C:/nxp/SDKPackages/SDK_2.6.0_K32W061DK6/middleware/wireless/framework/XCVR/lib\libRadio_Test_JN518x.a(radio.o)
                0x00002ab0                radio_Rc_Cal_algo
 .text.radio_Rc_Cal
                0x00002afc       0x10 C:/nxp/SDKPackages/SDK_2.6.0_K32W061DK6/middleware/wireless/framework/XCVR/lib\libRadio_Test_JN518x.a(radio.o)
                0x00002afc                radio_Rc_Cal
 .text.radio_Carrier_Frequency_Select_by_index
                0x00002b0c       0xa0 C:/nxp/SDKPackages/SDK_2.6.0_K32W061DK6/middleware/wireless/framework/XCVR/lib\libRadio_Test_JN518x.a(radio.o)
                0x00002b0c                radio_Carrier_Frequency_Select_by_index
 .text.radio_Synthesizer_Cw_Mode_Init
                0x00002bac       0x20 C:/nxp/SDKPackages/SDK_2.6.0_K32W061DK6/middleware/wireless/framework/XCVR/lib\libRadio_Test_JN518x.a(radio.o)
                0x00002bac                radio_Synthesizer_Cw_Mode_Init
 .text.radio_Trx_Packet_SW_Ctrl_Init
                0x00002bcc       0x20 C:/nxp/SDKPackages/SDK_2.6.0_K32W061DK6/middleware/wireless/framework/XCVR/lib\libRadio_Test_JN518x.a(radio.o)
                0x00002bcc                radio_Trx_Packet_SW_Ctrl_Init
 .text.radio_Disable_Auto_Kmod_Chan_and_Synth_Cal_Operation
                0x00002bec       0x20 C:/nxp/SDKPackages/SDK_2.6.0_K32W061DK6/middleware/wireless/framework/XCVR/lib\libRadio_Test_JN518x.a(radio.o)
                0x00002bec                radio_Disable_Auto_Kmod_Chan_and_Synth_Cal_Operation
 .text.radio_Synthesizer_Cal_Startup_init
                0x00002c0c       0x3c C:/nxp/SDKPackages/SDK_2.6.0_K32W061DK6/middleware/wireless/framework/XCVR/lib\libRadio_Test_JN518x.a(radio.o)
                0x00002c0c                radio_Synthesizer_Cal_Startup_init
 .text.radio_Synthesizer_Cal_Startup_algo
                0x00002c48      0x128 C:/nxp/SDKPackages/SDK_2.6.0_K32W061DK6/middleware/wireless/framework/XCVR/lib\libRadio_Test_JN518x.a(radio.o)
                0x00002c48                radio_Synthesizer_Cal_Startup_algo
 .text.radio_Synthesizer_Cal_Startup
                0x00002d70       0x7c C:/nxp/SDKPackages/SDK_2.6.0_K32W061DK6/middleware/wireless/framework/XCVR/lib\libRadio_Test_JN518x.a(radio.o)
                0x00002d70                radio_Synthesizer_Cal_Startup
 .text.radio_Synthesizer_Cal_Operation_And_Lock_init
                0x00002dec       0x70 C:/nxp/SDKPackages/SDK_2.6.0_K32W061DK6/middleware/wireless/framework/XCVR/lib\libRadio_Test_JN518x.a(radio.o)
                0x00002dec                radio_Synthesizer_Cal_Operation_And_Lock_init
 .text.radio_Synthesizer_Cal_Operation_And_Lock_algo
                0x00002e5c       0x44 C:/nxp/SDKPackages/SDK_2.6.0_K32W061DK6/middleware/wireless/framework/XCVR/lib\libRadio_Test_JN518x.a(radio.o)
                0x00002e5c                radio_Synthesizer_Cal_Operation_And_Lock_algo
 .text.radio_Synthesizer_Cal_Operation_And_Lock
                0x00002ea0       0x12 C:/nxp/SDKPackages/SDK_2.6.0_K32W061DK6/middleware/wireless/framework/XCVR/lib\libRadio_Test_JN518x.a(radio.o)
                0x00002ea0                radio_Synthesizer_Cal_Operation_And_Lock
 *fill*         0x00002eb2        0x2 ff
 .text.radio_Synthesizer_Kmod_Band_init
                0x00002eb4      0x100 C:/nxp/SDKPackages/SDK_2.6.0_K32W061DK6/middleware/wireless/framework/XCVR/lib\libRadio_Test_JN518x.a(radio.o)
                0x00002eb4                radio_Synthesizer_Kmod_Band_init
 .text.radio_Synthesizer_Kmod_Band_algo
                0x00002fb4       0xcc C:/nxp/SDKPackages/SDK_2.6.0_K32W061DK6/middleware/wireless/framework/XCVR/lib\libRadio_Test_JN518x.a(radio.o)
                0x00002fb4                radio_Synthesizer_Kmod_Band_algo
 .text.radio_Synthesizer_Kmod_Band
                0x00003080      0x1f8 C:/nxp/SDKPackages/SDK_2.6.0_K32W061DK6/middleware/wireless/framework/XCVR/lib\libRadio_Test_JN518x.a(radio.o)
                0x00003080                radio_Synthesizer_Kmod_Band
 .text.radio_Trx_Packet_HW_Ctrl_Init
                0x00003278       0x94 C:/nxp/SDKPackages/SDK_2.6.0_K32W061DK6/middleware/wireless/framework/XCVR/lib\libRadio_Test_JN518x.a(radio.o)
                0x00003278                radio_Trx_Packet_HW_Ctrl_Init
 .text.radio_Synthesizer_Full_Cal
                0x0000330c       0x54 C:/nxp/SDKPackages/SDK_2.6.0_K32W061DK6/middleware/wireless/framework/XCVR/lib\libRadio_Test_JN518x.a(radio.o)
                0x0000330c                radio_Synthesizer_Full_Cal
 .text.radio_PA_rewrite_lut
                0x00003360      0x2c4 C:/nxp/SDKPackages/SDK_2.6.0_K32W061DK6/middleware/wireless/framework/XCVR/lib\libRadio_Test_JN518x.a(radio.o)
                0x00003360                radio_PA_rewrite_lut
 .text.radio_PA_cal
                0x00003624        0x8 C:/nxp/SDKPackages/SDK_2.6.0_K32W061DK6/middleware/wireless/framework/XCVR/lib\libRadio_Test_JN518x.a(radio.o)
                0x00003624                radio_PA_cal
 .text.radio_DCO_cal_init
                0x0000362c      0x1f0 C:/nxp/SDKPackages/SDK_2.6.0_K32W061DK6/middleware/wireless/framework/XCVR/lib\libRadio_Test_JN518x.a(radio.o)
                0x0000362c                radio_DCO_cal_init
 .text.radio_DCO_cal
                0x0000381c      0x6c4 C:/nxp/SDKPackages/SDK_2.6.0_K32W061DK6/middleware/wireless/framework/XCVR/lib\libRadio_Test_JN518x.a(radio.o)
                0x0000381c                radio_DCO_cal
 .text.radio_IQ_cal
                0x00003ee0       0x50 C:/nxp/SDKPackages/SDK_2.6.0_K32W061DK6/middleware/wireless/framework/XCVR/lib\libRadio_Test_JN518x.a(radio.o)
                0x00003ee0                radio_IQ_cal
 .text.radio_PowerOnCheckXtal
                0x00003f30      0x144 C:/nxp/SDKPackages/SDK_2.6.0_K32W061DK6/middleware/wireless/framework/XCVR/lib\libRadio_Test_JN518x.a(radio.o)
                0x00003f30                radio_PowerOnCheckXtal
 .text.radio_PowerOn
                0x00004074       0x90 C:/nxp/SDKPackages/SDK_2.6.0_K32W061DK6/middleware/wireless/framework/XCVR/lib\libRadio_Test_JN518x.a(radio.o)
                0x00004074                radio_PowerOn
 .text.vRadio_PowerOnSpecific
                0x00004104       0x8c C:/nxp/SDKPackages/SDK_2.6.0_K32W061DK6/middleware/wireless/framework/XCVR/lib\libRadio_Test_JN518x.a(radio.o)
                0x00004104                vRadio_PowerOnSpecific
 .text.vRadio_InitXtal
                0x00004190       0x74 C:/nxp/SDKPackages/SDK_2.6.0_K32W061DK6/middleware/wireless/framework/XCVR/lib\libRadio_Test_JN518x.a(radio.o)
                0x00004190                vRadio_InitXtal
 .text.radio_get_retention_info
                0x00004204       0x48 C:/nxp/SDKPackages/SDK_2.6.0_K32W061DK6/middleware/wireless/framework/XCVR/lib\libRadio_Test_JN518x.a(radio.o)
                0x00004204                radio_get_retention_info
 .text.vRadio_Standard_Init
                0x0000424c      0x358 C:/nxp/SDKPackages/SDK_2.6.0_K32W061DK6/middleware/wireless/framework/XCVR/lib\libRadio_Test_JN518x.a(radio.o)
                0x0000424c                vRadio_Standard_Init
 .text.u8Radio_GetEDfromRSSI
                0x000045a4       0x28 C:/nxp/SDKPackages/SDK_2.6.0_K32W061DK6/middleware/wireless/framework/XCVR/lib\libRadio_Test_JN518x.a(radio.o)
                0x000045a4                u8Radio_GetEDfromRSSI
 .text.vGetCalInfo
                0x000045cc       0x40 C:/nxp/SDKPackages/SDK_2.6.0_K32W061DK6/middleware/wireless/framework/XCVR/lib\libRadio_Test_JN518x.a(radio.o)
                0x000045cc                vGetCalInfo
 .text.vRadio_RFT1778_bad_crc
                0x0000460c       0x40 C:/nxp/SDKPackages/SDK_2.6.0_K32W061DK6/middleware/wireless/framework/XCVR/lib\libRadio_Test_JN518x.a(radio.o)
                0x0000460c                vRadio_RFT1778_bad_crc
 .text.vRadio_AD_control
                0x0000464c       0x70 C:/nxp/SDKPackages/SDK_2.6.0_K32W061DK6/middleware/wireless/framework/XCVR/lib\libRadio_Test_JN518x.a(radio.o)
                0x0000464c                vRadio_AD_control
 .text.vRadio_UpdateRadioStandard
                0x000046bc       0x50 C:/nxp/SDKPackages/SDK_2.6.0_K32W061DK6/middleware/wireless/framework/XCVR/lib\libRadio_Test_JN518x.a(radio.o)
                0x000046bc                vRadio_UpdateRadioStandard
 .text.vRadio_InitialiseRadioStandard
                0x0000470c       0x20 C:/nxp/SDKPackages/SDK_2.6.0_K32W061DK6/middleware/wireless/framework/XCVR/lib\libRadio_Test_JN518x.a(radio.o)
                0x0000470c                vRadio_InitialiseRadioStandard
 .text.vRadio_SetChannelAndPower
                0x0000472c       0x50 C:/nxp/SDKPackages/SDK_2.6.0_K32W061DK6/middleware/wireless/framework/XCVR/lib\libRadio_Test_JN518x.a(radio.o)
                0x0000472c                vRadio_SetChannelAndPower
 .text.i8Radio_GetTxPowerLevel_dBm
                0x0000477c       0x18 C:/nxp/SDKPackages/SDK_2.6.0_K32W061DK6/middleware/wireless/framework/XCVR/lib\libRadio_Test_JN518x.a(radio.o)
                0x0000477c                i8Radio_GetTxPowerLevel_dBm
 .text.vRadio_Temp_GetInfos
                0x00004794       0x90 C:/nxp/SDKPackages/SDK_2.6.0_K32W061DK6/middleware/wireless/framework/XCVR/lib\libRadio_Test_JN518x.a(radio.o)
                0x00004794                vRadio_Temp_GetInfos
 .text.vRadio_Temp_SetInfos
                0x00004824       0x8c C:/nxp/SDKPackages/SDK_2.6.0_K32W061DK6/middleware/wireless/framework/XCVR/lib\libRadio_Test_JN518x.a(radio.o)
                0x00004824                vRadio_Temp_SetInfos
 .text.vRadio_start_rx_ISR
                0x000048b0       0x20 C:/nxp/SDKPackages/SDK_2.6.0_K32W061DK6/middleware/wireless/framework/XCVR/lib\libRadio_Test_JN518x.a(radio.o)
                0x000048b0                vRadio_start_rx_ISR
 .text.vRadio_remove_patch_ISR
                0x000048d0       0x2c C:/nxp/SDKPackages/SDK_2.6.0_K32W061DK6/middleware/wireless/framework/XCVR/lib\libRadio_Test_JN518x.a(radio.o)
                0x000048d0                vRadio_remove_patch_ISR
 .text.RFP_TMU_IRQHandler
                0x000048fc       0x40 C:/nxp/SDKPackages/SDK_2.6.0_K32W061DK6/middleware/wireless/framework/XCVR/lib\libRadio_Test_JN518x.a(radio.o)
                0x000048fc                RFP_TMU_IRQHandler
 .text.vRadio_Enable_DCO_DAC
                0x0000493c       0xe0 C:/nxp/SDKPackages/SDK_2.6.0_K32W061DK6/middleware/wireless/framework/XCVR/lib\libRadio_Test_JN518x.a(radio.o)
                0x0000493c                vRadio_Enable_DCO_DAC
 .text.vRadio_Disable_DCO_DAC
                0x00004a1c       0x40 C:/nxp/SDKPackages/SDK_2.6.0_K32W061DK6/middleware/wireless/framework/XCVR/lib\libRadio_Test_JN518x.a(radio.o)
                0x00004a1c                vRadio_Disable_DCO_DAC
 .text.vRadio_RadioDeInit
                0x00004a5c       0x18 C:/nxp/SDKPackages/SDK_2.6.0_K32W061DK6/middleware/wireless/framework/XCVR/lib\libRadio_Test_JN518x.a(radio.o)
                0x00004a5c                vRadio_RadioDeInit
 .text.bIsCalNeeded
                0x00004a74       0x50 C:/nxp/SDKPackages/SDK_2.6.0_K32W061DK6/middleware/wireless/framework/XCVR/lib\libRadio_Test_JN518x.a(radio.o)
                0x00004a74                bIsCalNeeded
 .text.vUpdateFlashCalData
                0x00004ac4       0x3c C:/nxp/SDKPackages/SDK_2.6.0_K32W061DK6/middleware/wireless/framework/XCVR/lib\libRadio_Test_JN518x.a(radio.o)
                0x00004ac4                vUpdateFlashCalData
 .text.vInitFlashCalData
                0x00004b00      0x27c C:/nxp/SDKPackages/SDK_2.6.0_K32W061DK6/middleware/wireless/framework/XCVR/lib\libRadio_Test_JN518x.a(radio.o)
                0x00004b00                vInitFlashCalData
 .text.vCheckFlashCalData
                0x00004d7c      0x178 C:/nxp/SDKPackages/SDK_2.6.0_K32W061DK6/middleware/wireless/framework/XCVR/lib\libRadio_Test_JN518x.a(radio.o)
                0x00004d7c                vCheckFlashCalData
 .text.vRadio_RadioInit
                0x00004ef4      0x2ec C:/nxp/SDKPackages/SDK_2.6.0_K32W061DK6/middleware/wireless/framework/XCVR/lib\libRadio_Test_JN518x.a(radio.o)
                0x00004ef4                vRadio_RadioInit
 .text.vRadio_Test_Jn518x_TxPowerTest
                0x000051e0       0xe0 C:/nxp/SDKPackages/SDK_2.6.0_K32W061DK6/middleware/wireless/framework/XCVR/lib\libRadio_Test_JN518x.a(radio_test_jn518x.o)
                0x000051e0                vRadio_Test_Jn518x_TxPowerTest
 .text.ZIGBEE_MODEM_IRQHandler
                0x000052c0       0x8c C:/nxp/SDKPackages/SDK_2.6.0_K32W061DK6/middleware/wireless/framework/XCVR/lib\libRadio_Test_JN518x.a(radio_test_jn518x.o)
                0x000052c0                ZIGBEE_MODEM_IRQHandler
 .text.ZIGBEE_MAC_IRQHandler
                0x0000534c       0x10 C:/nxp/SDKPackages/SDK_2.6.0_K32W061DK6/middleware/wireless/framework/XCVR/lib\libRadio_Test_JN518x.a(radio_test_jn518x.o)
                0x0000534c                ZIGBEE_MAC_IRQHandler
 .text          0x0000535c      0x378 c:/nxp/mcuxpressoide_11.1.0_3209/ide/plugins/com.nxp.mcuxpresso.tools.win32_11.1.0.201909161352/tools/bin/../lib/gcc/arm-none-eabi/8.3.1/thumb/v7e-m/nofp\libgcc.a(_arm_addsubdf3.o)
                0x0000535c                __aeabi_drsub
                0x00005364                __aeabi_dsub
                0x00005364                __subdf3
                0x00005368                __aeabi_dadd
                0x00005368                __adddf3
                0x000055e0                __floatunsidf
                0x000055e0                __aeabi_ui2d
                0x00005600                __floatsidf
                0x00005600                __aeabi_i2d
                0x00005624                __aeabi_f2d
                0x00005624                __extendsfdf2
                0x00005668                __floatundidf
                0x00005668                __aeabi_ul2d
                0x00005678                __floatdidf
                0x00005678                __aeabi_l2d
 .text          0x000056d4       0x50 c:/nxp/mcuxpressoide_11.1.0_3209/ide/plugins/com.nxp.mcuxpresso.tools.win32_11.1.0.201909161352/tools/bin/../lib/gcc/arm-none-eabi/8.3.1/thumb/v7e-m/nofp\libgcc.a(_arm_fixdfsi.o)
                0x000056d4                __aeabi_d2iz
                0x000056d4                __fixdfsi
 .text          0x00005724       0x30 c:/nxp/mcuxpressoide_11.1.0_3209/ide/plugins/com.nxp.mcuxpresso.tools.win32_11.1.0.201909161352/tools/bin/../lib/gcc/arm-none-eabi/8.3.1/thumb/v7e-m/nofp\libgcc.a(_aeabi_uldivmod.o)
                0x00005724                __aeabi_uldivmod
 .text          0x00005754      0x2d0 c:/nxp/mcuxpressoide_11.1.0_3209/ide/plugins/com.nxp.mcuxpresso.tools.win32_11.1.0.201909161352/tools/bin/../lib/gcc/arm-none-eabi/8.3.1/thumb/v7e-m/nofp\libgcc.a(_udivmoddi4.o)
                0x00005754                __udivmoddi4
 .text          0x00005a24        0x4 c:/nxp/mcuxpressoide_11.1.0_3209/ide/plugins/com.nxp.mcuxpresso.tools.win32_11.1.0.201909161352/tools/bin/../lib/gcc/arm-none-eabi/8.3.1/thumb/v7e-m/nofp\libgcc.a(_dvmd_tls.o)
                0x00005a24                __aeabi_idiv0
                0x00005a24                __aeabi_ldiv0
 .text.abs      0x00005a28        0x8 c:/nxp/mcuxpressoide_11.1.0_3209/ide/plugins/com.nxp.mcuxpresso.tools.win32_11.1.0.201909161352/tools/bin/../lib/gcc/arm-none-eabi/8.3.1/../../../../arm-none-eabi/lib/thumb/v7e-m/nofp\libg.a(lib_a-abs.o)
                0x00005a28                abs
 .text          0x00005a30      0x134 c:/nxp/mcuxpressoide_11.1.0_3209/ide/plugins/com.nxp.mcuxpresso.tools.win32_11.1.0.201909161352/tools/bin/../lib/gcc/arm-none-eabi/8.3.1/../../../../arm-none-eabi/lib/thumb/v7e-m/nofp\libg.a(lib_a-memcpy.o)
                0x00005a30                memcpy
 .text.memset   0x00005b64       0xa0 c:/nxp/mcuxpressoide_11.1.0_3209/ide/plugins/com.nxp.mcuxpresso.tools.win32_11.1.0.201909161352/tools/bin/../lib/gcc/arm-none-eabi/8.3.1/../../../../arm-none-eabi/lib/thumb/v7e-m/nofp\libg.a(lib_a-memset.o)
                0x00005b64                memset
 *fill*         0x00005c04       0x3c ff
 .text          0x00005c40       0xdc c:/nxp/mcuxpressoide_11.1.0_3209/ide/plugins/com.nxp.mcuxpresso.tools.win32_11.1.0.201909161352/tools/bin/../lib/gcc/arm-none-eabi/8.3.1/../../../../arm-none-eabi/lib/thumb/v7e-m/nofp\libg.a(lib_a-strlen.o)
                0x00005c40                strlen
 *(.rodata .rodata.* .constdata .constdata.*)
 .rodata.DbgConsole_Init.str1.1
                0x00005d1c      0x1b6 ./utilities/fsl_debug_console.o
 .rodata.DbgConsole_SendDataReliable.str1.1
                0x00005ed2       0xe9 ./utilities/fsl_debug_console.o
 .rodata.SerialManager_Init.str1.1
                0x00005fbb       0xc6 ./utilities/serial_manager.o
 .rodata.SerialManager_OpenReadHandle.str1.1
                0x00006081       0xcc ./utilities/serial_manager.o
 .rodata.SerialManager_OpenWriteHandle.str1.1
                0x0000614d       0xcc ./utilities/serial_manager.o
 .rodata.SerialManager_WriteBlocking.str1.1
                0x00006219      0x185 ./utilities/serial_manager.o
 .rodata.Serial_UartInit.str1.1
                0x0000639e       0xd0 ./utilities/serial_port_uart.o
 .rodata.Serial_UartWrite.str1.1
                0x0000646e      0x12c ./utilities/serial_port_uart.o
 .rodata.HAL_UartInit.str1.1
                0x0000659a      0x1b2 ./utilities/usart_adapter.o
 .rodata.HAL_UartSendBlocking.str1.1
                0x0000674c       0xfd ./utilities/usart_adapter.o
 *fill*         0x00006849        0x3 ff
 .rodata.s_UsartAdapterBase
                0x0000684c        0x8 ./utilities/usart_adapter.o
 .rodata.__main.str1.1
                0x00006854       0x1b ./source/tis_trp_dut.o
 *fill*         0x0000686f        0x1 ff
 .rodata.default_Clock32MCapacitanceCharacteristics
                0x00006870        0xc ./drivers/fsl_clock.o
                0x00006870                default_Clock32MCapacitanceCharacteristics
 .rodata.CTIMER_GetDefaultConfig.str1.1
                0x0000687c       0x5a ./drivers/fsl_ctimer.o
 .rodata.CTIMER_GetInstance.part.0.str1.1
                0x000068d6       0x6e ./drivers/fsl_ctimer.o
 .rodata.CTIMER_Init.str1.1
                0x00006944       0x59 ./drivers/fsl_ctimer.o
 *fill*         0x0000699d        0x3 ff
 .rodata.s_ctimerBases
                0x000069a0        0x8 ./drivers/fsl_ctimer.o
 .rodata.s_ctimerClocks
                0x000069a8        0x8 ./drivers/fsl_ctimer.o
 .rodata.s_ctimerIRQ
                0x000069b0        0x2 ./drivers/fsl_ctimer.o
 *fill*         0x000069b2        0x2 ff
 .rodata.s_ctimerResets
                0x000069b4        0x8 ./drivers/fsl_ctimer.o
 .rodata.FLEXCOMM0_DriverIRQHandler.str1.1
                0x000069bc       0x6d ./drivers/fsl_flexcomm.o
 .rodata.FLEXCOMM1_DriverIRQHandler.str1.1
                0x00006a29       0x6d ./drivers/fsl_flexcomm.o
 .rodata.FLEXCOMM2_DriverIRQHandler.str1.1
                0x00006a96       0x6d ./drivers/fsl_flexcomm.o
 .rodata.FLEXCOMM3_DriverIRQHandler.str1.1
                0x00006b03       0x6d ./drivers/fsl_flexcomm.o
 .rodata.FLEXCOMM4_DriverIRQHandler.str1.1
                0x00006b70       0x6d ./drivers/fsl_flexcomm.o
 .rodata.FLEXCOMM5_DriverIRQHandler.str1.1
                0x00006bdd       0x6d ./drivers/fsl_flexcomm.o
 .rodata.FLEXCOMM6_DriverIRQHandler.str1.1
                0x00006c4a       0x6d ./drivers/fsl_flexcomm.o
 .rodata.FLEXCOMM_GetInstance.str1.1
                0x00006cb7       0x5a ./drivers/fsl_flexcomm.o
 *fill*         0x00006d11        0x3 ff
 .rodata.s_flexcommBaseAddrs
                0x00006d14       0x1c ./drivers/fsl_flexcomm.o
 .rodata.s_flexcommClocks
                0x00006d30       0x1c ./drivers/fsl_flexcomm.o
 .rodata.lowpower_ldovoltage_reset
                0x00006d4c        0x9 ./drivers/fsl_power.o
 .rodata.RESET_ClearPeripheralReset.str1.1
                0x00006d55       0x5e ./drivers/fsl_reset.o
 .rodata.RESET_SetPeripheralReset.str1.1
                0x00006db3       0x5e ./drivers/fsl_reset.o
 .rodata.USART_GetDefaultConfig.str1.1
                0x00006e11       0x61 ./drivers/fsl_usart.o
 .rodata.USART_Init.str1.1
                0x00006e72       0x8e ./drivers/fsl_usart.o
 .rodata.USART_ReadBlocking.str1.1
                0x00006f00       0x76 ./drivers/fsl_usart.o
 .rodata.USART_SetBaudRate.str1.1
                0x00006f76       0x91 ./drivers/fsl_usart.o
 .rodata.USART_WriteBlocking.str1.1
                0x00007007       0x76 ./drivers/fsl_usart.o
 .rodata.ctimer_match0_callback.str1.1
                0x0000707d       0x10 ./Common/Command.o
 .rodata.vCommand_ResetCounters.str1.1
                0x0000708d       0x86 ./Common/Command.o
 .rodata.vCommand_SetPower.str1.1
                0x00007113       0x19 ./Common/Command.o
 .rodata.vCommand_StartModulatedWaveTx.str1.1
                0x0000712c       0x10 ./Common/Command.o
 .rodata.vCommand_Task.str1.1
                0x0000713c       0x2c ./Common/Command.o
 .rodata        0x00007168       0x32 C:/nxp/SDKPackages/SDK_2.6.0_K32W061DK6/middleware/wireless/framework/XCVR/lib\libRadio_Test_JN518x.a(radio.o)
 *fill*         0x0000719a        0x2 ff
 .rodata.assign_Synth_Cal_Op_Lock_init_regs
                0x0000719c       0x40 C:/nxp/SDKPackages/SDK_2.6.0_K32W061DK6/middleware/wireless/framework/XCVR/lib\libRadio_Test_JN518x.a(radio.o)
                0x0000719c                assign_Synth_Cal_Op_Lock_init_regs
 .rodata.assign_Synth_Cal_Startup_init_regs
                0x000071dc       0x44 C:/nxp/SDKPackages/SDK_2.6.0_K32W061DK6/middleware/wireless/framework/XCVR/lib\libRadio_Test_JN518x.a(radio.o)
                0x000071dc                assign_Synth_Cal_Startup_init_regs
 .rodata.assign_TMU_init_regs
                0x00007220       0x4c C:/nxp/SDKPackages/SDK_2.6.0_K32W061DK6/middleware/wireless/framework/XCVR/lib\libRadio_Test_JN518x.a(radio.o)
                0x00007220                assign_TMU_init_regs
 .rodata.assign_init_regs
                0x0000726c       0x70 C:/nxp/SDKPackages/SDK_2.6.0_K32W061DK6/middleware/wireless/framework/XCVR/lib\libRadio_Test_JN518x.a(radio.o)
                0x0000726c                assign_init_regs
 .rodata.assign_init_regs_ES2
                0x000072dc        0xc C:/nxp/SDKPackages/SDK_2.6.0_K32W061DK6/middleware/wireless/framework/XCVR/lib\libRadio_Test_JN518x.a(radio.o)
                0x000072dc                assign_init_regs_ES2
 .rodata.assign_init_regs_ES2MF
                0x000072e8        0xc C:/nxp/SDKPackages/SDK_2.6.0_K32W061DK6/middleware/wireless/framework/XCVR/lib\libRadio_Test_JN518x.a(radio.o)
                0x000072e8                assign_init_regs_ES2MF
 .rodata.assign_std_specific_banked_regs
                0x000072f4       0x38 C:/nxp/SDKPackages/SDK_2.6.0_K32W061DK6/middleware/wireless/framework/XCVR/lib\libRadio_Test_JN518x.a(radio.o)
                0x000072f4                assign_std_specific_banked_regs
 .rodata.assign_unbanked_common_regs
                0x0000732c       0x28 C:/nxp/SDKPackages/SDK_2.6.0_K32W061DK6/middleware/wireless/framework/XCVR/lib\libRadio_Test_JN518x.a(radio.o)
                0x0000732c                assign_unbanked_common_regs
 .rodata.assign_unbanked_std_specific_regs
                0x00007354       0x10 C:/nxp/SDKPackages/SDK_2.6.0_K32W061DK6/middleware/wireless/framework/XCVR/lib\libRadio_Test_JN518x.a(radio.o)
                0x00007354                assign_unbanked_std_specific_regs
 .rodata.assign_unbanked_zbble_specific_regs
                0x00007364       0x9c C:/nxp/SDKPackages/SDK_2.6.0_K32W061DK6/middleware/wireless/framework/XCVR/lib\libRadio_Test_JN518x.a(radio.o)
                0x00007364                assign_unbanked_zbble_specific_regs
 .rodata.assign_zbble_specific_banked_regs
                0x00007400       0x48 C:/nxp/SDKPackages/SDK_2.6.0_K32W061DK6/middleware/wireless/framework/XCVR/lib\libRadio_Test_JN518x.a(radio.o)
                0x00007400                assign_zbble_specific_banked_regs
 .rodata.freq_prog
                0x00007448       0x8c C:/nxp/SDKPackages/SDK_2.6.0_K32W061DK6/middleware/wireless/framework/XCVR/lib\libRadio_Test_JN518x.a(radio.o)
                0x00007448                freq_prog
 .rodata.lut_defaults
                0x000074d4       0x5c C:/nxp/SDKPackages/SDK_2.6.0_K32W061DK6/middleware/wireless/framework/XCVR/lib\libRadio_Test_JN518x.a(radio.o)
                0x000074d4                lut_defaults
 .rodata.lut_hiTx_defaults
                0x00007530       0x5c C:/nxp/SDKPackages/SDK_2.6.0_K32W061DK6/middleware/wireless/framework/XCVR/lib\libRadio_Test_JN518x.a(radio.o)
                0x00007530                lut_hiTx_defaults
                0x0000758c                . = ALIGN (0x4)

.glue_7         0x0000758c        0x0
 .glue_7        0x0000758c        0x0 linker stubs

.glue_7t        0x0000758c        0x0
 .glue_7t       0x0000758c        0x0 linker stubs

.vfp11_veneer   0x0000758c        0x0
 .vfp11_veneer  0x0000758c        0x0 linker stubs

.v4_bx          0x0000758c        0x0
 .v4_bx         0x0000758c        0x0 linker stubs

.iplt           0x0000758c        0x0
 .iplt          0x0000758c        0x0 ./utilities/MicroInt_arm_sdk2.o

.ARM.extab      0x0000758c        0x0
 FILL mask 0xff
 *(.ARM.extab* .gnu.linkonce.armextab.*)
                0x0000758c                __exidx_start = .

.ARM.exidx      0x0000758c        0x8
 FILL mask 0xff
 *(.ARM.exidx* .gnu.linkonce.armexidx.*)
 .ARM.exidx     0x0000758c        0x8 c:/nxp/mcuxpressoide_11.1.0_3209/ide/plugins/com.nxp.mcuxpresso.tools.win32_11.1.0.201909161352/tools/bin/../lib/gcc/arm-none-eabi/8.3.1/thumb/v7e-m/nofp\libgcc.a(_udivmoddi4.o)
                0x00007594                __exidx_end = .
                0x00007594                _etext = .

.rel.dyn        0x00007594        0x0
 .rel.iplt      0x00007594        0x0 ./utilities/MicroInt_arm_sdk2.o

.data_RAM2      0x04020000        0x0 load address 0x00007594
 FILL mask 0xff
                [!provide]                PROVIDE (__start_data_RAM2 = .)
 *(.ramfunc.$RAM2)
 *(.ramfunc.$RAM1)
 *(.data.$RAM2*)
 *(.data.$RAM1*)
                0x04020000                . = ALIGN (0x4)
                [!provide]                PROVIDE (__end_data_RAM2 = .)

.interrupts_ram
                0x04000400        0x0
                0x04000400                . = ALIGN (0x4)
                0x04000400                __VECTOR_RAM__ = .
                0x04000400                __interrupts_ram_start__ = .
 *(.m_interrupts_ram)
                0x04000400                . = (. + M_VECTOR_RAM_SIZE)
                0x04000400                . = ALIGN (0x4)
                0x04000400                __interrupts_ram_end__ = .

.uninit_RESERVED
                0x04000400        0x0
 *(.bss.$RESERVED*)
                0x04000400                . = ALIGN (0x4)
                0x04000400                _end_uninit_RESERVED = .

.data           0x04000400       0x84 load address 0x00007594
 FILL mask 0xff
                0x04000400                _data = .
 *(vtable)
 *(.ramfunc*)
 *(.data*)
 .data.SystemCoreClock
                0x04000400        0x4 ./startup/system_K32W061.o
                0x04000400                SystemCoreClock
 .data.active_trim_val
                0x04000404        0x1 ./drivers/fsl_power.o
 .data.pwd_trim_val
                0x04000405        0x1 ./drivers/fsl_power.o
 *fill*         0x04000406        0x2 ff
 .data.ctimer_callback_table
                0x04000408       0x20 ./Common/Command.o
                0x04000408                ctimer_callback_table
 .data.i8Power  0x04000428        0x1 ./Common/Command.o
 .data.u8Channel
                0x04000429        0x1 ./Common/Command.o
 .data.u8HwVersion
                0x0400042a        0x1 ./Common/Command.o
 .data.u8SwVersion
                0x0400042b        0x1 ./Common/Command.o
 .data.RadioConfiguration
                0x0400042c       0x54 C:/nxp/SDKPackages/SDK_2.6.0_K32W061DK6/middleware/wireless/framework/XCVR/lib\libRadio_Test_JN518x.a(radio.o)
                0x0400042c                RadioConfiguration
 .data.eCurrentTxMode
                0x04000480        0x1 C:/nxp/SDKPackages/SDK_2.6.0_K32W061DK6/middleware/wireless/framework/XCVR/lib\libRadio_Test_JN518x.a(radio.o)
                0x04000480                eCurrentTxMode
 .data.i8Radio_TxMaxPower
                0x04000481        0x1 C:/nxp/SDKPackages/SDK_2.6.0_K32W061DK6/middleware/wireless/framework/XCVR/lib\libRadio_Test_JN518x.a(radio.o)
                0x04000481                i8Radio_TxMaxPower
 .data.i8Radio_TxMaxPowerCh26
                0x04000482        0x1 C:/nxp/SDKPackages/SDK_2.6.0_K32W061DK6/middleware/wireless/framework/XCVR/lib\libRadio_Test_JN518x.a(radio.o)
                0x04000482                i8Radio_TxMaxPowerCh26
                0x04000484                . = ALIGN (0x4)
 *fill*         0x04000483        0x1 ff
                0x04000484                _edata = .
                0x04000400                __VECTOR_RAM = __VECTOR_RAM__
                0x00000000                __RAM_VECTOR_TABLE_SIZE_BYTES = DEFINED (__ram_vector_table__)?(__interrupts_ram_end__ - __interrupts_ram_start__):0x0

.igot.plt       0x04000484        0x0 load address 0x00007618
 .igot.plt      0x04000484        0x0 ./utilities/MicroInt_arm_sdk2.o

.bss_RAM2       0x04020000        0x0
                [!provide]                PROVIDE (__start_bss_RAM2 = .)
 *(.bss.$RAM2*)
 *(.bss.$RAM1*)
                0x04020000                . = ALIGN ((. != 0x0)?0x4:0x1)
                [!provide]                PROVIDE (__end_bss_RAM2 = .)

.bss            0x04000484      0x1d4
                0x04000484                _bss = .
 *(.bss*)
 .bss.s_debugConsoleState
                0x04000484       0x1c ./utilities/fsl_debug_console.o
 .bss.ctimerCallbackType
                0x040004a0        0x2 ./drivers/fsl_ctimer.o
 *fill*         0x040004a2        0x2 
 .bss.s_ctimerCallback
                0x040004a4        0x8 ./drivers/fsl_ctimer.o
 .bss.s_flexcommHandle
                0x040004ac       0x1c ./drivers/fsl_flexcomm.o
 .bss.s_flexcommIrqHandler
                0x040004c8       0x1c ./drivers/fsl_flexcomm.o
 .bss.warm_start.6992
                0x040004e4        0x1 ./drivers/fsl_power.o
 .bss.bStreamTestRunning
                0x040004e5        0x1 ./Common/Command.o
 *fill*         0x040004e6        0x2 
 .bss.matchConfig0
                0x040004e8        0xc ./Common/Command.o
 .bss.sRxTestReport
                0x040004f4       0x10 ./Common/Command.o
 .bss.bConfiguration
                0x04000504        0x1 C:/nxp/SDKPackages/SDK_2.6.0_K32W061DK6/middleware/wireless/ieee-802.15.4/lib\libMiniMac.a(MMAC.o)
 .bss.bWorkaroundTimerRunning
                0x04000505        0x1 C:/nxp/SDKPackages/SDK_2.6.0_K32W061DK6/middleware/wireless/ieee-802.15.4/lib\libMiniMac.a(MMAC.o)
 *fill*         0x04000506        0x2 
 .bss.prIntHandler
                0x04000508        0x4 C:/nxp/SDKPackages/SDK_2.6.0_K32W061DK6/middleware/wireless/ieee-802.15.4/lib\libMiniMac.a(MMAC.o)
 .bss.prPhyIntHandler
                0x0400050c        0x4 C:/nxp/SDKPackages/SDK_2.6.0_K32W061DK6/middleware/wireless/ieee-802.15.4/lib\libMiniMac.a(MMAC.o)
 .bss.u8MMAC_HpmCcaThreshold
                0x04000510        0x1 C:/nxp/SDKPackages/SDK_2.6.0_K32W061DK6/middleware/wireless/ieee-802.15.4/lib\libMiniMac.a(MMAC.o)
 .bss.u8SctlMask
                0x04000511        0x1 C:/nxp/SDKPackages/SDK_2.6.0_K32W061DK6/middleware/wireless/ieee-802.15.4/lib\libMiniMac.a(MMAC.o)
 .bss.eTxMode   0x04000512        0x1 C:/nxp/SDKPackages/SDK_2.6.0_K32W061DK6/middleware/wireless/framework/XCVR/lib\libRadio_Test_JN518x.a(radio.o)
                0x04000512                eTxMode
 .bss.eTxModeCh26
                0x04000513        0x1 C:/nxp/SDKPackages/SDK_2.6.0_K32W061DK6/middleware/wireless/framework/XCVR/lib\libRadio_Test_JN518x.a(radio.o)
                0x04000513                eTxModeCh26
 .bss.bRunning.21744
                0x04000514        0x1 C:/nxp/SDKPackages/SDK_2.6.0_K32W061DK6/middleware/wireless/framework/XCVR/lib\libRadio_Test_JN518x.a(radio_test_jn518x.o)
 *fill*         0x04000515        0x3 
 .bss.u32PhyMCtrl.21745
                0x04000518        0x4 C:/nxp/SDKPackages/SDK_2.6.0_K32W061DK6/middleware/wireless/framework/XCVR/lib\libRadio_Test_JN518x.a(radio_test_jn518x.o)
 .bss.u32PhyMtxCtrl.21746
                0x0400051c        0x4 C:/nxp/SDKPackages/SDK_2.6.0_K32W061DK6/middleware/wireless/framework/XCVR/lib\libRadio_Test_JN518x.a(radio_test_jn518x.o)
 .bss.vPrivateMacISR
                0x04000520        0x4 C:/nxp/SDKPackages/SDK_2.6.0_K32W061DK6/middleware/wireless/framework/XCVR/lib\libRadio_Test_JN518x.a(radio_test_jn518x.o)
                0x04000520                vPrivateMacISR
 *(COMMON)
 COMMON         0x04000524        0x4 ./utilities/fsl_debug_console.o
                0x04000524                g_serialHandle
 COMMON         0x04000528      0x108 ./Common/Command.o
                0x04000528                sFrame
                0x040005ac                sTFrame
 COMMON         0x04000630       0x28 C:/nxp/SDKPackages/SDK_2.6.0_K32W061DK6/middleware/wireless/framework/XCVR/lib\libRadio_Test_JN518x.a(radio.o)
                0x04000630                u32LnaOffsetGainSav
                0x04000634                tCalTempValues
                0x04000648                u32PhyOn_sav
                0x0400064c                u32XOSlaveSav
                0x04000650                b_event_in_process_patch_on
                0x04000654                u32TempReg
 *(g_u32NwkFrameCounter)
                0x04000658                . = ALIGN (0x4)
                0x04000658                _ebss = .
                [!provide]                PROVIDE (end = .)

.bss_MAC        0x04000658        0x0
                0x04000658                __mac_buffer_start = .
 *(.mac_buffer)
                0x04000658                . = ALIGN ((. != 0x0)?0x4:0x1)

.heap           0x04000658      0x2f4
                0x04000658                _heap = .
                0x0400094c                . = (. + HEAP_SIZE)
 *fill*         0x04000658      0x2f4 
                0x0400094c                . = ALIGN (0x4)
                0x0400094c                _end_heap = .

.noinit_RAM2    0x04020000        0x0
 *(.noinit.$RAM2*)
 *(.noinit.$RAM1*)
                0x04020000                . = ALIGN (0x4)

.noinit         0x0400094c        0x0
                0x0400094c                _noinit = .
 *(.noinit*)
                0x0400094c                . = ALIGN (0x4)
                0x0400094c                _end_noinit = .
                0x0400094c                _end_fw_retention = .

.boot_resume_stack
                0x0400094c      0x400
                0x0400094c                _boot_resume_stack = .
 *(.boot_resume_stack*)
                0x04000d4c                . = (. + BOOT_RESUME_STACK_SIZE)
 *fill*         0x0400094c      0x400 
                0x04000d4c                . = ALIGN (0x4)
                0x04000d4c                _end_boot_resume_stack = .
                [!provide]                PROVIDE (_pvHeapStart = DEFINED (__user_heap_base)?__user_heap_base:_heap)
                [!provide]                PROVIDE (_pvHeapLimit = (_pvHeapStart + HEAP_SIZE))
                0x04015fe0                PROVIDE (_vStackTop = DEFINED (__user_stack_top)?__user_stack_top:(__top_RAM0 - 0x20))
                0x04000000                PROVIDE (__mac_buffer_base = (__mac_buffer_start & 0xfffe0000))
                0x04015000                __StackLimit = (_vStackTop - STACK_SIZE)
                0x00000001                ASSERT ((__StackLimit >= _end_boot_resume_stack), Possible stack corruption with data/bss/boot_stack)
OUTPUT(JN-AN-1255-K32W061-Zigbee_RF_Performance_Test_TISTRP_DUT.elf elf32-littlearm)

.debug_info     0x00000000    0x5c7ae
 .debug_info    0x00000000      0x439 ./utilities/MicroInt_arm_sdk2.o
 .debug_info    0x00000439      0x15a ./utilities/Panic.o
 .debug_info    0x00000593     0x1886 ./utilities/fsl_debug_console.o
 .debug_info    0x00001e19      0xf7e ./utilities/serial_manager.o
 .debug_info    0x00002d97      0x59a ./utilities/serial_port_uart.o
 .debug_info    0x00003331     0x1821 ./utilities/usart_adapter.o
 .debug_info    0x00004b52     0x14d9 ./startup/startup_K32W061.o
 .debug_info    0x0000602b     0x124d ./startup/system_K32W061.o
 .debug_info    0x00007278     0x1a85 ./source/tis_trp_dut.o
 .debug_info    0x00008cfd     0x27b4 ./drivers/fsl_clock.o
 .debug_info    0x0000b4b1     0x22b4 ./drivers/fsl_ctimer.o
 .debug_info    0x0000d765     0x1779 ./drivers/fsl_flexcomm.o
 .debug_info    0x0000eede     0x2742 ./drivers/fsl_power.o
 .debug_info    0x00011620      0xf74 ./drivers/fsl_reset.o
 .debug_info    0x00012594      0x8c1 ./drivers/fsl_str.o
 .debug_info    0x00012e55     0x2588 ./drivers/fsl_usart.o
 .debug_info    0x000153dd     0x1125 ./board/board.o
 .debug_info    0x00016502     0x1293 ./board/hardware_init.o
 .debug_info    0x00017795      0x745 ./board/pin_mux.o
 .debug_info    0x00017eda      0x683 ./Common/CRC.o
 .debug_info    0x0001855d     0x23f9 ./Common/Command.o
 .debug_info    0x0001a956    0x220dc C:/nxp/SDKPackages/SDK_2.6.0_K32W061DK6/middleware/wireless/framework/XCVR/lib\libRadio_Test_JN518x.a(radio.o)
 .debug_info    0x0003ca32    0x1fd7c C:/nxp/SDKPackages/SDK_2.6.0_K32W061DK6/middleware/wireless/framework/XCVR/lib\libRadio_Test_JN518x.a(radio_test_jn518x.o)

.debug_abbrev   0x00000000     0x47f8
 .debug_abbrev  0x00000000      0x1ef ./utilities/MicroInt_arm_sdk2.o
 .debug_abbrev  0x000001ef       0xdc ./utilities/Panic.o
 .debug_abbrev  0x000002cb      0x3a8 ./utilities/fsl_debug_console.o
 .debug_abbrev  0x00000673      0x2ad ./utilities/serial_manager.o
 .debug_abbrev  0x00000920      0x1d4 ./utilities/serial_port_uart.o
 .debug_abbrev  0x00000af4      0x2db ./utilities/usart_adapter.o
 .debug_abbrev  0x00000dcf      0x2ac ./startup/startup_K32W061.o
 .debug_abbrev  0x0000107b      0x2b7 ./startup/system_K32W061.o
 .debug_abbrev  0x00001332      0x358 ./source/tis_trp_dut.o
 .debug_abbrev  0x0000168a      0x489 ./drivers/fsl_clock.o
 .debug_abbrev  0x00001b13      0x4b5 ./drivers/fsl_ctimer.o
 .debug_abbrev  0x00001fc8      0x312 ./drivers/fsl_flexcomm.o
 .debug_abbrev  0x000022da      0x4e9 ./drivers/fsl_power.o
 .debug_abbrev  0x000027c3      0x243 ./drivers/fsl_reset.o
 .debug_abbrev  0x00002a06      0x2bd ./drivers/fsl_str.o
 .debug_abbrev  0x00002cc3      0x4ad ./drivers/fsl_usart.o
 .debug_abbrev  0x00003170      0x240 ./board/board.o
 .debug_abbrev  0x000033b0      0x1da ./board/hardware_init.o
 .debug_abbrev  0x0000358a      0x1e7 ./board/pin_mux.o
 .debug_abbrev  0x00003771      0x1c0 ./Common/CRC.o
 .debug_abbrev  0x00003931      0x4b9 ./Common/Command.o
 .debug_abbrev  0x00003dea      0x4f1 C:/nxp/SDKPackages/SDK_2.6.0_K32W061DK6/middleware/wireless/framework/XCVR/lib\libRadio_Test_JN518x.a(radio.o)
 .debug_abbrev  0x000042db      0x51d C:/nxp/SDKPackages/SDK_2.6.0_K32W061DK6/middleware/wireless/framework/XCVR/lib\libRadio_Test_JN518x.a(radio_test_jn518x.o)

.debug_loc      0x00000000     0xae11
 .debug_loc     0x00000000       0x94 ./utilities/MicroInt_arm_sdk2.o
 .debug_loc     0x00000094      0x6ac ./utilities/fsl_debug_console.o
 .debug_loc     0x00000740      0xefe ./utilities/serial_manager.o
 .debug_loc     0x0000163e      0x308 ./utilities/serial_port_uart.o
 .debug_loc     0x00001946      0x3d8 ./utilities/usart_adapter.o
 .debug_loc     0x00001d1e      0x453 ./startup/startup_K32W061.o
 .debug_loc     0x00002171      0x140 ./startup/system_K32W061.o
 .debug_loc     0x000022b1       0x7f ./source/tis_trp_dut.o
 .debug_loc     0x00002330     0x1120 ./drivers/fsl_clock.o
 .debug_loc     0x00003450      0xc62 ./drivers/fsl_ctimer.o
 .debug_loc     0x000040b2      0x266 ./drivers/fsl_flexcomm.o
 .debug_loc     0x00004318      0x5d4 ./drivers/fsl_power.o
 .debug_loc     0x000048ec      0x25d ./drivers/fsl_reset.o
 .debug_loc     0x00004b49     0x1076 ./drivers/fsl_str.o
 .debug_loc     0x00005bbf     0x125f ./drivers/fsl_usart.o
 .debug_loc     0x00006e1e       0x51 ./board/board.o
 .debug_loc     0x00006e6f      0x230 ./board/pin_mux.o
 .debug_loc     0x0000709f      0x495 ./Common/CRC.o
 .debug_loc     0x00007534      0x5fc ./Common/Command.o
 .debug_loc     0x00007b30     0x2483 C:/nxp/SDKPackages/SDK_2.6.0_K32W061DK6/middleware/wireless/framework/XCVR/lib\libRadio_Test_JN518x.a(radio.o)
 .debug_loc     0x00009fb3      0xe5e C:/nxp/SDKPackages/SDK_2.6.0_K32W061DK6/middleware/wireless/framework/XCVR/lib\libRadio_Test_JN518x.a(radio_test_jn518x.o)

.debug_aranges  0x00000000      0xdf8
 .debug_aranges
                0x00000000       0x28 ./utilities/MicroInt_arm_sdk2.o
 .debug_aranges
                0x00000028       0x28 ./utilities/Panic.o
 .debug_aranges
                0x00000050       0x90 ./utilities/fsl_debug_console.o
 .debug_aranges
                0x000000e0       0x68 ./utilities/serial_manager.o
 .debug_aranges
                0x00000148       0x38 ./utilities/serial_port_uart.o
 .debug_aranges
                0x00000180       0x38 ./utilities/usart_adapter.o
 .debug_aranges
                0x000001b8      0x128 ./startup/startup_K32W061.o
 .debug_aranges
                0x000002e0       0x28 ./startup/system_K32W061.o
 .debug_aranges
                0x00000308       0x38 ./source/tis_trp_dut.o
 .debug_aranges
                0x00000340      0x148 ./drivers/fsl_clock.o
 .debug_aranges
                0x00000488       0x80 ./drivers/fsl_ctimer.o
 .debug_aranges
                0x00000508       0x68 ./drivers/fsl_flexcomm.o
 .debug_aranges
                0x00000570       0x90 ./drivers/fsl_power.o
 .debug_aranges
                0x00000600       0x38 ./drivers/fsl_reset.o
 .debug_aranges
                0x00000638       0x30 ./drivers/fsl_str.o
 .debug_aranges
                0x00000668       0xb0 ./drivers/fsl_usart.o
 .debug_aranges
                0x00000718       0x30 ./board/board.o
 .debug_aranges
                0x00000748       0x28 ./board/hardware_init.o
 .debug_aranges
                0x00000770       0x20 ./board/pin_mux.o
 .debug_aranges
                0x00000790       0x68 ./Common/CRC.o
 .debug_aranges
                0x000007f8       0x50 ./Common/Command.o
 .debug_aranges
                0x00000848      0x3b0 C:/nxp/SDKPackages/SDK_2.6.0_K32W061DK6/middleware/wireless/framework/XCVR/lib\libRadio_Test_JN518x.a(radio.o)
 .debug_aranges
                0x00000bf8      0x200 C:/nxp/SDKPackages/SDK_2.6.0_K32W061DK6/middleware/wireless/framework/XCVR/lib\libRadio_Test_JN518x.a(radio_test_jn518x.o)

.debug_ranges   0x00000000     0x1198
 .debug_ranges  0x00000000       0x30 ./utilities/MicroInt_arm_sdk2.o
 .debug_ranges  0x00000030       0x18 ./utilities/Panic.o
 .debug_ranges  0x00000048       0x98 ./utilities/fsl_debug_console.o
 .debug_ranges  0x000000e0      0x170 ./utilities/serial_manager.o
 .debug_ranges  0x00000250       0x28 ./utilities/serial_port_uart.o
 .debug_ranges  0x00000278       0x28 ./utilities/usart_adapter.o
 .debug_ranges  0x000002a0      0x160 ./startup/startup_K32W061.o
 .debug_ranges  0x00000400       0x70 ./startup/system_K32W061.o
 .debug_ranges  0x00000470       0x28 ./source/tis_trp_dut.o
 .debug_ranges  0x00000498      0x150 ./drivers/fsl_clock.o
 .debug_ranges  0x000005e8       0xe8 ./drivers/fsl_ctimer.o
 .debug_ranges  0x000006d0       0x90 ./drivers/fsl_flexcomm.o
 .debug_ranges  0x00000760       0xc8 ./drivers/fsl_power.o
 .debug_ranges  0x00000828       0x28 ./drivers/fsl_reset.o
 .debug_ranges  0x00000850       0x68 ./drivers/fsl_str.o
 .debug_ranges  0x000008b8      0x118 ./drivers/fsl_usart.o
 .debug_ranges  0x000009d0       0x20 ./board/board.o
 .debug_ranges  0x000009f0       0x18 ./board/hardware_init.o
 .debug_ranges  0x00000a08       0x68 ./board/pin_mux.o
 .debug_ranges  0x00000a70       0x58 ./Common/CRC.o
 .debug_ranges  0x00000ac8      0x128 ./Common/Command.o
 .debug_ranges  0x00000bf0      0x3b8 C:/nxp/SDKPackages/SDK_2.6.0_K32W061DK6/middleware/wireless/framework/XCVR/lib\libRadio_Test_JN518x.a(radio.o)
 .debug_ranges  0x00000fa8      0x1f0 C:/nxp/SDKPackages/SDK_2.6.0_K32W061DK6/middleware/wireless/framework/XCVR/lib\libRadio_Test_JN518x.a(radio_test_jn518x.o)

.debug_line     0x00000000     0xf6aa
 .debug_line    0x00000000      0x322 ./utilities/MicroInt_arm_sdk2.o
 .debug_line    0x00000322      0x28c ./utilities/Panic.o
 .debug_line    0x000005ae      0x85f ./utilities/fsl_debug_console.o
 .debug_line    0x00000e0d      0x892 ./utilities/serial_manager.o
 .debug_line    0x0000169f      0x3d6 ./utilities/serial_port_uart.o
 .debug_line    0x00001a75      0x480 ./utilities/usart_adapter.o
 .debug_line    0x00001ef5      0x78b ./startup/startup_K32W061.o
 .debug_line    0x00002680      0x34e ./startup/system_K32W061.o
 .debug_line    0x000029ce      0x554 ./source/tis_trp_dut.o
 .debug_line    0x00002f22      0xff5 ./drivers/fsl_clock.o
 .debug_line    0x00003f17      0x905 ./drivers/fsl_ctimer.o
 .debug_line    0x0000481c      0x521 ./drivers/fsl_flexcomm.o
 .debug_line    0x00004d3d      0xd0b ./drivers/fsl_power.o
 .debug_line    0x00005a48      0x3af ./drivers/fsl_reset.o
 .debug_line    0x00005df7      0xa47 ./drivers/fsl_str.o
 .debug_line    0x0000683e      0xf74 ./drivers/fsl_usart.o
 .debug_line    0x000077b2      0x3a4 ./board/board.o
 .debug_line    0x00007b56      0x31f ./board/hardware_init.o
 .debug_line    0x00007e75      0x378 ./board/pin_mux.o
 .debug_line    0x000081ed      0x3be ./Common/CRC.o
 .debug_line    0x000085ab      0x92c ./Common/Command.o
 .debug_line    0x00008ed7     0x4601 C:/nxp/SDKPackages/SDK_2.6.0_K32W061DK6/middleware/wireless/framework/XCVR/lib\libRadio_Test_JN518x.a(radio.o)
 .debug_line    0x0000d4d8     0x21d2 C:/nxp/SDKPackages/SDK_2.6.0_K32W061DK6/middleware/wireless/framework/XCVR/lib\libRadio_Test_JN518x.a(radio_test_jn518x.o)

.debug_str      0x00000000   0x160605
 .debug_str     0x00000000      0x37a ./utilities/MicroInt_arm_sdk2.o
                                0x41e (size before relaxing)
 .debug_str     0x0000037a       0x97 ./utilities/Panic.o
                                0x2af (size before relaxing)
 .debug_str     0x00000411     0x1566 ./utilities/fsl_debug_console.o
                               0x192a (size before relaxing)
 .debug_str     0x00001977      0x2a3 ./utilities/serial_manager.o
                                0x810 (size before relaxing)
 .debug_str     0x00001c1a      0x2d9 ./utilities/serial_port_uart.o
                                0x836 (size before relaxing)
 .debug_str     0x00001ef3      0x7b2 ./utilities/usart_adapter.o
                               0x1cf5 (size before relaxing)
 .debug_str     0x000026a5      0x56c ./startup/startup_K32W061.o
                                0xe21 (size before relaxing)
 .debug_str     0x00002c11      0x28d ./startup/system_K32W061.o
                                0xc1f (size before relaxing)
 .debug_str     0x00002e9e      0x3b4 ./source/tis_trp_dut.o
                               0x1a9e (size before relaxing)
 .debug_str     0x00003252     0x1349 ./drivers/fsl_clock.o
                               0x271b (size before relaxing)
 .debug_str     0x0000459b      0x8aa ./drivers/fsl_ctimer.o
                               0x2220 (size before relaxing)
 .debug_str     0x00004e45      0x288 ./drivers/fsl_flexcomm.o
                               0x1b25 (size before relaxing)
 .debug_str     0x000050cd      0x667 ./drivers/fsl_power.o
                               0x2779 (size before relaxing)
 .debug_str     0x00005734       0xd7 ./drivers/fsl_reset.o
                                0xdd9 (size before relaxing)
 .debug_str     0x0000580b      0x1c7 ./drivers/fsl_str.o
                                0x452 (size before relaxing)
 .debug_str     0x000059d2      0x5b9 ./drivers/fsl_usart.o
                               0x21e1 (size before relaxing)
 .debug_str     0x00005f8b       0xa4 ./board/board.o
                               0x1622 (size before relaxing)
 .debug_str     0x0000602f       0x39 ./board/hardware_init.o
                               0x15c0 (size before relaxing)
 .debug_str     0x00006068       0x54 ./board/pin_mux.o
                                0x946 (size before relaxing)
 .debug_str     0x000060bc       0xfc ./Common/CRC.o
                                0x3af (size before relaxing)
 .debug_str     0x000061b8      0x56b ./Common/Command.o
                               0x24f7 (size before relaxing)
 .debug_str     0x00006723   0x158f43 C:/nxp/SDKPackages/SDK_2.6.0_K32W061DK6/middleware/wireless/framework/XCVR/lib\libRadio_Test_JN518x.a(radio.o)
                             0x15d4a2 (size before relaxing)
 .debug_str     0x0015f666      0xf9f C:/nxp/SDKPackages/SDK_2.6.0_K32W061DK6/middleware/wireless/framework/XCVR/lib\libRadio_Test_JN518x.a(radio_test_jn518x.o)
                             0x158d5e (size before relaxing)

.comment        0x00000000       0x76
 .comment       0x00000000       0x76 ./utilities/MicroInt_arm_sdk2.o
                                 0x77 (size before relaxing)
 .comment       0x00000076       0x77 ./utilities/Panic.o
 .comment       0x00000076       0x77 ./utilities/fsl_debug_console.o
 .comment       0x00000076       0x77 ./utilities/serial_manager.o
 .comment       0x00000076       0x77 ./utilities/serial_port_uart.o
 .comment       0x00000076       0x77 ./utilities/usart_adapter.o
 .comment       0x00000076       0x77 ./startup/startup_K32W061.o
 .comment       0x00000076       0x77 ./startup/system_K32W061.o
 .comment       0x00000076       0x77 ./source/tis_trp_dut.o
 .comment       0x00000076       0x77 ./drivers/fsl_clock.o
 .comment       0x00000076       0x77 ./drivers/fsl_ctimer.o
 .comment       0x00000076       0x77 ./drivers/fsl_flexcomm.o
 .comment       0x00000076       0x77 ./drivers/fsl_power.o
 .comment       0x00000076       0x77 ./drivers/fsl_reset.o
 .comment       0x00000076       0x77 ./drivers/fsl_str.o
 .comment       0x00000076       0x77 ./drivers/fsl_usart.o
 .comment       0x00000076       0x77 ./board/board.o
 .comment       0x00000076       0x77 ./board/hardware_init.o
 .comment       0x00000076       0x77 ./board/pin_mux.o
 .comment       0x00000076       0x77 ./Common/CRC.o
 .comment       0x00000076       0x77 ./Common/Command.o
 .comment       0x00000076       0x77 C:/nxp/SDKPackages/SDK_2.6.0_K32W061DK6/middleware/wireless/ieee-802.15.4/lib\libMiniMac.a(MMAC.o)
 .comment       0x00000076       0x77 C:/nxp/SDKPackages/SDK_2.6.0_K32W061DK6/middleware/wireless/ieee-802.15.4/lib\libMiniMac.a(MMAC_RadioInit_JN518x.o)
 .comment       0x00000076       0x77 C:/nxp/SDKPackages/SDK_2.6.0_K32W061DK6/middleware/wireless/framework/XCVR/lib\libRadio_Test_JN518x.a(radio.o)
 .comment       0x00000076       0x77 C:/nxp/SDKPackages/SDK_2.6.0_K32W061DK6/middleware/wireless/framework/XCVR/lib\libRadio_Test_JN518x.a(radio_test_jn518x.o)

.ARM.attributes
                0x00000000       0x2c
 .ARM.attributes
                0x00000000       0x2e ./utilities/MicroInt_arm_sdk2.o
 .ARM.attributes
                0x0000002e       0x2e ./utilities/Panic.o
 .ARM.attributes
                0x0000005c       0x2e ./utilities/fsl_debug_console.o
 .ARM.attributes
                0x0000008a       0x2e ./utilities/serial_manager.o
 .ARM.attributes
                0x000000b8       0x2e ./utilities/serial_port_uart.o
 .ARM.attributes
                0x000000e6       0x2e ./utilities/usart_adapter.o
 .ARM.attributes
                0x00000114       0x2e ./startup/startup_K32W061.o
 .ARM.attributes
                0x00000142       0x2e ./startup/system_K32W061.o
 .ARM.attributes
                0x00000170       0x2e ./source/tis_trp_dut.o
 .ARM.attributes
                0x0000019e       0x2e ./drivers/fsl_clock.o
 .ARM.attributes
                0x000001cc       0x2e ./drivers/fsl_ctimer.o
 .ARM.attributes
                0x000001fa       0x2e ./drivers/fsl_flexcomm.o
 .ARM.attributes
                0x00000228       0x2e ./drivers/fsl_power.o
 .ARM.attributes
                0x00000256       0x2e ./drivers/fsl_reset.o
 .ARM.attributes
                0x00000284       0x2e ./drivers/fsl_str.o
 .ARM.attributes
                0x000002b2       0x2e ./drivers/fsl_usart.o
 .ARM.attributes
                0x000002e0       0x2e ./board/board.o
 .ARM.attributes
                0x0000030e       0x2e ./board/hardware_init.o
 .ARM.attributes
                0x0000033c       0x2e ./board/pin_mux.o
 .ARM.attributes
                0x0000036a       0x2e ./Common/CRC.o
 .ARM.attributes
                0x00000398       0x2e ./Common/Command.o
 .ARM.attributes
                0x000003c6       0x2e C:/nxp/SDKPackages/SDK_2.6.0_K32W061DK6/middleware/wireless/ieee-802.15.4/lib\libMiniMac.a(MMAC.o)
 .ARM.attributes
                0x000003f4       0x2e C:/nxp/SDKPackages/SDK_2.6.0_K32W061DK6/middleware/wireless/ieee-802.15.4/lib\libMiniMac.a(MMAC_RadioInit_JN518x.o)
 .ARM.attributes
                0x00000422       0x2e C:/nxp/SDKPackages/SDK_2.6.0_K32W061DK6/middleware/wireless/framework/XCVR/lib\libRadio_Test_JN518x.a(radio.o)
 .ARM.attributes
                0x00000450       0x2e C:/nxp/SDKPackages/SDK_2.6.0_K32W061DK6/middleware/wireless/framework/XCVR/lib\libRadio_Test_JN518x.a(radio_test_jn518x.o)
 .ARM.attributes
                0x0000047e       0x1e c:/nxp/mcuxpressoide_11.1.0_3209/ide/plugins/com.nxp.mcuxpresso.tools.win32_11.1.0.201909161352/tools/bin/../lib/gcc/arm-none-eabi/8.3.1/thumb/v7e-m/nofp\libgcc.a(_arm_addsubdf3.o)
 .ARM.attributes
                0x0000049c       0x1e c:/nxp/mcuxpressoide_11.1.0_3209/ide/plugins/com.nxp.mcuxpresso.tools.win32_11.1.0.201909161352/tools/bin/../lib/gcc/arm-none-eabi/8.3.1/thumb/v7e-m/nofp\libgcc.a(_arm_fixdfsi.o)
 .ARM.attributes
                0x000004ba       0x1e c:/nxp/mcuxpressoide_11.1.0_3209/ide/plugins/com.nxp.mcuxpresso.tools.win32_11.1.0.201909161352/tools/bin/../lib/gcc/arm-none-eabi/8.3.1/thumb/v7e-m/nofp\libgcc.a(_aeabi_uldivmod.o)
 .ARM.attributes
                0x000004d8       0x2e c:/nxp/mcuxpressoide_11.1.0_3209/ide/plugins/com.nxp.mcuxpresso.tools.win32_11.1.0.201909161352/tools/bin/../lib/gcc/arm-none-eabi/8.3.1/thumb/v7e-m/nofp\libgcc.a(_udivmoddi4.o)
 .ARM.attributes
                0x00000506       0x1e c:/nxp/mcuxpressoide_11.1.0_3209/ide/plugins/com.nxp.mcuxpresso.tools.win32_11.1.0.201909161352/tools/bin/../lib/gcc/arm-none-eabi/8.3.1/thumb/v7e-m/nofp\libgcc.a(_dvmd_tls.o)
 .ARM.attributes
                0x00000524       0x2e c:/nxp/mcuxpressoide_11.1.0_3209/ide/plugins/com.nxp.mcuxpresso.tools.win32_11.1.0.201909161352/tools/bin/../lib/gcc/arm-none-eabi/8.3.1/../../../../arm-none-eabi/lib/thumb/v7e-m/nofp\libg.a(lib_a-abs.o)
 .ARM.attributes
                0x00000552       0x1c c:/nxp/mcuxpressoide_11.1.0_3209/ide/plugins/com.nxp.mcuxpresso.tools.win32_11.1.0.201909161352/tools/bin/../lib/gcc/arm-none-eabi/8.3.1/../../../../arm-none-eabi/lib/thumb/v7e-m/nofp\libg.a(lib_a-memcpy.o)
 .ARM.attributes
                0x0000056e       0x2e c:/nxp/mcuxpressoide_11.1.0_3209/ide/plugins/com.nxp.mcuxpresso.tools.win32_11.1.0.201909161352/tools/bin/../lib/gcc/arm-none-eabi/8.3.1/../../../../arm-none-eabi/lib/thumb/v7e-m/nofp\libg.a(lib_a-memset.o)
 .ARM.attributes
                0x0000059c       0x1c c:/nxp/mcuxpressoide_11.1.0_3209/ide/plugins/com.nxp.mcuxpresso.tools.win32_11.1.0.201909161352/tools/bin/../lib/gcc/arm-none-eabi/8.3.1/../../../../arm-none-eabi/lib/thumb/v7e-m/nofp\libg.a(lib_a-strlen.o)

.debug_frame    0x00000000     0x2650
 .debug_frame   0x00000000       0x30 ./utilities/MicroInt_arm_sdk2.o
 .debug_frame   0x00000030       0x30 ./utilities/Panic.o
 .debug_frame   0x00000060      0x1c8 ./utilities/fsl_debug_console.o
 .debug_frame   0x00000228      0x128 ./utilities/serial_manager.o
 .debug_frame   0x00000350       0x78 ./utilities/serial_port_uart.o
 .debug_frame   0x000003c8       0x7c ./utilities/usart_adapter.o
 .debug_frame   0x00000444      0x33c ./startup/startup_K32W061.o
 .debug_frame   0x00000780       0x38 ./startup/system_K32W061.o
 .debug_frame   0x000007b8       0x68 ./source/tis_trp_dut.o
 .debug_frame   0x00000820      0x354 ./drivers/fsl_clock.o
 .debug_frame   0x00000b74      0x178 ./drivers/fsl_ctimer.o
 .debug_frame   0x00000cec      0x108 ./drivers/fsl_flexcomm.o
 .debug_frame   0x00000df4      0x178 ./drivers/fsl_power.o
 .debug_frame   0x00000f6c       0x6c ./drivers/fsl_reset.o
 .debug_frame   0x00000fd8       0x78 ./drivers/fsl_str.o
 .debug_frame   0x00001050      0x208 ./drivers/fsl_usart.o
 .debug_frame   0x00001258       0x48 ./board/board.o
 .debug_frame   0x000012a0       0x48 ./board/hardware_init.o
 .debug_frame   0x000012e8       0x2c ./board/pin_mux.o
 .debug_frame   0x00001314       0xfc ./Common/CRC.o
 .debug_frame   0x00001410       0xfc ./Common/Command.o
 .debug_frame   0x0000150c      0xa80 C:/nxp/SDKPackages/SDK_2.6.0_K32W061DK6/middleware/wireless/framework/XCVR/lib\libRadio_Test_JN518x.a(radio.o)
 .debug_frame   0x00001f8c      0x53c C:/nxp/SDKPackages/SDK_2.6.0_K32W061DK6/middleware/wireless/framework/XCVR/lib\libRadio_Test_JN518x.a(radio_test_jn518x.o)
 .debug_frame   0x000024c8       0xac c:/nxp/mcuxpressoide_11.1.0_3209/ide/plugins/com.nxp.mcuxpresso.tools.win32_11.1.0.201909161352/tools/bin/../lib/gcc/arm-none-eabi/8.3.1/thumb/v7e-m/nofp\libgcc.a(_arm_addsubdf3.o)
 .debug_frame   0x00002574       0x24 c:/nxp/mcuxpressoide_11.1.0_3209/ide/plugins/com.nxp.mcuxpresso.tools.win32_11.1.0.201909161352/tools/bin/../lib/gcc/arm-none-eabi/8.3.1/thumb/v7e-m/nofp\libgcc.a(_arm_fixdfsi.o)
 .debug_frame   0x00002598       0x2c c:/nxp/mcuxpressoide_11.1.0_3209/ide/plugins/com.nxp.mcuxpresso.tools.win32_11.1.0.201909161352/tools/bin/../lib/gcc/arm-none-eabi/8.3.1/thumb/v7e-m/nofp\libgcc.a(_aeabi_uldivmod.o)
 .debug_frame   0x000025c4       0x34 c:/nxp/mcuxpressoide_11.1.0_3209/ide/plugins/com.nxp.mcuxpresso.tools.win32_11.1.0.201909161352/tools/bin/../lib/gcc/arm-none-eabi/8.3.1/thumb/v7e-m/nofp\libgcc.a(_udivmoddi4.o)
 .debug_frame   0x000025f8       0x20 c:/nxp/mcuxpressoide_11.1.0_3209/ide/plugins/com.nxp.mcuxpresso.tools.win32_11.1.0.201909161352/tools/bin/../lib/gcc/arm-none-eabi/8.3.1/../../../../arm-none-eabi/lib/thumb/v7e-m/nofp\libg.a(lib_a-abs.o)
 .debug_frame   0x00002618       0x38 c:/nxp/mcuxpressoide_11.1.0_3209/ide/plugins/com.nxp.mcuxpresso.tools.win32_11.1.0.201909161352/tools/bin/../lib/gcc/arm-none-eabi/8.3.1/../../../../arm-none-eabi/lib/thumb/v7e-m/nofp\libg.a(lib_a-memset.o)

.debug_macro    0x00000000    0x28ebe
 .debug_macro   0x00000000      0x5ec C:/nxp/SDKPackages/SDK_2.6.0_K32W061DK6/middleware/wireless/framework/XCVR/lib\libRadio_Test_JN518x.a(radio.o)
 .debug_macro   0x000005ec      0xaa8 C:/nxp/SDKPackages/SDK_2.6.0_K32W061DK6/middleware/wireless/framework/XCVR/lib\libRadio_Test_JN518x.a(radio.o)
 .debug_macro   0x00001094       0x16 C:/nxp/SDKPackages/SDK_2.6.0_K32W061DK6/middleware/wireless/framework/XCVR/lib\libRadio_Test_JN518x.a(radio.o)
 .debug_macro   0x000010aa       0x38 C:/nxp/SDKPackages/SDK_2.6.0_K32W061DK6/middleware/wireless/framework/XCVR/lib\libRadio_Test_JN518x.a(radio.o)
 .debug_macro   0x000010e2       0x10 C:/nxp/SDKPackages/SDK_2.6.0_K32W061DK6/middleware/wireless/framework/XCVR/lib\libRadio_Test_JN518x.a(radio.o)
 .debug_macro   0x000010f2      0x12e C:/nxp/SDKPackages/SDK_2.6.0_K32W061DK6/middleware/wireless/framework/XCVR/lib\libRadio_Test_JN518x.a(radio.o)
 .debug_macro   0x00001220      0x5b3 C:/nxp/SDKPackages/SDK_2.6.0_K32W061DK6/middleware/wireless/framework/XCVR/lib\libRadio_Test_JN518x.a(radio.o)
 .debug_macro   0x000017d3       0x1c C:/nxp/SDKPackages/SDK_2.6.0_K32W061DK6/middleware/wireless/framework/XCVR/lib\libRadio_Test_JN518x.a(radio.o)
 .debug_macro   0x000017ef       0x22 C:/nxp/SDKPackages/SDK_2.6.0_K32W061DK6/middleware/wireless/framework/XCVR/lib\libRadio_Test_JN518x.a(radio.o)
 .debug_macro   0x00001811       0xdf C:/nxp/SDKPackages/SDK_2.6.0_K32W061DK6/middleware/wireless/framework/XCVR/lib\libRadio_Test_JN518x.a(radio.o)
 .debug_macro   0x000018f0      0xff5 C:/nxp/SDKPackages/SDK_2.6.0_K32W061DK6/middleware/wireless/framework/XCVR/lib\libRadio_Test_JN518x.a(radio.o)
 .debug_macro   0x000028e5       0xe2 C:/nxp/SDKPackages/SDK_2.6.0_K32W061DK6/middleware/wireless/framework/XCVR/lib\libRadio_Test_JN518x.a(radio.o)
 .debug_macro   0x000029c7       0x10 C:/nxp/SDKPackages/SDK_2.6.0_K32W061DK6/middleware/wireless/framework/XCVR/lib\libRadio_Test_JN518x.a(radio.o)
 .debug_macro   0x000029d7     0x9cc0 C:/nxp/SDKPackages/SDK_2.6.0_K32W061DK6/middleware/wireless/framework/XCVR/lib\libRadio_Test_JN518x.a(radio.o)
 .debug_macro   0x0000c697      0x213 C:/nxp/SDKPackages/SDK_2.6.0_K32W061DK6/middleware/wireless/framework/XCVR/lib\libRadio_Test_JN518x.a(radio.o)
 .debug_macro   0x0000c8aa       0x16 C:/nxp/SDKPackages/SDK_2.6.0_K32W061DK6/middleware/wireless/framework/XCVR/lib\libRadio_Test_JN518x.a(radio.o)
 .debug_macro   0x0000c8c0       0x22 C:/nxp/SDKPackages/SDK_2.6.0_K32W061DK6/middleware/wireless/framework/XCVR/lib\libRadio_Test_JN518x.a(radio.o)
 .debug_macro   0x0000c8e2       0x22 C:/nxp/SDKPackages/SDK_2.6.0_K32W061DK6/middleware/wireless/framework/XCVR/lib\libRadio_Test_JN518x.a(radio.o)
 .debug_macro   0x0000c904       0xd0 C:/nxp/SDKPackages/SDK_2.6.0_K32W061DK6/middleware/wireless/framework/XCVR/lib\libRadio_Test_JN518x.a(radio.o)
 .debug_macro   0x0000c9d4       0xbc C:/nxp/SDKPackages/SDK_2.6.0_K32W061DK6/middleware/wireless/framework/XCVR/lib\libRadio_Test_JN518x.a(radio.o)
 .debug_macro   0x0000ca90       0xa9 C:/nxp/SDKPackages/SDK_2.6.0_K32W061DK6/middleware/wireless/framework/XCVR/lib\libRadio_Test_JN518x.a(radio.o)
 .debug_macro   0x0000cb39       0xcf C:/nxp/SDKPackages/SDK_2.6.0_K32W061DK6/middleware/wireless/framework/XCVR/lib\libRadio_Test_JN518x.a(radio.o)
 .debug_macro   0x0000cc08       0x10 C:/nxp/SDKPackages/SDK_2.6.0_K32W061DK6/middleware/wireless/framework/XCVR/lib\libRadio_Test_JN518x.a(radio.o)
 .debug_macro   0x0000cc18      0x398 C:/nxp/SDKPackages/SDK_2.6.0_K32W061DK6/middleware/wireless/framework/XCVR/lib\libRadio_Test_JN518x.a(radio.o)
 .debug_macro   0x0000cfb0      0x4f6 C:/nxp/SDKPackages/SDK_2.6.0_K32W061DK6/middleware/wireless/framework/XCVR/lib\libRadio_Test_JN518x.a(radio.o)
 .debug_macro   0x0000d4a6      0x494 C:/nxp/SDKPackages/SDK_2.6.0_K32W061DK6/middleware/wireless/framework/XCVR/lib\libRadio_Test_JN518x.a(radio.o)
 .debug_macro   0x0000d93a     0xddcb C:/nxp/SDKPackages/SDK_2.6.0_K32W061DK6/middleware/wireless/framework/XCVR/lib\libRadio_Test_JN518x.a(radio.o)
 .debug_macro   0x0001b705     0xd2d4 C:/nxp/SDKPackages/SDK_2.6.0_K32W061DK6/middleware/wireless/framework/XCVR/lib\libRadio_Test_JN518x.a(radio.o)
 .debug_macro   0x000289d9      0x150 C:/nxp/SDKPackages/SDK_2.6.0_K32W061DK6/middleware/wireless/framework/XCVR/lib\libRadio_Test_JN518x.a(radio.o)
 .debug_macro   0x00028b29       0xff C:/nxp/SDKPackages/SDK_2.6.0_K32W061DK6/middleware/wireless/framework/XCVR/lib\libRadio_Test_JN518x.a(radio.o)
 .debug_macro   0x00028c28      0x27a C:/nxp/SDKPackages/SDK_2.6.0_K32W061DK6/middleware/wireless/framework/XCVR/lib\libRadio_Test_JN518x.a(radio_test_jn518x.o)
 .debug_macro   0x00028ea2       0x1c C:/nxp/SDKPackages/SDK_2.6.0_K32W061DK6/middleware/wireless/framework/XCVR/lib\libRadio_Test_JN518x.a(radio_test_jn518x.o)
